:100000000C94DC310C940D320C940D320C940D32A6
:100010000C940D320C949D8B0C940D320C940D327B
:100020000C94898E0C940D320C940D320D94695DF4
:100030000C940D320D946E3A0C940D320C940D32DA
:100040000C940D320D943A700C940D320C940D32C8
:100050000C940D320C940D320C9424DC0D941F3C46
:100060000C940D320C94929B0C940D320C940D3226
:100070000C940D320C940D320C940D320C940D3204
:100080000C940D320C940D320C940D320C940D32F4
:100090000C944E9B0C940D320C940D320C940D323A
:1000A0000C940D320C940D320C940D320C940D32D4
:1000B0000C940D320C940D320C940D320C940D32C4
:1000C0000C940D320C940D320C940D320C940D32B4
:1000D0000C940D320C940D320C940D320C940D32A4
:1000E0000C940D323240354038403B403E40414058
:1000F0004440DE40114146417941AC41DF4112426A
:10010000C49FC89FCD9FD59FEA9F03A02EA05BA050
:1001100008AA1FAA33AA49AA5AAA88AAA4AA5CAB09
:1001200088AB98ABB5ABD3AB01AC09AC11AC11AC9F
:1001300011AC37AC37AC37AC19AC47AC37AC23ACEF
:1001400036019C0186016C0180014E01A2015E0115
:1001500054019A0146018401620158014E01420195
:100160004A013C018A01A00176018E016601560117
:100170005A0164016A014C019E01A40144018201FB
:1001800056013E01A601A801AA01600152017401B5
:1001900088013A0172016E01900178017C01084AE0
:1001A000D73B3BCE016E84BCBFFDC12F3D6C74318B
:1001B0009ABD56833DDA3D00C77F11BED9E4BB4CE2
:1001C0003E916BAAAABE000000803F05A84CCDB2AC
:1001D000D44EB93836A9020C50B9918688083CA68D
:1001E000AAAA2ABE000000803F07634236B79BD808
:1001F000A71A39685618AEBAAB558C1D3CB7CC5708
:1002000063BD6DEDFD753EF6177231BF00000080D5
:100210003F08000000BE922449123EABAAAA2ABEA3
:10022000CDCCCC4C3E00000080BEABAAAAAA3E00BA
:10023000000000BF000000803F00000000000841F7
:1002400078D3BB4387D1133D190E3CC3BD4282AD69
:100250002B3E68EC8276BED98FE1A93E4C80EFFF41
:10026000BE01C4FF7F3F0000000000000D945C3918
:100270000D94BC390D9465610D9491390D94A93B91
:100280000D9488A10D9489390D94953B0D94753981
:100290000D9478830D948D390D94723B0D9496399D
:1002A0000D9454210D9417610D946D390D94C73B35
:1002B0000D9483390D94583B0D94921D0D9467391C
:1002C0000D9410610D947F390D94603B0D944E3B5D
:1002D0000D9416390D94683B0D9452390D948E612E
:1002E0000D94FA890D9471610D9435610D943A3B2A
:1002F0000D94C3610D94FE020D94EF610D94178966
:100300000D9458390D949F3B0D947B390D944E39C3
:100310000D945E610D94303B0D9437920D94443BE7
:100320000D94A6610D946C7F0D949E850D94AF9FE6
:100330000D94FF8D0D9471390D945F390D947C3BB4
:100340000D94353B0D9463390D94863B0D94B33B6E
:100350000D94BD3B0D94F8604E414E494E495459A1
:10036000494E46CDCCCC3D0AD7233C17B7D1387780
:10037000CC2B329595E6241FB14F0A000020410096
:1003800000C84200401C4620BCBE4CCA1B0E5AAEE0
:10039000C59D7400407A10F35A00A0724E180900EF
:1003A00010A5D4E80000E87648170000E40B5402DA
:1003B0000000CA9A3B000000E1F505000080969815
:1003C00000000040420F000000A086010000001065
:1003D0002700000000E803000000006400000000A7
:1003E000000A00000000000100000000002C76D888
:1003F00088DC674F0823DFC1DFAE59E1B1B796E56E
:10040000E3E453C63AE651997696E8E6C28426EBD1
:10041000898C9B62ED407C6FFCEFBC9C9F40F2BAE4
:10042000A56FA5F490055A2AF75C936B6CF9676D7C
:10043000C11BFCE0E40D47FEF520E6B500D0ED90D1
:100440002E0300943577050080841E080000204E9E
:100450000A000000C80C333333330F986E12831137
:1004600041EF8D2114893BE65516CFFEE6DB18D10E
:10047000844B381BF77C1D901DA4BBE424203284E0
:10048000725E228100C9F124ECA1E53D2744657428
:10049000656B6F76616E206E6172617A2E004372B9
:1004A0006173682064657465637465642E005344E9
:1004B000207072696E74696E6720627974652000BD
:1004C00050726F73696D20616B7475616C697A75B8
:1004D0006A74652E00506C65617365207570677273
:1004E0006164652E005679736C61206E6F766120B1
:1004F0007665727A65206669726D776172653A0019
:100500004E6577206669726D7761726520766572D7
:1005100073696F6E20617661696C61626C653A0027
:100520006120737469736B6E65746520746C6163AC
:1005300069746B6F00616E642070726573732074F0
:100540006865206B6E6F6200566C6F7A746520660A
:10055000696C616D656E7400496E736572742066B6
:10056000696C616D656E74004261727661206E65C2
:100570006E6920636973746100436F6C6F72206EE3
:100580006F7420636F72726563740046696C616D8D
:10059000656E74206E657A61766564656E00466985
:1005A0006C616D656E74206E6F74206C6F61646534
:1005B000640056796D656E61206F6B3F0043686122
:1005C0006E67656420636F72726563746C793F0057
:1005D00043697374656E69206261727679004C6F4D
:1005E0006164696E6720636F6C6F72005A6D656E2F
:1005F000612075737065736E6121004368616E6779
:100600006520737563636573732100457874727533
:1006100064657200567962657274652065787472DB
:10062000756465723A0043686F6F7365206578740E
:1006300072756465723A0041637469766520457825
:100640007472756465723A2000496E76616C6964F3
:100650002065787472756465720050726F73696D8D
:10066000206F746576726574652069646C657220AC
:1006700061206D616E75616C6E65206F647374725C
:10068000616E74652066696C616D656E742E0050D4
:100690006C65617365206F70656E2069646C65724E
:1006A00020616E642072656D6F76652066696C618D
:1006B0006D656E74206D616E75616C6C792E004293
:1006C000796C6F20767973756E7574692066696CC4
:1006D000616D656E74752075737065736E653F002E
:1006E0005761732066696C616D656E7420756E6C00
:1006F0006F6164207375636365737366756C3F0027
:1007000050726F73696D2076796A6D6574652075B6
:10071000727963686C656E652066696C616D656E83
:100720007400506C656173652070756C6C206F751A
:10073000742066696C616D656E7420696D6D6564A9
:10074000696174656C79005679736F7576616D2097
:1007500066696C616D656E7400556E6C6F6164697D
:100760006E672066696C616D656E740050726F20F3
:100770006E61687261746920747279736B7920613B
:1007800020706F6B7261636F76616E69207374693C
:10079000736B6E65746520746C616369746B6F2E26
:1007A000005072657373206B6E6F6220746F2070DF
:1007B000726568656174206E6F7A7A6C6520616E0F
:1007C0006420636F6E74696E75652E0050726F20C1
:1007D000767973756E7574692066696C616D656E86
:1007E000747520737469736B6E6574652070726FB5
:1007F00073696D20746C616369746B6F00506C6514
:1008000061736520707265737320746865206B6E08
:100810006F6220746F20756E6C6F61642066696C06
:10082000616D656E74005A204F666673657400557D
:100830006E6B6E6F776E20636F6D6D616E643A20C4
:1008400022004D32303020496E76616C696420653B
:100850007874727564657220007A5F6D61783A20F1
:10086000007A5F6D696E3A2000795F6D61783A2099
:1008700000795F6D696E3A2000785F6D61783A208B
:10088000006F70656E005452494747455245440019
:10089000785F6D696E3A20005265706F7274696E90
:1008A0006720656E6473746F702073746174757300
:1008B0000020436F756E7420583A20004649524D0F
:1008C000574152455F4E414D453A4D61726C696EDC
:1008D0002056312E302E323B20537072696E746573
:1008E000722F6772626C206D617368757020666F1D
:1008F000722067656E36204649524D574152455F1A
:1009000055524C3A68747470733A2F2F6769746843
:1009100075622E636F6D2F707275736133642F5023
:10092000727573612D69332D506C75732F20505281
:100930004F544F434F4C5F56455253494F4E3A31F7
:100940002E30204D414348494E455F545950453A59
:100950005072757361206933204D4B3320455854D4
:1009600052554445525F434F554E543A31205555E8
:1009700049443A30303030303030302D3030303043
:100980002D303030302D303030302D303030303070
:10099000303030303030300A004F666600456E64CB
:1009A0002066696C65206C69737400426567696EC6
:1009B0002066696C65206C697374004E6F206D6FE2
:1009C00076652E004F626E6F76656E69207469736E
:1009D0006B7500526573756D696E67207072696E14
:1009E00074005761697420666F7220757365722E8A
:1009F0002E2E004B616C696272616365205A207310
:100A0000656C68616C612E2053656E736F72207324
:100A100065706E756C207072696C6973207679737D
:100A20006F6B6F2E2043656B616D206E6120726568
:100A30007365742E00426564206C6576656C696E22
:100A400067206661696C65642E2053656E736F72F2
:100A50002074726967676572656420746F6F2068BF
:100A60006967682E2057616974696E6720666F72C6
:100A70002072657365742E004B616C6962726163EC
:100A800065205A2073656C68616C612E2053656E19
:100A9000736F72206A65206F64706F6A656E79206B
:100AA0006E65626F20707265727573656E79206B0A
:100AB0006162656C2E2043656B616D206E612072F2
:100AC000657365742E00426564206C6576656C699B
:100AD0006E67206661696C65642E2053656E736F66
:100AE0007220646973636F6E6E6563746564206FF2
:100AF00072206361626C652062726F6B656E2E207E
:100B000057616974696E6720666F722072657365DC
:100B1000742E004B616C696272616365205A2073A8
:100B2000656C68616C612E2053656E736F72206E08
:100B3000657365706E756C2E205A6E65636973748B
:100B4000656E6120747279736B613F2043656B61E0
:100B50006D206E612072657365742E00426564209D
:100B60006C6576656C696E67206661696C65642E7C
:100B70002053656E736F72206469646E74207472A2
:100B800069676765722E20446562726973206F6EB3
:100B9000206E6F7A7A6C653F2057616974696E6761
:100BA00020666F722072657365742E005465706CD8
:100BB0006F746E69206B616C696272616365206439
:100BC0006F6B6F6E63656E612E20506F6B72616329
:100BD000756A746520737469736B656D20746C61DC
:100BE0006369746B612E0054656D70657261747514
:100BF00072652063616C6962726174696F6E2069ED
:100C0000732066696E69736865642E20436C69633E
:100C10006B20746F20636F6E74696E75652E005360
:100C20006C6565702E2E2E0043524153485F52452D
:100C3000434F5645520047323820582059009E04F1
:100C40008D040A002F00AE040A002E0044656C6576
:100C500074696F6E206661696C65642C2046696CEE
:100C6000653A200046696C652064656C657465644E
:100C70003A002E0020573A0020453A00543A00D559
:100C800004C004000005E504504944204175746F18
:100C900074756E652066696E69736865642120509D
:100CA000757420746865206C617374204B702C20FF
:100CB0004B6920616E64204B6420636F6E737461B6
:100CC0006E74732066726F6D2061626F7665206945
:100CD0006E746F20436F6E66696775726174696FB9
:100CE0006E2E6800504944204175746F74756E65AE
:100CF000206661696C6564212074696D656F757427
:100D00000020403A006F6B20543A006F6B20423A4B
:100D100000504944204175746F74756E652066619A
:100D2000696C6564212054656D70657261747572BB
:100D30006520746F6F206869676800204B643A20F3
:100D400000204B693A2000204B703A200020436C71
:100D500061737369632050494420002054753A2020
:100D600000204B753A2000206D61783A2000206DFC
:100D7000696E3A200020643A200020626961733A6B
:100D8000200053657474696E67732053746F7265C5
:100D9000640046696C616D656E7420736574746976
:100DA0006E67733A2044697361626C656400202049
:100DB000204D32303020440046696C616D656E74A0
:100DC0002073657474696E67733A002020204D3279
:100DD00030392053004175746F2D52657472616310
:100DE000743A20533D3020746F2064697361626CE3
:100DF000652C203120746F20696E74657270726585
:100E00007420657874727564652D6F6E6C79206DD1
:100E10006F76657320617320726574726163747399
:100E2000206F72207265636F76657269657300204A
:100E300046002020204D3230382053005265636F29
:100E40007665723A20533D4578747261206C656E08
:100E500067746820286D6D2920463A537065656473
:100E600020286D6D2F6D2900205A0020460020207B
:100E7000204D323037205300526574726163743AEA
:100E800020533D4C656E67746820286D6D2920469F
:100E90003A537065656420286D6D2F6D29205A3A8C
:100EA000205A4C69667420286D6D2900204400206A
:100EB00049002020204D3330342050005049442038
:100EC000686561746265642073657474696E6773C4
:100ED0003A002044002049002020204D33303120AA
:100EE00050005049442073657474696E67733A000A
:100EF000205A0020590020204D323036205800481A
:100F00006F6D65206F666673657420286D6D293A74
:100F100000204500205A002059002058002042009F
:100F200020540020204D323035205300416476613A
:100F30006E636564207661726961626C65733A20E4
:100F4000533D4D696E206665656472617465202845
:100F50006D6D2F73292C20543D4D696E2074726184
:100F600076656C20666565647261746520286D6DB8
:100F70002F73292C20423D6D696E696D756D20734C
:100F800065676D656E742074696D6520286D7329C1
:100F90002C20583D6D6178696D756D205859206A17
:100FA00065726B20286D6D2F73292C20205A3D6DA2
:100FB0006178696D756D205A206A65726B20286DA5
:100FC0006D2F73292C2020453D6D6178696D756DFD
:100FD0002045206A65726B20286D6D2F73290020D3
:100FE000540020204D323034205300416363656C3F
:100FF00065726174696F6E3A20533D616363656C1D
:1010000065726174696F6E2C20543D7265747261F3
:10101000637420616363656C65726174696F6E00EF
:10102000204500205A0020590020204D3230312028
:1010300058004D6178696D756D20416363656C651D
:10104000726174696F6E20286D6D2F7332293A00BA
:10105000204500205A0020590020204D32303320F6
:1010600058004D6178696D756D20666565647261C3
:1010700074657320286D6D2F73293A002045002078
:101080005A0020590020204D3932205800537465F1
:1010900070732070657220756E69743A0035052092
:1010A0000558054805790568059E058B05BD05B2FF
:1010B00005DE05D005FB05EC05746D633231333078
:1010C0005F7072696E745F63757272656E74732897
:1010D000290A094809520A580925640925640A5948
:1010E0000925640925640A5A0925640925640A4505
:1010F0000925640925640A000B0626061406222821
:10110000322900370649065400496E76616C6964DD
:10111000205420636F64652E004D323230205325F9
:1011200069008F065A06E006BF0622070007590726
:101130004707A1076C07FD07CC07203A20000026CF
:10114000084C414E472053454C20464F524345449E
:101150000022283129002F0842085908610869082F
:1011600071087908810886089008980820453A0097
:10117000205A3A0020593A00B10820453A00205A36
:101180003A0020593A00583A00BC084D313133201A
:1011900053002E002000990920423A0020453A00D1
:1011A000543A0020413A0020503A002042403A0090
:1011B00020403A00202F003A00205400202F002029
:1011C000423A00202F006F6B20543A002569206DB1
:1011D000696E2C20256920736563009D09AB09BBEE
:1011E00009D309C409E2094D65736820626564206A
:1011F0006C6576656C696E67206E6F7420616374D0
:101200006976652E000A002020000A4D656173751D
:1012100072656420706F696E74733A000A5A2073A5
:101220006561726368206865696768743A20002C9C
:10123000004E756D20582C593A2000206D6963725C
:101240006F6E732E004D69644C65667420206820B3
:101250003D00206D6963726F6E732E00526561727E
:101260004C65667420202067203D00206D69637204
:101270006F6E732E005265617243656E747220202A
:1012800066203D00206D6963726F6E732E0052659B
:1012900061725269676874202065203D00206D6985
:1012A00063726F6E732E004D6964526967687420B3
:1012B000202064203D00206D6963726F6E732E00E4
:1012C00046726F6E7452696768742063203D002017
:1012D0006D6963726F6E732E0046726F6E74436534
:1012E0006E74722062203D00206D6963726F6E73B0
:1012F0002E0046726F6E744C656674202061203D2E
:1013000000206D6963726F6E730045786365737357
:1013100069766520626564206C6576656C696E67C8
:1013200020636F7272656374696F6E3A2000350ACC
:10133000F309C60A780A5C0B130B47323820573082
:10134000003A2000E70BAC0B54656D706572617458
:101350007572652063616C6962726174696F6E2079
:10136000646F6E652E20436F6E74696E75652077AD
:10137000697468207072657373696E67207468653C
:10138000206B6E6F622E0000205A207368696674AD
:1013900020286D6D293A0050494E44412074656DF6
:1013A00070657261747572653A2000002F360053C3
:1013B0007465703A200000205A20736869667420B2
:1013C000286D6D293A0050494E44412074656D7076
:1013D000657261747572653A20002F362028736B30
:1013E00069707065642900537465703A2000005A72
:1013F00045524F3A20000073746172742074656D19
:1014000070657261747572653A200050494E4441AE
:101410002070726F62652063616C696272617469C9
:101420006F6E207374617274004732382057300039
:101430000A00205A3A200020593A200020583A2029
:10144000001F0C656E717565696E67202200446F20
:101450006E65207072696E74696E672066696C656E
:101460000053544F505045442E20005072696E7402
:1014700065722073746F7070656420647565207484
:101480006F206572726F72732E20466978207468BF
:1014900065206572726F7220616E642075736520BD
:1014A0004D39393920746F20726573746172742EEE
:1014B000202854656D70657261747572652069735A
:1014C0002072657365742E205365742069742061E1
:1014D000667465722072657374617274696E6729CF
:1014E000004E6F204C696E65204E756D62657220EE
:1014F0007769746820636865636B73756D2C204C25
:10150000617374204C696E653A20004E6F20436809
:1015100065636B73756D2077697468206C696E659F
:10152000206E756D6265722C204C617374204C695D
:101530006E653A2000636865636B73756D206D6935
:10154000736D617463682C204C617374204C696EF8
:10155000653A20004C696E65204E756D626572209B
:101560006973206E6F74204C617374204C696E65D2
:10157000204E756D6265722B312C204C6173742086
:101580004C696E653A200022206661696C65643A98
:10159000204275666665722066756C6C21002200BB
:1015A0004314256920686F757273202569206D6961
:1015B0006E75746573004E1454494D454F55543A39
:1015C0000061146B14E1140B15351554154D3131B0
:1015D000300046756C6C2052582042756666657204
:1015E000005641524F56414E493A204E657A6E613F
:1015F0006D612C206E65706F64706F726F76616EB6
:1016000061207665727A65206669726D77617265B0
:101610002E20506F757A697469206E6120766C6136
:1016200073746E69206E6562657A70656369210006
:101630005741524E494E473A2054686973206973A6
:1016400020616E20756E6F6666696369616C2C201F
:10165000756E737570706F72746564206275696CF5
:10166000642E2055736520617420796F7572206F28
:10167000776E207269736B210050727573612069F7
:1016800033204D4B33206F6B0050727573612069AE
:1016900033204D4B332072656164792E00446574AC
:1016A000656B6F76616E207679706164656B207012
:1016B000726F7564752E4F626E6F766974207469EF
:1016C000736B3F00426C61636B6F7574206F636373
:1016D00075727265642E205265636F766572207034
:1016E00072696E743F004E656E69207A6B616C6939
:1016F00062726F76616E6120767A64616C656E6F7E
:10170000737420747279736B79206F6420746973B9
:101710006B6F766520706F646C6F7A6B792E2050DA
:101720006F73747570756A74652070726F73696D0C
:1017300020706F646C65206D616E75616C752C2016
:101740006B617069746F6C61205A6163696E616D61
:10175000652C206F64737461766563204E617374C9
:101760006176656E69207072766E69207672737428
:1017700076792E0044697374616E636520626574C6
:101780007765656E20746970206F662074686520C7
:101790006E6F7A7A6C6520616E6420746865206271
:1017A0006564207375726661636520686173206E7D
:1017B0006F74206265656E20736574207965742E80
:1017C00020506C6561736520666F6C6C6F77207458
:1017D0006865206D616E75616C2C20636861707442
:1017E00065722046697273742073746570732C205F
:1017F00073656374696F6E204669727374206C61DF
:101800007965722063616C6962726174696F6E2EB2
:10181000005469736B61726E61206E6562796C61F0
:10182000206A65737465207A6B616C6962726F7689
:10183000616E612E20506F73747570756A746520C7
:1018400070726F73696D20706F646C65206D616E6E
:1018500075616C752C206B617069746F6C61205AB6
:101860006163696E616D652C206F64737461766568
:101870006320506F73747570206B616C6962726164
:1018800063652E005072696E746572206861732002
:101890006E6F74206265656E2063616C696272614F
:1018A000746564207965742E20506C6561736520C1
:1018B000666F6C6C6F7720746865206D616E756102
:1018C0006C2C206368617074657220466972737451
:1018D0002073746570732C2073656374696F6E2058
:1018E00043616C6962726174696F6E20666C6F77B8
:1018F0002E002020506C616E6E65724275666665C2
:101900007242797465733A20002046726565204DF5
:10191000656D6F72793A2000207C20417574686F84
:10192000723A2000204C61737420557064617465B4
:10193000643A200020536F667477617265205265A7
:1019400073657400205761746368646F6720526523
:10195000736574002042726F776E206F7574205229
:1019600065736574002045787465726E616C2052F1
:101970006573657400506F7765725570006572729B
:101980006F722077726974696E6720746F20666960
:101990006C6500656E6473746F7073206869743A67
:1019A0002000446F6E6520736176696E67206669FA
:1019B0006C652E006F6B00202D20496E76616C697E
:1019C00064206578747275646572206E756D6265E9
:1019D000722021001B5B324A1B5B313B31484F7246
:1019E0006967696E616C2050727573612069331B81
:1019F0005B323B3348507275736120526573656189
:101A000072636800466163746F7279205245534572
:101A100054003016E1155052555341334446570097
:101A200089167916C4169D167417E61684181118AF
:101A3000F21809194A616E203235203230313800EF
:101A4000436F6D70696C65643A20002833642D67BC
:101A50007573736E65722C48290018194A616E20DF
:101A6000323520323031382031323A35333A32365D
:101A70000024193419441954196519751920332E85
:101A8000312E312D5243352D3135310A00737461B9
:101A90007274002055706C6F616420696E207072E2
:101AA0006F6772657373007D195A00205A3A0059A6
:101AB0000020593A00580020583A0093194D36300A
:101AC000300043524153485F4445544543544544D4
:101AD00000A219B4194D3239004F626E6F766F76DD
:101AE000616E69207469736B752020202000526537
:101AF000636F766572696E67207072696E742020FC
:101B00002020005A206C6976652061646A757374C0
:101B1000206F7574206F662072616E67652E20538A
:101B2000657474696E6720746F20302E20436C6971
:101B3000636B20746F20636F6E74696E75652E0021
:101B40005A206C6976652061646A757374206F75BC
:101B500074206F662072616E67652E205365747401
:101B6000696E6720746F20300020423A0020453AA9
:101B700000543A0055564C4F202D20656E6400737A
:101B800074707300494E54340029002C20002C201E
:101B900000776F726C6420636F6F7264696E61743A
:101BA00065733A20280029002C20002C2000706842
:101BB00079736963616C20636F6F7264696E6174BD
:101BC00065733A2028007265636F7665725F6D6198
:101BD0006368696E655F73746174655F616674657F
:101BE000725F706F7765725F70616E69632C2069D8
:101BF0006E697469616C20007265636F7665725FEF
:101C00006D616368696E655F73746174655F616659
:101C10007465725F706F7765725F70616E69632C57
:101C200020696E697469616C200047393220450073
:101C30004D3234004D32362053256C75004D313015
:101C4000362053004D383200473120462564004786
:101C5000312045322A312046343830004731205A6D
:101C600000204632303030002059004731205800E3
:101C70004D383300506F736974696F6E20726561FF
:101C8000642066726F6D20656570726F6D3A004DED
:101C90003233202573002E67636F004665656472DA
:101CA0006174653A0063757272656E745F706F730C
:101CB0006974696F6E5B455F415849535D3A0063D3
:101CC000757272656E745F706F736974696F6E5B45
:101CD0005A5F415849535D3A0043757272656E749C
:101CE00020706F736974696F6E20595F4158495352
:101CF0003A0043757272656E7420706F736974690F
:101D00006F6E20585F415849533A004166746572BE
:101D10002077616974696E6720666F722074656DE3
:101D2000703A00473120452D312046343830004785
:101D3000312045352046313230004D3833004D31A9
:101D4000393020532564004D31303920532564004B
:101D500047323820582059004731205A3235204622
:101D6000383030004D31343020532564004D31304F
:101D7000342053256400EE1AD91A627573793A201B
:101D800070617573656420666F7220696E7075741A
:101D900000627573793A2070617573656420666FAF
:101DA00072207573657200627573793A2070726F74
:101DB00063657373696E6700000021104220633011
:101DC0008440A550C660E770088129914AA16BB193
:101DD0008CC1ADD1CEE1EFF131121002733252223B
:101DE000B5529442F772D662399318837BB35AA3E3
:101DF000BDD39CC3FFF3DEE362244334200401140B
:101E0000E664C774A44485546AA54BB52885099532
:101E1000EEE5CFF5ACC58DD55336722611163006DA
:101E2000D776F6669556B4465BB77AA71997388782
:101E3000DFF7FEE79DD7BCC7C448E5588668A7789A
:101E40004008611802282338CCC9EDD98EE9AFF9D2
:101E5000488969990AA92BB9F55AD44AB77A966A7A
:101E6000711A500A333A122AFDDBDCCBBFFB9EEB22
:101E7000799B588B3BBB1AABA66C877CE44CC55C4A
:101E8000222C033C600C411CAEED8FFDECCDCDDD72
:101E90002AAD0BBD688D499D977EB66ED55EF44E1A
:101EA000133E322E511E700E9FFFBEEFDDDFFCCFC2
:101EB0001BBF3AAF599F788F8891A981CAB1EBA116
:101EC0000CD12DC14EF16FE18010A100C230E32092
:101ED0000450254046706760B9839893FBA3DAB33A
:101EE0003DC31CD37FE35EF3B1029012F322D232E2
:101EF0003542145277625672EAB5CBA5A89589850A
:101F00006EF54FE52CD50DC5E234C324A014810431
:101F10006674476424540544DBA7FAB79987B897D9
:101F20005FE77EF71DC73CD7D326F2369106B01681
:101F300057667676154634564CD96DC90EF92FE999
:101F4000C899E9898AB9ABA94458654806782768D1
:101F5000C018E1088238A3287DCB5CDB3FEB1EFB79
:101F6000F98BD89BBBAB9ABB754A545A376A167A21
:101F7000F10AD01AB32A923A2EFD0FED6CDD4DCD49
:101F8000AABD8BADE89DC98D267C076C645C454C71
:101F9000A23C832CE01CC10C1FEF3EFF5DCF7CDF19
:101FA0009BAFBABFD98FF89F176E367E554E745EC1
:101FB000932EB23ED10EF01E7C3C3E5E2B3D3F2F59
:101FC0005B5D3B2C2A225C00454550524F4D20451D
:101FD00072726F720048617264636F64656420445A
:101FE000656661756C742053657474696E677320DF
:101FF0004C6F6164656400436F6E74696E75652033
:102000007769746820616E6F7468657220626F779B
:1020100064656E3F00250020202020202000202025
:10202000202020200045524153494E4720616C6CCE
:10203000206461746100466163746F727920524557
:1020400053455400454E41424C45440A00444953CF
:1020500041424C45440A004653656E736F7220003E
:10206000504154393132355F696E69743A25640ADA
:102070000000007F43000052430000524300000074
:1020800000000080C09A99193E0000000000008006
:10209000C09A99193E0000A0400000A04000000036
:1020A000404E656A6472697665207A61766564740B
:1020B0006520504C412066696C616D656E742070BE
:1020C000726F73696D2E00506C65617365206C6F63
:1020D000616420504C412066696C616D656E7420AE
:1020E00066697273742E004A6520504C41206669FF
:1020F0006C616D656E74207A61766564656E3F0013
:10210000497320504C412066696C616D656E742086
:102110006C6F616465643F0050726F73696D207A03
:1021200061766564746520504C412066696C616D10
:10213000656E74206120706F207465206F626E6F11
:102140007674652057697A6172646120737469736B
:102150006B6E7574696D20726573657420746C6143
:102160006369746B612E00506C65617365206C6FE0
:10217000616420504C412066696C616D656E74200D
:10218000616E64207468656E20726573756D65207C
:1021900057697A617264206279207265626F6F7428
:1021A000696E6720746865207072696E7465722E3E
:1021B0000050726F73696D206E61686C65646E6546
:1021C000746520646F206D616E75616C752061208F
:1021D0006F7072617674652070726F626C656D2EBF
:1021E00020506F207465206F626E6F767465205783
:1021F000697A61726461207265626F6F746F766173
:102200006E696D207469736B61726E792E00506C0B
:102210006561736520636865636B206F7572206804
:10222000616E64626F6F6B20616E642066697820F6
:102230007468652070726F626C656D2E20546865DD
:102240006E20726573756D65207468652057697AB4
:10225000617264206279207265626F6F74696E6763
:1022600020746865207072696E7465722E005673F2
:1022700065206A6520686F746F766F2E00416C6C04
:1022800020697320646F6E652E204861707079201C
:102290007072696E74696E67210057697A61726441
:1022A00061206D757A657465206B64796B6F6C69FC
:1022B00076207A6E6F7675207370757374697420EA
:1022C0007A206D656E752043616C69627261746914
:1022D0006F6E202D3E2057697A61726400596F75C8
:1022E0002063616E20616C7761797320726573750C
:1022F0006D65207468652057697A61726420667222
:102300006F6D2043616C6962726174696F6E202D1C
:102310003E2057697A6172642E0050726F73696D46
:10232000206F6369737465746520686561746265A4
:1023300064206120737469736B6E65746520746CBE
:10234000616369746B6F2E00506C65617365206307
:102350006C65616E206865617462656420616E649D
:10236000207468656E2070726573732074686520D0
:102370006B6E6F622E00436863657465206F7061D9
:102380006B6F76617420706F736C65646E69206B1F
:10239000726F6B206120706F7A6D656E6974207644
:1023A0007A64616C656E6F7374206D657A692074F0
:1023B0007279736B6F752061206865617462656402
:1023C0003F00446F20796F752077616E7420746FC1
:1023D00020726570656174206C617374207374651C
:1023E0007020746F20726561646A7573742064690B
:1023F0007374616E6365206265747765656E206EC7
:102400006F7A7A6C6520616E6420686561746265BC
:10241000643F005A61636E75207469736B6E6F75EB
:1024200074206C696E6B752061205679206275642A
:1024300065746520706F737475706E6520736E6956
:102440007A6F76617420747279736B75206F746122
:1024500063656E696D20746C616369746B6120647F
:102460006F6B7564206E65646F7361686E6574650B
:10247000206F7074696D616C6E69207679736B7909
:102480002E2050726F686C65646E65746520736988
:10249000206F6272617A6B792076206E6173692099
:1024A00070726972756363652076206B6170697400
:1024B0006F6C65204B616C696272616365004920D5
:1024C00077696C6C20737461727420746F20707201
:1024D000696E74206C696E6520616E6420796F7519
:1024E0002077696C6C206772616475616C6C79200F
:1024F0006C6F77657220746865206E6F7A7A6C6590
:1025000020627920726F746174696E6720746865E7
:10251000206B6E6F622C20756E74696C20796F75FC
:10252000207265616368206F7074696D616C2068EA
:1025300065696768742E20436865636B20746865FD
:1025400020706963747572657320696E206F75728F
:102550002068616E64626F6F6B20696E20636861D2
:10256000707465722043616C6962726174696F6E28
:102570002E004E796E69207A6B616C696272756AA1
:102580006920767A64616C656E6F7374206D657A0C
:1025900069206B6F6E63656D20747279736B79203F
:1025A0006120706F76726368656D20686561746222
:1025B0006564752E004E6F7720492077696C6C201A
:1025C00063616C6962726174652064697374616EC1
:1025D0006365206265747765656E20746970206F2D
:1025E0006620746865206E6F7A7A6C6520616E640F
:1025F00020686561746265642073757266616365E5
:102600002E004A6520746F20504C412066696C6131
:102610006D656E743F00497320697420504C4120F1
:1026200066696C616D656E743F005A6176616465C0
:102630006E692066696C616D656E7475004C6F61C2
:1026400064696E672066696C616D656E74005072B6
:102650006F73696D20766C6F7A746520504C4120E1
:1026600066696C616D656E7420646F206578747244
:1026700075646572752C20706F20746520737469A1
:10268000736B6E65746520746C616369746B6F2025
:1026900070726F207A61766564656E692066696C18
:1026A000616D656E74752E00506C6561736520698F
:1026B0006E7365727420504C412066696C616D6563
:1026C0006E7420746F207468652065787472756408
:1026D00065722C207468656E207072657373206B50
:1026E0006E6F6220746F206C6F61642069742E00BD
:1026F000507265646568726976616D207472797371
:102700006B752E2050726F73696D2063656B656AFF
:1027100074652E0050726568656174696E67206E1D
:102720006F7A7A6C652E20506C65617365207761D5
:1027300069742E004E796E692070726564656872E6
:10274000656A6920747279736B752070726F20509E
:102750004C412E004E6F7720492077696C6C2070B9
:10276000726568656174206E6F7A7A6C6520666F39
:102770007220504C412E004A652066696C616D657F
:102780006E74207A61766564656E3F0049732066D9
:10279000696C616D656E74206C6F616465643F0087
:1027A000556D6973746574652070726F73696D20FF
:1027B0007469736B6F767920706C6174206E612020
:1027C0006865617462656400506C65617365207052
:1027D0006C61636520737465656C207368656574EE
:1027E000206F6E20686561746265642E004A652002
:1027F0007469736B6F767920706C6174206E6120E0
:10280000686561746265643F00497320737465652F
:102810006C207368656574206F6E206865617462F2
:1028200065643F004E796E692070726F76656475DD
:10283000207A206B616C6962726163692E004920A5
:1028400077696C6C2072756E207A2063616C6962A6
:10285000726174696F6E206E6F772E004E796E69AB
:102860002070726F766564752078797A206B616C60
:102870006962726163692E205A61626572652074B3
:102880006F20707269626C697A6E65203132206DDA
:10289000696E2E00492077696C6C2072756E207805
:1028A000797A2063616C6962726174696F6E206EFF
:1028B0006F772E2049742077696C6C2074616B658A
:1028C00020617070726F782E203132206D696E73C6
:1028D0002E004E656A6472697620706F6D6F636951
:1028E0002073656C667465737475207A6B6F6E7493
:1028F0006F6C756A69206E656A63617374656A736B
:102900006920636879627920767A6E696B616A6999
:1029100063692070726920736573746176656E698E
:10292000207469736B61726E792E004669727374DC
:102930002C20492077696C6C2072756E2074686554
:102940002073656C667465737420746F20636865AA
:10295000636B206D6F737420636F6D6D6F6E20619C
:102960007373656D626C792070726F626C656D73E4
:102970002E00446F6272792064656E2C206A736544
:102980006D2076617365207469736B61726E61206E
:102990004F726967696E616C20507275736120694E
:1029A000332E204368636574652061627963682013
:1029B0005661732070726F7665646C61206B616C18
:1029C00069627261636E696D2070726F63657365B1
:1029D0006D3F0048692C204920616D20796F757228
:1029E000204F726967696E616C2050727573612047
:1029F0006933207072696E7465722E20576F756C22
:102A00006420796F75206C696B65206D6520746F2B
:102A100020677569646520796F75207468726F75B9
:102A20006768207468652073657475702070726FB4
:102A3000636573733F0054726964656E69205B411E
:102A40006265636564615D00536F72743A20205B58
:102A5000416C7068616265745D0054726964656E92
:102A60006920202020205B4361735D00536F7274E6
:102A70003A2020202020205B54696D655D0053447E
:102A8000206361726420205B6E6F726D616C5D000B
:102A900053442063617264205B466C7368416972C1
:102AA0005D005679626572206A617A796B610053C4
:102AB000656C656374206C616E6775616765005253
:102AC000506920706F7274202020205B7A61705DE5
:102AD0000052506920706F727420202020205B6F9C
:102AE0006E5D0052506920706F7274202020205B50
:102AF0007679705D0052506920706F7274202020CA
:102B0000205B6F66665D005465706C2E206B616C97
:102B10002E20205B7A61705D0054656D702E2063FD
:102B2000616C2E2020205B6F6E5D005465706C2EF2
:102B3000206B616C2E20205B7679705D0054656D92
:102B4000702E2063616C2E20205B6F66665D004BEB
:102B50006F6E74722E2076656E742E5B7679705D62
:102B60000046616E7320636865636B20205B6F664F
:102B7000665D004B6F6E74722E2076656E742E5BF0
:102B80007A61705D0046616E7320636865636B20D7
:102B900020205B6F6E5D0054726964656E69202051
:102BA000205B5A61646E655D00536F72743A202039
:102BB000202020205B4E6F6E655D00462E206175E3
:102BC000746F7A61762E205B7679705D00462E20D8
:102BD0006175746F6C6F6164205B6F66665D004643
:102BE0002E206175746F7A61762E205B7A61705D3C
:102BF00000462E206175746F6C6F616420205B6FDE
:102C00006E5D00462E206175746F7A61762E205BB2
:102C10004E2F415D00462E206175746F6C6F6164AC
:102C2000205B4E2F415D0046696C2E2073656E7AE5
:102C30006F72205B4E2F415D0046696C2E207365DC
:102C40006E736F72205B4E2F415D005679706E6F10
:102C50007574206D6F746F72790044697361626C72
:102C60006520737465707065727300506F73756E54
:102C70006F7574206F7375004D6F7665206178698C
:102C800073005465706C6F74610054656D7065728B
:102C900061747572650047373600C720A120002196
:102CA000E720672118210E22B1217D226E22DD222C
:102CB0009A2253746174653A200048231A23C22370
:102CC0007623BE241324B5257225162602263D261A
:102CD0002A26A8264E261427F026542734278C2788
:102CE0007727C827A0270928ED273E2824289428DD
:102CF0005C282B29D228D329722947393900446905
:102D00007361626C65206661726D206D6F64653FF2
:102D100000482A362A6C2A5A2A7E2A902AAF2AA2EA
:102D20002AD12ABF2AF52AE32A4661726D206E75E0
:102D30006D62657200192B072B3D2B2B2B44697399
:102D400061626C65206661726D206D6F6465006103
:102D50002B4F2B852B732BA92B972BCD2BBB2BF11B
:102D60002BDF2B152C032C392C272C4D3834005AF3
:102D70002C4B2C782C6B2C8A2C822C506F757A65FE
:102D800020616B7475616C6E690043757272656E5B
:102D90007400506F757A69746520626568656D208E
:102DA0007469736B75005573656420647572696E20
:102DB00067207072696E740056736500416C6C0018
:102DC000504944206B616C2E20756B6F6E63656E8D
:102DD00061005049442063616C2E2066696E6973FE
:102DE00068656400504944206B616C2E20202020CF
:102DF00020202020202020005049442063616C2E98
:102E00002020202020202020202020004D3131377C
:102E1000204B616C2E207072766E6920767273740E
:102E20007679004D313137204669727374206C61B8
:102E30007965722063616C2E004F626E6F766F76DB
:102E4000616E69207469736B7500526573756D6985
:102E50006E67207072696E74005469736B20706FB6
:102E60007A6173746176656E005072696E74207059
:102E70006175736564008A2D7B2DA62D922DBC2D66
:102E8000B82D496E76616C696420504944206361B5
:102E90006C2E20726573756C74732E204E6F7420C7
:102EA00073746F72656420746F20454550524F4DA6
:102EB0002E004D35303000D22DC02DF82DE42D4799
:102EC00031205A3135204631353030004739310014
:102ED000473120583530205931393020453020468F
:102EE0003730303000473930004D373032004D3701
:102EF00030322043004D3730322055004D373032CC
:102F0000004731205A3135204631353030004739BD
:102F10003100473120583530205931393020453083
:102F2000204637303030004D383300473930004DBF
:102F30003834004D313034205330004D38340047A0
:102F4000312058313020593138302046343030303B
:102F5000004731205A31302046313330302E303066
:102F600030004D313430205330004D313034205357
:102F700030004D31303700473120452D302E30376D
:102F80003530302046323130302E30303030300065
:102F9000473120583530205935352045332E3632CB
:102FA00037373300473120583230302059353520FB
:102FB00045302E34393338360047312058323030DE
:102FC000205937352045332E3632373733004731D5
:102FD00020583530205937352045302E3439333894
:102FE0003600473120583530205939352045332EA9
:102FF0003632373733004731205832303020593994
:10300000352045302E343933383600473120583298
:10301000303020593131352045332E363237373371
:103020000047312058353020593131352045302E78
:103030003439333836004731205835302059313350
:10304000352045332E36323737330047312058325A
:10305000303020593133352045302E363631373433
:103060000047312058323030205931353520453233
:103070002E3632373733004731205831303020591F
:103080003135352045320047312058373520593108
:1030900035352045322E3500473120463130383025
:1030A000004731205835302059313535004731201F
:1030B0004634303030004D323034205331303030EF
:1030C000004731205A302E313530204637323030EB
:1030D0002E30303000473120452D312E3530303004
:1030E000302046323130302E3030303030004D38E4
:1030F00033004739300047323100473932204530FC
:103100002E3000473120583130302E3020453132BA
:103110002E352046313030302E30004731205836A1
:10312000302E302045392E302046313030302E3090
:10313000004739322045302E3000473238004738BA
:103140003700232E0C2E4D313039205332313500CB
:103150004D31393020533630004D31343020533624
:1031600030004D3130342053323135004D3130375D
:10317000004A2E392E473930004731204531004D65
:103180003832004731204531004D3833004D313061
:103190003620532564004D323230205325640069B7
:1031A0002E592E5A63686C6164697400436F6F6CAA
:1031B000646F776E0054657A6B65207A6B6F736508
:1031C0006E693A0053657665726520736B65773A70
:1031D000004C65686B65207A6B6F73656E693A00A9
:1031E000536C6967687420736B65773A004D65723C
:1031F000656E65207A6B6F73656E693A004D656127
:10320000737572656420736B65773A0050726176EE
:10321000793A0052696768743A004C6576793A00E9
:103220004C6566743A005920767A64616C656E6FFD
:103230007374206F64206D696E3A0059206469735D
:1032400074616E63652066726F6D206D696E3A0001
:103250004E617065746900566F6C746167657300C8
:103260005465706C6F74790054656D70657261742B
:103270007572657300537461762072656D656E7545
:103280000042656C742073746174757300457874C2
:10329000727564657220696E666F00446574616959
:1032A0006C792058595A206B616C2E0058595A205D
:1032B00063616C2E2064657461696C730044617491
:1032C000756D3A00446174653A00686F77746F2ECB
:1032D000707275736133642E637A00686F77746FF0
:1032E0002E707275736133642E636F6D00666F723A
:1032F000756D2E707275736133642E637A00666F1C
:1033000072756D2E707275736133642E636F6D000C
:10331000707275736133642E637A007072757361B5
:1033200033642E636F6D001B5B323B3148416D622D
:1033300069656E743A2020256425631B5B333B313D
:103340004850494E44413A202020202564256300FE
:103350001B5B303B31484E6F7A7A6C653A202020F7
:10336000256425631B5B313B31484265643A20206C
:103370002020202025642563001B5B313B31485011
:1033800057523A20202020202025642E25303164F9
:1033900056001B5B303B314842656C74207374618E
:1033A0007475731B5B313B3248582025641B5B32BC
:1033B0003B32485920256400AC31A331464C455876
:1033C000202D20203234302F353000505020202046
:1033D0002D20203235342F313030004849505320D1
:1033E0002D20203232302F31303000414253202006
:1033F0002D20203235352F313030005045542020DB
:103400002D20203233302F383500504C4120202DD4
:1034100020203231352F3630006661726D20202D2C
:1034200020203235302F34300000C431B53100E077
:1034300031D1312D2D2D2D2D2D2D2D2D2D2D2D2D10
:103440002D2D2D2D2D2D2D004E2F4100FD31ED3137
:103450004E2F41006D6D000013320C3220321A32B3
:103460003B32263257325032683260328132753206
:103470008D32AC329B322D2D2D2D2D2D2D2D2D2D20
:103480002D2D00466C6173684169722049502041BE
:103490006464723A002D2D2D2D2D2D2D2D2D2D2DC9
:1034A0002D002833642D677573736E65722C48295F
:1034B0000031323A35333A3433004A616E203235C6
:1034C000203230313800C432BD322D2D2D2D2D2D1E
:1034D0002D2D2D2D2D2D00453344763666756C6CC3
:1034E0000045494E595F30346100315F37356D6DAD
:1034F0005F4D4B33002D2D2D2D2D2D2D2D2D2D2DB3
:103500002D00DB32CA32FE32ED321B331033207213
:1035100065706F20507275736133442F4D4B3300CB
:1035200020332E312E312D5243352D313531004689
:1035300069726D776172653A0025642E25642E25C7
:10354000642E2564004B616C696272756A69205A49
:103550000043616C6962726174696E67205A004948
:103560007465726163652000497465726174696F86
:103570006E2000207A203400206F662034005A6CC0
:10358000657073756A6920707265736E6F737420ED
:103590006B616C69627261636E69686F20626F64EF
:1035A0007500496D70726F76696E67206265642080
:1035B00063616C6962726174696F6E20706F696EAD
:1035C00074004B616C6962726163652058595A20BE
:1035D0007620706F7261646B752E205A6B6F736505
:1035E0006E692062756465206175746F6D617469C0
:1035F000636B79207679726F766E616E6F20707270
:1036000069207469736B752E0058595A2063616C78
:103610006962726174696F6E20616C6C2072696797
:1036200068742E20536B65772077696C6C20626517
:1036300020636F72726563746564206175746F6D69
:1036400061746963616C6C792E004B616C696272A4
:103650006163652058595A207620706F7261646BDF
:10366000752E20582F59206F7379206D69726E6501
:10367000207A6B6F73656E652E20446F62726120D5
:103680007072616365210058595A2063616C6962E8
:10369000726174696F6E20616C6C20726967687406
:1036A0002E20582F59206178657320617265207330
:1036B0006C696768746C7920736B657765642E201C
:1036C000476F6F64206A6F6221004B616C696272A0
:1036D0006163652058595A207620706F7261646B5F
:1036E000752E20582F59206F7379206A736F7520BB
:1036F0006B6F6C6D652E2047726174756C756A69AD
:10370000210058595A2063616C6962726174696F53
:103710006E206F6B2E20582F5920617865732061C1
:1037200072652070657270656E646963756C617234
:103730002E20436F6E67726174756C6174696F6E71
:103740007321004B616C6962726163652058595A3C
:10375000206E65707265736E612E204C65767920DF
:10376000707265646E6920626F64206D6F6320768D
:1037700070726564752E0058595A2063616C6962D5
:10378000726174696F6E20636F6D70726F6D6973B3
:1037900065642E204C6566742066726F6E742063BB
:1037A000616C6962726174696F6E20706F696E74AA
:1037B000206E6F7420726561636861626C652E00B3
:1037C0004B616C6962726163652058595A206E655D
:1037D000707265736E612E20507265646E69206B25
:1037E000616C69627261636E6920626F6479206DD9
:1037F0006F63207670726564752E0058595A206385
:10380000616C6962726174696F6E20636F6D707252
:103810006F6D697365642E2046726F6E74206361EC
:103820006C6962726174696F6E20706F696E747317
:10383000206E6F7420726561636861626C652E0032
:103840004B616C6962726163652058595A207365D7
:103850006C68616C612E204C6576792070726564AD
:103860006E6920626F64206D6F632076707265648C
:10387000752E2053726F766E656A74652074697355
:103880006B61726E752E0058595A2063616C6962C3
:10389000726174696F6E206661696C65642E204C7C
:1038A0006566742066726F6E742063616C69627203
:1038B0006174696F6E20706F696E74206E6F742012
:1038C000726561636861626C652E004B616C696250
:1038D000726163652058595A2073656C68616C6128
:1038E0002E20507265646E69206B616C6962726132
:1038F000636E6920626F6479206D6F6320767072E9
:103900006564752E2053726F766E656A74652074D7
:1039100069736B61726E752E0058595A2063616C21
:103920006962726174696F6E206661696C65642E8C
:103930002046726F6E742063616C69627261746993
:103940006F6E20706F696E7473206E6F7420726575
:1039500061636861626C652E004B616C69627261C3
:1039600063652058595A2073656C68616C612E201C
:103970004E61686C65646E65746520646F206D616E
:103980006E75616C752E0058595A2063616C6962BE
:10399000726174696F6E206661696C65642E205077
:1039A0006C6561736520636F6E73756C74207468E9
:1039B00065206D616E75616C2E004B616C69627281
:1039C0006163652058595A2073656C68616C612E7B
:1039D000204B616C69627261636E6920626F642062
:1039E000706F646C6F7A6B79206E656E616C657A4E
:1039F000656E2E0058595A2063616C696272617459
:103A0000696F6E206661696C65642E204265642072
:103A100063616C6962726174696F6E20706F696E48
:103A20007420776173206E6F7420666F756E642EDC
:103A300000207A203400206F66203400486C6564D2
:103A4000616D206B616C69627261636E6920626F87
:103A50006420706F646C6F7A6B7900536561726378
:103A600068696E67206265642063616C6962726177
:103A700074696F6E20706F696E7400556D69737430
:103A8000657465206C69737420706170697275204B
:103A90006E6120706F646C6F7A6B75206120756445
:103AA000727A756A7465206A656A20706F64207422
:103AB0007279736B6F7520626568656D206D6572D4
:103AC000656E69207072766E696368203420626F5B
:103AD00064752E20506F6B756420747279736B61FE
:103AE000207A6163687974692070617069722C2032
:103AF0007679706E657465207469736B61726E752A
:103B00002E00506C616365206120736865657420C8
:103B10006F6620706170657220756E6465722074C6
:103B20006865206E6F7A7A6C6520647572696E675D
:103B3000207468652063616C6962726174696F6E7C
:103B4000206F66206669727374203420706F696E0E
:103B500074732E20496620746865206E6F7A7A6CC3
:103B600065206361746368657320746865207061A3
:103B70007065722C20706F776572206F6666207496
:103B80006865207072696E74657220696D6D656418
:103B9000696174656C792E0050726F207573706561
:103BA000736E6F75206B616C696272616369206FFF
:103BB000636973746574652070726F73696D2074C6
:103BC00069736B6F766F7520747279736B752E20C5
:103BD000506F74767264746520746C616369746B81
:103BE000656D2E00506C6561736520636C65616E58
:103BF00020746865206E6F7A7A6C6520666F72201B
:103C000063616C6962726174696F6E2E20436C69C6
:103C1000636B207768656E20646F6E652E004F645D
:103C2000737472616E7465207469736B6F7679203A
:103C3000706C6174207A20686561746265642070BC
:103C4000726F73696D2E00506C65617365207265CB
:103C50006D6F766520737465656C20736865657437
:103C60002066726F6D20686561746265642E000065
:103C7000007F43000056439AD95143FFFFFF51355F
:103C80004535203C20005741524E494E473A204688
:103C9000726F6E7420706F696E74206E6F74207214
:103CA0006561636861626C652E205920636F6F7275
:103CB00064696E6174653A000068355F3549746502
:103CC000726174696F6E3A200043616C63756C6158
:103CD00074696F6E206F6620746865206D6163681B
:103CE000696E6520736B657720616E64206F666610
:103CF000736574206661696C65642E007835733570
:103D0000A2357E350936C23587364A360237CA367D
:103D100077374337FB37C037873840381939CB38C6
:103D200087395939F439BA3943616C6962726174FF
:103D3000696F6E206661696C656421204368656304
:103D40006B20746865206178657320616E642072F1
:103D5000756E20616761696E2E00363A313A5B3AC2
:103D60003C3A023B7B3AE43B983B473C1E3C10000C
:103D7000C90210012C014001220170011801B0019B
:103D80000E01F00104015002FA00B002F00030030D
:103D9000E600D003DC009004D2007005C800A00645
:103DA000BE000008B400B009AA00D00BA000600E4D
:103DB000960060118C000015820020197800C01D4B
:103DC0006E00A0226400B0275A00902C50000031F1
:103DD0004600E0343C0010383200903A2800603C45
:103DE0001E00A03D1400803E0A00203F0000204835
:103DF0004F54454E4420544845524D414C20525555
:103E00004E415741590020484541544245442054B1
:103E10004845524D414C2052554E4157415900544E
:103E20004845524D414C2052554E41574159004250
:103E3000454420544845524D414C2052554E41571F
:103E400041590020544845524D414C2052554E4155
:103E50005741592028205052454845415420484F49
:103E600054454E44290020544845524D414C20525F
:103E7000554E4157415920282050524548454154FC
:103E80002048454154424544290050524548454147
:103E900054204552524F520042454420505245480A
:103EA000454154204552524F52004572723A204DBE
:103EB000415854454D50003A2045787472756465F8
:103EC00072207377697463686564206F66662E205C
:103ED0004D415854454D502074726967676572654D
:103EE000642021004572723A204D415854454D508E
:103EF000204245440054656D706572617475726549
:103F000020686561746564206265642073776974F4
:103F100063686564206F66662E204D415854454D98
:103F2000502074726967676572656420210045726C
:103F3000723A204D494E54454D502042454400545C
:103F4000656D706572617475726520686561746510
:103F50006420626564207377697463686564206FA8
:103F600066662E204D494E54454D50207472696747
:103F700067657265642021004572723A204D494E92
:103F800054454D50003A204578747275646572202E
:103F90007377697463686564206F66662E204D4987
:103FA0004E54454D50207472696767657265642090
:103FB00021004E4F524D414C00535445414C544802
:103FC00000746D63323133305F696E697428292C57
:103FD000206D6F64653D25530A00544D43204452C3
:103FE00049564552204F56455254454D5020007475
:103FF0006D63323133305F7365745F637572726500
:104000006E745F6828617869733D25642C20637540
:104010007272656E743D25640A00746D63323133CB
:10402000305F7365745F63757272656E745F72285A
:10403000617869733D25642C2063757272656E74B6
:104040003D25640A0050726F73696D2063656B656E
:104050006A746500506C65617365207761697400EE
:104060004175746F6D617469636B65207A61766107
:1040700064656E692066696C616D656E747520613A
:104080006B7469766E692C20737469736B6E6574DA
:104090006520746C616369746B6F206120766C6F4E
:1040A0007A74652066696C616D656E742E2E2E00C3
:1040B0004175746F6C6F6164696E672066696C61CD
:1040C0006D656E74206973206163746976652C2058
:1040D0006A75737420707265737320746865206BE1
:1040E0006E6F6220616E6420696E73657274206603
:1040F000696C616D656E742E2E2E0043656C6B6F5E
:10410000767920636173203A00546F74616C20707B
:1041100072696E742074696D65203A0046696C613D
:104120006D656E742063656C6B656D203A00546F2D
:1041300074616C2066696C616D656E74203A004331
:104140006173207469736B75203A20200050726986
:104150006E742074696D653A20200046696C616D4B
:10416000656E74203A20200046696C616D656E743E
:1041700020757365643A20200041646A7573746920
:104180006E67205A004D692E4C6566742020685B6E
:10419000756D5D0052652E4C6566742020675B75F9
:1041A0006D5D0052652E43656E747220665B756DA1
:1041B0005D0052652E526967687420655B756D5DA0
:1041C000004D692E526967687420645B756D5D00EF
:1041D00046722E526967687420635B756D5D004698
:1041E000722E43656E747220625B756D5D0046725F
:1041F0002E4C6566742020615B756D5D004E6173A9
:104200007461767465207465706C6F74753A0053D0
:1042100065742074656D70657261747572653A00BD
:10422000544045404D37303100B04060400941FBBB
:10423000402E411C414D413F4168415B41457874EE
:10424000727564657200580059005A0079418541C1
:104250009441A341B241C141D041DF41EE410F42FF
:10426000FD4120003E003E0020003E003E004E6129
:1042700068726976616E692050494E444100504928
:104280004E44412048656174696E67005465706CE6
:104290002E206B616C2E202020202020202020202A
:1042A0000054656D702E2063616C2E20202020202C
:1042B0002020202020004B616C69627261636520C0
:1042C0004F4B0043616C6962726174696F6E206468
:1042D0006F6E65004B616C696272756A69205A0085
:1042E00043616C6962726174696E67205A0042654D
:1042F00064204F4B2E0042656420646F6E65005A47
:104300006168726976616E69206265640042656405
:104310002048656174696E67005A616872697661E8
:104320006E69204F4B2E0048656174696E6720648A
:104330006F6E652E005A6168726976616E69004819
:10434000656174696E67005072696E74657220648D
:104350006973636F6E6E6563746564003A20007EF6
:10436000426E42A1428C42C342B64220202020200D
:10437000202020202020202020202020202000205D
:104380003A2000E042D4422020202020202020207B
:10439000202020202020202020202000F642EE4255
:1043A0000D43FF42274319433F433543202020203C
:1043B0002020202020202020200025730020200005
:1043C0002D2D3A2D2D002000200020004C00202013
:1043D000002046002D2D2D003E5553420053440031
:1043E0002D2D00252020202020002020002020002E
:1043F0000120002020202D2D2D200020205A0020DB
:10440000200001200047434578747275646572008E
:10441000506F73756E6F7574205A004D6F766520FE
:104420005A00506F73756E6F75742059004D6F761A
:1044300065205900506F73756E6F75742058004D6C
:104440006F76652058001B5B324A437261736820A7
:10445000646574656B6365206D757A651B5B313BC4
:104460003048627974207A61706E75746120706F63
:10447000757A6520761B5B323B30484E6F726D61FA
:104480006C206D6F6475001B5B324A437261736808
:1044900020646574656374696F6E2063616E1B5B75
:1044A000313B30486265207475726E6564206F6EB2
:1044B000206F6E6C7920696E1B5B323B30484E6F0B
:1044C000726D616C206D6F6465001B5B324A504FEA
:1044D0005A4F523A1B5B313B30484372617368203C
:1044E000646574656B63651B5B323B304864656172
:1044F0006B7469766F76616E612076651B5B333B0A
:104500003048537465616C7468206D6F6475001B6E
:104510005B324A5741524E494E473A1B5B313B3062
:1045200048437261736820646574656374696F6E73
:104530001B5B323B304864697361626C656420695F
:104540006E1B5B333B3048537465616C7468206D3F
:104550006F6465004175746F6D617469636B65208C
:104560007A61766164656E692066696C616D656EFD
:10457000747520646F737475706E6520706F757AD2
:104580006520707269207A61706E7574656D206641
:10459000696C616D656E742073656E7A6F72752ECD
:1045A0002E2E004175746F6C6F6164696E672066B2
:1045B000696C616D656E7420617661696C61626CB5
:1045C00065206F6E6C79207768656E2066696C6116
:1045D0006D656E742073656E736F722069732074DD
:1045E00075726E6564206F6E2E2E2E004348594200
:1045F000413A2046696C616D656E742073656E7A10
:104600006F72206E6572656167756A652C207A6BC2
:104610006F6E74726F6C756A7465207A61706F6A00
:10462000656E692E004552524F523A2046696C61C0
:104630006D656E742073656E736F72206973206E82
:104640006F7420726573706F6E64696E672C207072
:104650006C6561736520636865636B20636F6E6E64
:10466000656374696F6E2E005A6B616C6962726F5C
:104670007661740043616C696272617465005A30DE
:10468000005A31005930005931005830005831007B
:10469000456E642073746F707320646961670007EE
:1046A000441B4410442D4422443F44344487444630
:1046B000440F45CA44A34554452546EC4547383088
:1046C000004D3435205A00744668464D3234004D52
:1046D0003233202573006175746F25692E6700538E
:1046E000746F7265642073657474696E6773207289
:1046F0006574726965766564006563686F3A005435
:10470000726964656E6920736F75626F72750053AC
:104710006F7274696E672066696C6573004E656BB5
:104720007465726520736F75626F7279206E656251
:1047300075646F7520736574726964656E792E2077
:104740004D6178696D616C6E6920706F636574206E
:10475000736F75626F72752070726F2073657472FB
:104760006964656E69206A65203130302E00536FB0
:104770006D652066696C65732077696C6C206E6F5F
:104780007420626520736F727465642E204D6178A9
:104790002E204E6F2E206F662066696C657320692F
:1047A0006E203120666F6C64657220666F722073B4
:1047B0006F7274696E67206973203130302E005734
:1047C000726974696E6720746F2066696C653A203F
:1047D0000046696C652073656C65637465640020D0
:1047E00053697A653A200046696C65206F70656E82
:1047F00065643A20006F70656E206661696C65645F
:104800002C2046696C653A20004E65004E6F0041D1
:104810006E6F00596573000F47FF466E471D47BF17
:10482000472E002E00D147DF47E7472E00F5474EC1
:104830006F772066726573682066696C653A200040
:104840004E6F7720646F696E672066696C653A20E9
:10485000002220706F73002220706172656E743ABE
:104860002200535542524F5554494E452043414C26
:104870004C207461726765743A2200747279696EB3
:104880006720746F2063616C6C207375622D6763A1
:104890006F64652066696C6573207769746820743D
:1048A0006F6F206D616E79206C6576656C732E205C
:1048B0004D4158206C6576656C2069733A000C4850
:1048C00009483E0013480F483E0020003E003E00CD
:1048D000200000004041FFFFBF4000005C43FFFF9D
:1048E000BF4000005C430000464300004041000020
:1048F000464350726564656872656A7465207472B7
:1049000079736B75210050726568656174207468F5
:1049100065206E6F7A7A6C65210043485942413AAE
:10492000004552524F523A00506F64706F726100EE
:10493000537570706F727400537461746973746925
:104940006B61202000537461746973746963732010
:1049500020004B616C6962726163650043616C6940
:1049600062726174696F6E0056796A6D6F7574203A
:1049700066696C616D656E7400556E6C6F61642064
:1049800066696C616D656E74005A6176657374203A
:1049900066696C616D656E74004C6F616420666958
:1049A0006C616D656E74004175746F5A61766564F3
:1049B000656E692066696C2E004175746F4C6F617D
:1049C000642066696C616D656E74005A61646E6125
:1049D000205344206B61727461004E6F2053442059
:1049E0006361726400506F6B7261636F7661740013
:1049F000526573756D65207072696E7400506F7AC0
:104A000061737461766974207469736B00506175A9
:104A10007365207072696E740050726564656872A7
:104A200065760050726568656174004C61646974F4
:104A30000054756E6500446F6C6164656E69206F2B
:104A40007379205A004C6976652061646A757374C5
:104A5000205A00496E666F726D61636500496E662B
:104A60006F2073637265656E00446F6B6F6E636F6A
:104A700076616E6920706F687962750046696E694B
:104A80007368696E67206D6F76656D656E7473000F
:104A90004372617368206465742E20205B4E2F4141
:104AA0005D004372617368206465742E20205B7A18
:104AB00061705D004372617368206465742E20200C
:104AC000205B6F6E5D004372617368206465742EB5
:104AD00020205B7679705D004372617368206465A5
:104AE000742E20205B6F66665D004D6F6420202071
:104AF00020205B537465616C74685D004D6F646564
:104B0000202020205B537465616C74685D004D6FDC
:104B1000642020202020205B4E6F726D616C5D0050
:104B20004D6F646520202020205B4E6F726D616C9C
:104B30005D0046696C2E2073656E7A6F72205B7A19
:104B400061705D0046696C2E2073656E736F722014
:104B5000205B6F6E5D0046696C2E2073656E7A6F08
:104B600072205B7679705D0046696C2E2073656EED
:104B7000736F72205B6F66665D0056796D656E6956
:104B8000742066696C616D656E74004368616E6760
:104B9000652066696C616D656E7400507275746F26
:104BA0006B00466C6F7700527963686C6F737400AA
:104BB0005370656564000649F24821491A494D372A
:104BC000303200304928494661696C207374617441
:104BD0007300454938495C495249794968499949BE
:104BE0008949B949A7494661726D206E756D626544
:104BF0007200DA49CB49F049E5490D4AFD49234A9B
:104C0000194A314A2B4A454A364A5D4A534A7C4A38
:104C1000694A4D36303000904AB44AA24AD84AC652
:104C20004AFC4AEA4A204B0E4B444B324B684B56E7
:104C30004B8B4B7A4BA24B9B4BB04BA74B20746FCB
:104C40006F206C6F6E6720657874727573696F6E14
:104C50002070726576656E7465640020636F6C64A5
:104C600020657874727573696F6E207072657665F1
:104C70006E74656400062833D036C23E013F15418C
:104C800032423B43F2443B45F24622473B48F2491D
:104C90003B4AF05898590C5A085B0C5C0861106745
:104CA0009B6E2271077208FF095A0D000EFF19044E
:104CB0005E0820642B6D322FFF3D4C5B4C436879BE
:104CC0006261202D20446F736C6F206B20707265C1
:104CD00070697375207374617469636B65207061AA
:104CE0006D65746921004572726F72202D20737496
:104CF00061746963206D656D6F72792068617320DE
:104D00006265656E206F7665727772697474656E20
:104D1000004B617274612076796A6D75746100432D
:104D20006172642072656D6F766564004B617274A8
:104D30006120766C6F7A656E6100436172642069F0
:104D40006E73657274656400E64CBD4C1F4D114D69
:104D50003A4D2C4D00002100240027002A002D0090
:104D60003000330001010000040107010A010000C6
:104D700020002300260029002C002F003200000113
:104D8000000003010601090100000A0B02090C0DD5
:104D90000E080703040100000000000000000000EE
:104DA0000000000000000000000000000000000003
:104DB00000000000121110000000000000000000C0
:104DC00000000000000000000000000000000000E3
:104DD00000000000000000000000000000004E6520
:104DE000746F6369207365004E6F74207370696E11
:104DF0006E696E6700546F63692073650053706954
:104E00006E6E696E67004C6576792076656E7420EB
:104E10006E61207472797363653F004C656674201F
:104E2000686F74656E642066616E3F0050726564E1
:104E30006E69207469736B6F76792076656E743F46
:104E40000046726F6E74207072696E742066616EB7
:104E50003F00546573742076656E74696C61746F7D
:104E600072750046616E207465737400E84DDE4D06
:104E7000FD4DF54D1B4E064E414E2C4E634E524E8F
:104E8000010210202008081020401020408002015C
:104E90000201080402010102040810204080804041
:104EA0002010080402018004020180402010080440
:104EB00002010804020101020408102040800102DE
:104EC000040810204080100804088010204004408E
:104ED00080102040048000002200250028002B00C4
:104EE0002E003100340002010000050108010B0111
:104EF00005050505070508080808020202020A0A56
:104F00000808040404040101010101010101030373
:104F1000030303030303040707070C0C0C0C0C0C1E
:104F20000C0C0202020206060606060606060B0B1B
:104F30000B0B0B0B0B0B07070A0A0A0A0A0A0505DB
:104F40000504040408080222206661696C65643A5D
:104F5000204275666665722066756C6C2100456E30
:104F6000717565696E6720746F207468652066725C
:104F70006F6E743A2022004572726F723A002200FE
:104F8000456E717565696E6720746F207468652061
:104F900066726F6E743A202200207A203900206FEA
:104FA000662039004D6572696D20726566657265AF
:104FB0006E636E69207679736B75206B616C6962C4
:104FC0007261636E69686F20626F6475004D656120
:104FD000737572696E67207265666572656E63656A
:104FE00020686569676874206F662063616C696218
:104FF000726174696F6E20706F696E7400457872AB
:10500000656D65207370616E206F66207468652021
:105010005A2076616C756573210000004041FFFFE6
:10502000BF400000E442FFFFBF4000005743FFFFC6
:10503000BF40000057430000CC420000E4420000A3
:10504000CC42000040410000CC4200004041000042
:1050500046430000E442000046430000574300007E
:1050600046439E4F994FCD4FA44F53656E7A6F7252
:105070002066696C616D656E74750046696C616D62
:10508000656E742073656E736F720050726F686F17
:105090007A656E6500537761707065640050726563
:1050A000646E692F6C6576792076656E742E004685
:1050B000726F6E742F6C6566742066616E73004F3C
:1050C000736100417869730044656C6B61206F7394
:1050D000790041786973206C656E67746800557655
:1050E0006F6C6E656E612072656D656E69636B6174
:1050F000004C6F6F73652070756C6C657900456E40
:105100006473746F70206E6F742068697400456EEC
:105110006473746F70004D6F746F7200456E6473CA
:10512000746F7073004368796261207A61706F6A8E
:10513000656E6900576972696E67206572726F7279
:1051400000426564202F20486561746572004E65D9
:105150007A61706F6A656E6F20202020004E6F7438
:1051600020636F6E6E656374656400486561746585
:10517000722F546865726D6973746F72005A6B6F29
:105180006E74726F6C756A7465203A00506C65615C
:10519000736520636865636B203A0053656C6674C1
:1051A000657374206572726F7220210053656E7A88
:1051B0006F722066696C616D656E74753A00466940
:1051C0006C616D656E742073656E736F723A005416
:1051D00069736B6F76792076656E742E3A00507223
:1051E000696E742066616E3A004C6576792076654A
:1051F0006E742E3A0045787472756465722066612B
:105200006E3A0053656C66746573742073656C68E0
:10521000616C20200053656C667465737420666150
:10522000696C6564202000567365204F4B20202058
:10523000202020202020202000416C6C20636F72F1
:1052400072656374202020202020004B6F6E7472E2
:105250006F6C612073656E7A6F7275004368656369
:105260006B696E672073656E736F727320004B6F8E
:105270006E74726F6C6120626564202020202000B3
:10528000436865636B696E67206265642020202037
:1052900020004B6F6E74726F6C61205A20617869C8
:1052A00073202000436865636B696E67205A206134
:1052B0007869732020004B6F6E74726F6C61205997
:1052C0002061786973202000436865636B696E67AD
:1052D000205920617869732020004B6F6E74726FC3
:1052E0006C612058206178697320200043686563F1
:1052F0006B696E67205820617869732020004B6FBE
:105300006E74726F6C6120686F74656E642020002B
:10531000436865636B696E6720686F74656E6420AF
:1053200020004B6F6E74726F6C6120656E647374D5
:105330006F707300436865636B696E6720656E64A8
:1053400073746F70730041786973206C656E677455
:105350006820646966666572656E63653A004D65CE
:105360006173757265642061786973206C656E671E
:1053700074683A0025632041584953205347313D12
:1053800025640A007B506A5095508B50AF509D5059
:10539000C350BF50D250C850F150DE50FE500E5195
:1053A00016511C513451255141515D514E516B5193
:1053B0008C517D519B51BE51AC51DE51CF51F551B5
:1053C000E95115520352395227525C524B528052C6
:1053D0006E52A4529252C852B652EC52DA52105344
:1053E000FE52345322534572723A205052494E5461
:1053F0002046414E204552524F52004552524F5284
:105400003A205072696E742066616E207370656513
:1054100064206973206C6F776572207468656E20F4
:105420006578706563746564004572723A2045580A
:1054300054522E2046414E204552524F5200455262
:10544000524F523A204578747275646572206661D5
:105450006E207370656564206973206C6F77657268
:10546000207468656E20657870656374656400708B
:10547000012C0190012701B0012201C0011D01F0A2
:105480000118011002130130020E0160020901909F
:10549000020401C002FF000003FA004003F500808F
:1054A00003F000D003EB002004E6007004E100E00C
:1054B00004DC004005D700C005D2004006CD00D076
:1054C00006C8008007C3003008BE00F008B900C05D
:1054D00009B400B00AAF00B00BAA00D00CA50000C0
:1054E0000EA000500F9B00C01096005012910000BB
:1054F000148C00C0158700B0178200B0197D00D051
:105500001B7800001E730040206E0090226900F09E
:1055100024640040275F0090295A00E02B550010BA
:105520002E500020304B0010324600E033410090F6
:10553000353C001037370070383200A0392D00B0EC
:105540003A2800A03B2300603C1E00103D1900904B
:105550003D1400103E0F00703E0A00C03E050000E2
:105560003F000090137D00B0157800F017730060C5
:105570001A6E00F01C6900A01F640050225F00201A
:10558000255A00E0275500902A5000202D4B00A0FE
:105590002F4600F031410010343C00F0353700A0B8
:1055A00037320020392D00603A2800703B2300601C
:1055B0003C1E00203D1900C03D1400403E0F00A0DD
:1055C0003E0A00F03E0500403F0000703FFBFF90A8
:1055D0003FF6FFB03FF1FFC03FECFFD03FE7FFE0F9
:1055E0003FE2FFF03FDDFFF03FD8FF53746570727C
:1055F00061746520746F6F20686967683A2000EBFA
:105600005524F4D43050C38E20C2A24017828B7030
:1056100011127A910D816CD90AA861E108C7586608
:1056200007615143061E4B5D05C145A7041A411190
:1056300004093D9803713931034036DB026533912B
:1056400002D4305402802E1D02632CEE01752AC54F
:1056500001B028A001102781018F2564012B244B64
:1056600001E0223401AC211F018D200D01801FFCBF
:1056700000841EED00971DDF00B81CD200E61BC69B
:1056800000201BBC00641AB200B219A8000A19A0BD
:10569000006A189900D117910040178B00B5168445
:1056A0000031167E00B31579003A157300C7146FE8
:1056B0000058146A00EE1366008813630025135E19
:1056C00000C7125B006C12570015125400C1115133
:1056D0000070114F0021114B00D61049008D10476A
:1056E000004610440002104200C00F4000800F3EF0
:1056F00000420F3C00060F3B00CB0E3800930E37E4
:10570000005C0E3500270E3400F30D3200C10D3160
:1057100000900D3000600D2E00320D2D00050D2C77
:1057200000D90C2B00AE0C2900850C29005C0C273D
:1057300000350C27000E0C2600E80B2400C40B24B7
:1057400000A00B23007D0B23005A0B2100390B21F5
:1057500000180B2000F80A1F00D90A1E00BB0A1E01
:10576000009D0A1D00800A1D00630A1C00470A1BD9
:10577000002C0A1B00110A1A00F7091A00DD09198A
:1057800000C4091900AB091900920917007B091818
:1057900000630917004C0916003609160020091687
:1057A000000A091500F5081500E0081400CC0814DB
:1057B00000B8081400A4081400900813007D081213
:1057C000006B081300580812004608120034081134
:1057D00000230811001208110001081100F0071041
:1057E00000E0071000D0071000C0071000B0070F3E
:1057F00000A107100091070E0083070F0074070F28
:105800000065070E0057070E0049070E003B070D05
:10581000002E070E0020070D0013070D0006070DD0
:1058200000F9060C00ED060D00E0060C00D4060C95
:1058300000C8060C00BC060C00B0060C00A4060B49
:105840000099060C008D060B0082060B0077060BF4
:10585000006C060B0061060A0057060B004C060A96
:105860000042060A0038060A002E060A0024060A2C
:10587000001A060A001006090007060A00FD0509BD
:1058800000F4050900EB050900E2050900D9050946
:1058900000D0050900C7050900BE050900B50508C7
:1058A00000AD050800A50509009C05080094050841
:1058B000008C050800840508007C050800740508B4
:1058C000006C050700650508005D05070056050822
:1058D000004E05070047050700400508003805078A
:1058E00000310507002A050700230507001C0506EF
:1058F00000160507000F050700080506000205074A
:1059000000FB040600F5040700EE040600E80406A8
:1059100000E2040700DB040600D5040600CF0406FD
:1059200000C9040600C3040600BD040600B704064F
:1059300000B1040500AC040600A6040600A004059E
:10594000009B04060095040500900406008A0405E7
:105950000085040500800406007A0405007504052E
:1059600000700405006B0405006604050061040571
:10597000005C04050057040500520405004D0405B1
:105980000048040500430405003E0404003A0405F1
:105990000035040500300404002C0405002704042D
:1059A00000230405001E0404001A04040016040564
:1059B00000110404000D040400090405000404049B
:1059C0000000040400FC030400F8030400F40304D2
:1059D00000F0030400EC030400E8030400E4030403
:1059E00000E0030400DC030400D8030400D4030433
:1059F00000D0030400CC030400C8030300C5030364
:105A00000024F404D9201BC40C5C0E9804C4095F64
:105A10000265077101F405F900FB04B3004804872F
:105A200000C10369005803550003034500BE023A54
:105A3000008402310053022A0029022500040220BA
:105A400000E4011C00C8011900AF011700980114FF
:105A50000084011300710110006101100051010E5A
:105A60000043010D0036010B002B010B0020010B40
:105A700000150109000C01090003010800FB0008E2
:105A800000F3000800EB000700E4000600DE00065B
:105A900000D8000600D2000600CC000500C70005B3
:105AA00000C2000500BD000400B9000400B50004F8
:105AB00000B1000400AD000400A9000400A500032B
:105AC00000A20003009F0004009B00030098000355
:105AD000009500020093000300900003008D000277
:105AE000008B00030088000200860002008400038F
:105AF00000810002007F0002007D0002007B0002A6
:105B000000790002007700010076000200740002B4
:105B10000072000100710002006F0002006D0001C0
:105B2000006C0002006A00010069000200670001C9
:105B300000660001006500010064000200620001CF
:105B40000061000100600001005F0002005D0001D3
:105B5000005C0001005B0001005A000100590001D7
:105B600000580001005700010056000100550001D7
:105B700000540001005300000053000100520001D6
:105B80000051000100500001004F0001004E0000D4
:105B9000004E0001004D0001004C0001004B0000D0
:105BA000004B0001004A00010049000100480000CC
:105BB00000480001004700010046000000460001C7
:105BC00000450000004500010044000100430000C2
:105BD00000430001004200000042000100410000BB
:105BE0000041000100400001003F0000003F0001B3
:105BF000003E0000003E0001003D0000003D0001AD
:105C0000003C0000003C0000003C0001003B0000A4
:105C1000003B0001003A0000003A0001003900009A
:105C20000039000100380000003800000038000191
:105C30000037000000370001003600000036000089
:105C4000003600010035000000350000003500017D
:105C50000034000000340000003400010033000074
:105C60000033000000330001003200000032000069
:105C7000003200010031000000310000003100015D
:105C8000003000000030000000300001002F000054
:105C9000002F0000002F0000002F0001002E000048
:105CA000002E0000002E0001002D0000002D00003D
:105CB000002D0000002D0001002C0000002C000031
:105CC000002C0000002C0001002B0000002B000025
:105CD000002B0000002B0001002A0000002A000019
:105CE000002A0000002A000100290000002900000D
:105CF0000029000000290000002900010028000000
:105D000000280000002800000028000000280001F2
:105D100000270000002700000027000000270000E7
:105D200000270001002600000026000000260000D9
:105D300000260000002600010025000000250000CC
:105D400000250000002500000025000000250001BE
:105D500000240000002400000024000000240000B3
:105D600000240001002300000023000000230000A5
:105D70000023000000230000002300000023000196
:105D8000002200000022000000220000002200008B
:105D9000002200000022000100210000002100007C
:105DA000002100000021000000210000002100006F
:105DB0000021000100200000002000000020000061
:105DC0000020000000200000002000000020000053
:105DD00000200001001F0000001F0000001F000045
:105DE000001F0000001F0000001F0000001F000136
:105DF000001E0000001E0000001E0000001E00002B
:105E00000043616E6E6F7420656E746572207375E9
:105E1000626469723A200053442063617264206FA7
:105E20006B006F70656E526F6F74206661696C6590
:105E30006400766F6C756D652E696E69742066619D
:105E4000696C656400534420696E697420666169F9
:105E50006C00332E312E312D5243350072630062B7
:105E600065746100616C7068610064657600015E54
:105E70006F6B0A002046002045004731205A00176A
:105E80005E225E325E455E527963686C6F73742089
:105E900076656E742E0046616E20737065656400D1
:105EA00042656400547279736B61004E6F7A7A6C4C
:105EB00065004E6173746176656E69005365747434
:105EC000696E6773005469736B20707265727573C5
:105ED000656E005072696E742061626F72746564E1
:105EE000005A61737461766974207469736B00532E
:105EF000746F70207072696E7400536F75626F7288
:105F0000206E656B6F6D706C65746E692E20506FBE
:105F10006B7261636F7661743F0046696C652069DE
:105F20006E636F6D706C6574652E20436F6E74695F
:105F30006E756520616E797761793F005469736B86
:105F4000207A205344005072696E742066726F6D1F
:105F500020534400486C61766E69206E616269640A
:105F60006B61004D61696E00965E875EA05EAB5E00
:105F7000A45EBC5EB25ED35EC55EEF5EE15E4D3296
:105F800034001A5FFA5E4D323320257300465F3CC1
:105F90005F052E2E00635F545F526573656E643A31
:105FA00020004B494C4C45442E20005072696E74C1
:105FB00065722068616C7465642E206B696C6C2856
:105FC000292063616C6C656421004D3232312049B7
:105FD0006E76616C69642065787472756465722090
:105FE000004D32313820496E76616C6964206578E5
:105FF00074727564657220004D31303920496E76B7
:10600000616C696420657874727564657220004DF6
:1060100031303520496E76616C6964206578747220
:106020007564657220004D31303420496E76616CA4
:1060300069642065787472756465722000995F4D9B
:1060400037303100A25FAB5F4B494C4C3A2000CA5D
:106050005FE15FF85F0F6026605370757374656E63
:10606000692057697A617264612076796D617A6519
:1060700020756C6F7A656E65207679736C65646BDC
:1060800079207673656368206B616C696272616305
:1060900069206120737075737469206B616C69622B
:1060A0007261636E692070726F636573206F642024
:1060B0007A616361746B752E20506F6B7261636FD0
:1060C0007661743F0052756E6E696E672057697A0B
:1060D0006172642077696C6C2064656C65746520FE
:1060E00063757272656E742063616C69627261744B
:1060F000696F6E20726573756C747320616E6420B5
:1061000073746172742066726F6D207468652062AA
:106110006567696E6E696E672E20436F6E74696E77
:1061200075653F005465706C6F742E206B616C69EF
:1061300062726163650054656D702E2063616C69E5
:1061400062726174696F6E0052657365742058598C
:106150005A206B616C6962722E00526573657420FF
:1061600058595A2063616C6962722E0053746176CB
:10617000206B6F6E632E207370696E2E0053686FF4
:106180007720656E642073746F70730050494420EB
:106190006B616C69627261636500504944206361A0
:1061A0006C6962726174696F6E004B6F72656B63CC
:1061B0006520706F646C6F7A6B7900426564206C47
:1061C0006576656C20636F7272656374004D6573EC
:1061D0006820426564204C6576656C696E67004B8B
:1061E000616C6962726F766174205A0043616C69F8
:1061F0006272617465205A004B616C6962726163FE
:10620000652058595A0043616C6962726174652057
:1062100058595A0053656C667465737420202020A9
:106220002020202020004175746F20686F6D65006C
:106230004B616C2E207072766E6920767273747664
:1062400079004669727374206C61796572206361AC
:106250006C2E0057697A6172640043657374696ECD
:106260006100456E676C69736800C56059604D34A4
:106270003500366124614D3434005A6148617D61D6
:106280006C619A618C61BB61AA61CD61EC61DF6177
:106290000662F86114624732382057002662426273
:1062A0003062536262625A6243656B616E69206E4E
:1062B00061207A63686C61646E75746920747279A8
:1062C000736B79206120706F646C6F7A6B792E002C
:1062D00057616974696E6720666F72206E6F7A7A93
:1062E0006C6520616E642062656420636F6F6C6909
:1062F0006E670053656C662074657374204F4B00A5
:1063000053656C66207465737420737461727420B5
:106310002000D062A862F3624D3834004731205A21
:1063200031350047323820570000635469736B2EB3
:106330002076656E743A005072696E742046414E44
:106340003A2000547279736B2E2076656E743A0091
:106350004E6F7A7A6C652046414E3A0037632B6364
:106360005063436346696C616D656E742076797421
:106370006C6163656E20612073707261766E65205A
:1063800062617276793F0046696C616D656E74205A
:10639000657874727564696E672026207769746801
:1063A00020636F727265637420636F6C6F723F005D
:1063B000876364634001960111241FBECFEFD1E2D1
:1063C000DEBFCDBF00E00CBF18E0A0E0B2E0ECE51E
:1063D000FBE703E00BBF02C007900D92AC34B1079E
:1063E000D9F72AE1ACE4B8E001C01D92AA3CB2079B
:1063F000E1F711E3CBEDD1E300E006C021970109FD
:10640000802FFE010F946BBCCA3DD10780E00807C6
:10641000A9F70F94CC940D949DBD0C9400002F927D
:106420003F924F925F926F927F928F929F92AF9224
:10643000BF92CF92DF92EF92FF920F931F93CF9371
:10644000DF93CDB7DEB7CC58D1090FB6F894DEBFD5
:106450000FBECDBF82E090E09093730280937202F2
:1064600087EB93E00E9429998823B1F08091550829
:10647000909156086AE270E005960F94D2BC00979E
:1064800011F0DC011C9280915508909156080596F8
:106490000F94A83F0C94A0678CEB93E00E9429997D
:1064A000882389F10F94EC6F81E00F945C420E9485
:1064B000ABEF82E00F94EB4086E69FE00F94F8B6D6
:1064C00061E0680F86E69FE00F940AB781E00F94C1
:1064D0005C4282E00F94EB40E091AB0FF0E0EE0FF6
:1064E000FF1FE25CF34F859194910F94933F61E01D
:1064F00086E39CE00E94477461E088E29CE00E9491
:1065000047740C94A0678BEC93E00E942999882330
:1065100051F08091131581110F94BA7B81E0809323
:1065200011020C94A06789ED93E00E9429998823B9
:1065300049F01092270C0F94B34681E0809311022A
:106540000C94A06786EE93E00E942999882309F4B1
:1065500082C18CEE93E00E942999882391F080916A
:10656000480F882311F40C94A0670F94133C609398
:10657000210C7093220C8093230C9093240C0C9488
:10658000A06781EF93E00E942999882341F08091D0
:10659000210A9091220A0F94ED060C94A06785EFD2
:1065A00093E00E9429998823F1F109EF13E0F801A3
:1065B00081918F01882319F00E947986F8CF80910C
:1065C000AF1A9091B01A2CE3289FB001299F700D4B
:1065D0001124072E000C880B990B0F9496038DEF56
:1065E00093E00F94DB0602E014E0D8018D918D0159
:1065F000882319F00E947986F8CF8091B11A909182
:10660000B21A2CE3289FB001299F700D1124072E88
:10661000000C880B990B0F9496038DEF93E00F9469
:10662000DB060C94A06788E094E00E9429998823F7
:1066300091F08091480F882341F0809184089091D7
:1066400085080F94E7060C94A0678BE094E00F9404
:10665000DB060C94A0678DE194E00E9429998823C1
:1066600039F1809155089091560841E061E0039618
:106670000F940B188091880E9091890EA0918A0E2C
:10668000B0918B0E8093350F9093360FA093370FF8
:10669000B093380F80E89EE00E94737B8C010E94CB
:1066A00079860A30110531F70F94B3460C94A06730
:1066B00080E294E00E942999882381F00E94E79368
:1066C00081E08093AA08809155089091560841E096
:1066D00060E004960F940B180C94A06784E294E099
:1066E0000E9429998823C9F18091480F882309F4D1
:1066F000ACCF1092B30A07E214E0F80181918F0148
:10670000882319F00E947986F8CF00E010E0FF247A
:10671000F3948091AF0A9091B00A2091B10A309120
:10672000B20A821B930B8F779927892B59F00F940C
:10673000B906F092B30A0E9479860F5F1F4F10923C
:10674000B30AE7CF0331110524F381E08093B30A44
:106750008AE00E9479860C94A0678AE294E00E9405
:106760002999882379F00EE214E0D8018D918D01EA
:10677000882319F00E947986F8CF8AE00E947986F2
:106780000C94A06788E394E00E942999882351F033
:106790000CE314E0F80181918F01882371F30E94CA
:1067A0007986F8CF8AE594E00E942999882321F020
:1067B0000E945CFC0C94A0678FE594E00E942999EC
:1067C000882341F060E070E088EF9FE00E9448EC91
:1067D0000C94A06782E694E00E942999882349F0EE
:1067E00082E694E00F94DB0660E072EC81E090E0DA
:1067F0000EC08DE694E00E942999882361F08DE611
:1068000094E00F94DB0660E074E981E190E00F947E
:106810003D060C946C7389E794E00E9429998823C3
:1068200061F00F94133C60931D0C70931E0C8093C9
:106830001F0C9093200C0C94A0678EE794E00E94AC
:106840002999882311F40C94A06761E080E00E94EC
:10685000999C0C94A0678EE50E943D9929968FAF74
:10686000299781110C94A06787E40E943D99F82E26
:10687000882311F40C94D9430E9420990F94E3B813
:106880006C34710509F4E7C38CF56430710509F4C3
:106890000AC154F46230710509F4EDC00CF0F7C080
:1068A00077FF79C00C94BF436C31710509F44FC177
:1068B00074F46A30710509F445C16B30710511F04B
:1068C0000C94BF4380E00F9481A30C94A0676E31B9
:1068D000710509F41BC36B34710511F00C94BF43AF
:1068E00048E2C42ED12CE12CF12CA4C368357105EB
:1068F00011F40C94A0670CF56135710511F40C943A
:106900009A4264F46F34710511F40C94CE3C6035F6
:10691000710511F40C94023D0C94BF43663571056A
:1069200011F40C9443436735710511F00C94BF4387
:1069300081E00E9452990C94A0676C35710511F4A6
:106940000C944C437CF46A35710511F40C94484363
:106950006B35710511F00C94BF4381E08093911A5F
:106960000C94A0676236710511F40C94AA43633647
:10697000710511F00C94BF431092480F81E0809391
:106980006D0260E084EC9FE00F940AB782E00F9400
:10699000EB400C94A06780916B0981110C94A06767
:1069A0000F94D8AB60915B1A70915C1A80915D1A5C
:1069B00090915E1A0F9485B16B017C014090F50FA8
:1069C0005090F60F6090F70F7090F80F80900F15B1
:1069D00090901015A0901115B0901215A50194017A
:1069E000C301B2010F9483B720E030E048EC52E4D9
:1069F0000F94D4AC9B01AC01C701B6010F94CFB981
:106A00001816E4F4A3019201C501B4010F9483B7F1
:106A100020E030E048EC52E40F94D4AC9B01AC0190
:106A2000C701B6010F9484B70F94E9B860935B1A5D
:106A300070935C1A80935D1A90935E1A8091BD0AE0
:106A40008823A9F088E50E943D99811110C089E54D
:106A50000E943D9981110BC08AE50E943D998111E8
:106A600006C085E40E943D9981110C94CD670F9476
:106A700095A90C94A06780916B0981110C94A06773
:106A80000F945BAC81E00F94F1A50C94A06780910A
:106A90006B0981110C94A0670F945BAC80E00F949C
:106AA000F1A50C94A06780E50E943D99882339F0F8
:106AB0000E9420990F94E9B86B017C0103C0C12C9E
:106AC000D12C760183E50E943D99882361F00E94D4
:106AD000209920E030E04AE754E40F94D4AC0F94BE
:106AE000E9B86B017C01C114D104E104F10431F077
:106AF000E1E4F4E1859194910F94933F0F94EC6F4E
:106B00000F94133CC60ED71EE81EF91E0F94133CBB
:106B10006093961A7093971A8093981A9093991A83
:106B20000F94133C6C157D058E059F0510F00C9499
:106B3000A0670F94526980E00F94C88780E00F949B
:106B4000EB40EECF81E00F9481A30C94A0670F94EB
:106B5000EC6F81E080936B1A88E50E943D99182FB5
:106B600089E50E943D99082F8AE50E943D99682E8B
:106B7000101308C0181711F0012F04C06624639485
:106B800001E011E00F94775A5090480B1092480B97
:106B900082E00F94D96F6093F10F7093F20F80939E
:106BA000F30F9093F40F61100F9417A38091860256
:106BB00090918702A0918802B091890280934C083D
:106BC00090934D08A0934E08B0934F0880916702B0
:106BD00090916802909321098093200984E690E0C7
:106BE00090936802809367020F94133C6093961A07
:106BF0007093971A8093981A9093991A81E08093D2
:106C0000620280E1E9EEFFE0A3E0B5E101900D92C0
:106C10008A95E1F7109286021092870210928802FC
:106C200010928902112321F080E090E00E94B69436
:106C3000002321F081E090E00E94B69488E50E9454
:106C40003D99882341F00F94EC9F672B682B692BAB
:106C500011F00C94FC6789E50E943D99882341F06E
:106C60000F94EC9F672B682B692B11F00C94126822
:106C7000662009F4DDC080917A08882321F0809194
:106C80007B08811108C080E090E00E94B69481E00A
:106C900090E00E94B6940F94495BEEE1F0E5859197
:106CA0009591A591B49188A399A3AAA3BBA3EAE166
:106CB000F0E585919591A591B49189839A83AB83F1
:106CC000BC8327E035E143E055E1BE01605E7F4FC4
:106CD000CE0101960E946C990F94CB5A20E030E0CF
:106CE00040E850EC609107157091081580910915E6
:106CF00090910A150F9481B187FF0CC080E090E05D
:106D0000A0E8B0EC8093071590930815A09309159F
:106D1000B0930A1580E090E0A0EAB0E480930B15F0
:106D200090930C15A0930D15B0930E1580E090E094
:106D3000A0EAB2E48093860290938702A09388022F
:106D4000B09389021092F10F1092F20F1092F30F8C
:106D50001092F40F109262022091ED0F3091EE0F1D
:106D60004091EF0F5091F00F6091E90F7091EA0F91
:106D70008091EB0F9091EC0FE12CF12C87010F9497
:106D8000D94C8090860290908702A0908802B090A3
:106D90008902E0900B15F0900C1500910D151091E3
:106DA0000E15209107153091081540910915509145
:106DB0000A15609103157091041580910515909145
:106DC0000615E4E1F5E1FF93EF93EFE0CE2EE5E168
:106DD000DE2E0F949D280F94EC6F809103159091F7
:106DE0000415A0910515B09106158093E90F9093B5
:106DF000EA0FA093EB0FB093EC0F809107159091E1
:106E00000815A0910915B0910A158093ED0F909384
:106E1000EE0FA093EF0FB093F00F81E0809362022A
:106E20000F94BC7882E090E00E94B6940F900F908F
:106E30008AE50E943D99882341F00F94EC9F672BCF
:106E4000682B692B11F00C942868E090F10FF090FA
:106E5000F20F0091F30F1091F40F2091ED0F30918C
:106E6000EE0F4091EF0F5091F00F6091E90F70918C
:106E7000EA0F8091EB0F9091EC0F0F94D94C109288
:106E8000620280914C0890914D08A0914E08B091FB
:106E90004F088093860290938702A0938802B09354
:106EA0008902809120099091210990936802809332
:106EB00067020F94133C6093961A7093971A80930D
:106EC000981A9093991A0F94BC780F94495B0F9479
:106ED000B15888E50E943D9981110C94496789E574
:106EE0000E943D9981110C94496787E50E943D9964
:106EF00081110C9449678AE50E943D9981110C9497
:106F000049670F94EC6F10926B1A7CC50F94EC6F6D
:106F100081E00E942A9480E090E0A8E4B4E48093A9
:106F2000860290938702A0938802B093890260E062
:106F300070E080E291EC0F949116ECE6FFE505918C
:106F40001491F8018491882329F00E9479860F5FBB
:106F50001F4FF7CFECE3F4E184918F01882339F0E0
:106F60000E9479860F5F1F4FF8018491F7CF6091DF
:106F7000E90F7091EA0F8091EB0F9091EC0F45E0D3
:106F80000F94B103E7E3F4E184918F01882339F092
:106F90000E9479860F5F1F4FF8018491F7CF6091AF
:106FA000ED0F7091EE0F8091EF0F9091F00F45E093
:106FB0000F94B103E2E3F4E184918F01882339F067
:106FC0000E9479860F5F1F4FF8018491F7CF60917F
:106FD000F10F7091F20F8091F30F9091F40F45E053
:106FE0000F94B103E0E3F4E184918F01882339F039
:106FF0000E9479860F5F1F4FF8018491F7CF0E949E
:1070000005940C94A067B801110F880B990B0F948D
:1070100087B10E944E8F0F94F306BFEFCB1ADB0AA5
:10702000EB0AFB0AEFE6CE16D104E104F10411F4F9
:107030000C94A0678601C701B6010F9496033DE149
:10704000A32E38E0B32ED5018D915D018823D9F2AE
:107050000E947986F8CF80917A08882341F0809148
:107060007B08882321F080917C08811109C081E090
:1070700080931F1289E294E10F94F2420C94A0676E
:1070800081E090E09093730280937202EBE0F4E170
:1070900084918F01882339F00E9479860F5F1F4FFA
:1070A000F8018491F7CF8AE00E9479861A821982CA
:1070B000C0904009D0904109E0904209F090430906
:1070C00020E030E040EA50E4C701B6010F9472B806
:1070D0000F94E3B825E0269FA001279F500D1124AF
:1070E000BA01550F880B990B0F9487B11B012C0126
:1070F00020E030E04CE052E40F9481B187FF06C0FD
:10710000212C312C2CE0422E22E4522EA701960194
:10711000C201B1010F9481B187FF0AC020E030E0C5
:1071200040EA50E4C201B1010F9484B71B012C0165
:10713000E7EFF3E184918F01882339F00E9479868B
:107140000F5F1F4FF8018491F7CFC201B1010F9477
:10715000F30620E030E040EF51E4C201B1010F94AA
:1071600083B720E030E04CE852E40F9484B70F94EA
:10717000E3B8709395086093940884E090E090934E
:107180004C0F80934B0F81E090E090931B0980930C
:107190001A09E091AB0FF0E0EE0FFF1FED59FC4B29
:1071A00025913491232B09F480E080934D0F80E0EA
:1071B00090E0A0EAB1E48093E90F9093EA0FA093E6
:1071C000EB0FB093EC0F80E090E0A0E7B2E4809387
:1071D000ED0F9093EE0FA093EF0FB093F00F8AE9AD
:1071E00099E9A9E1BEE38093F10F9093F20FA09388
:1071F000F30FB093F40F84E195E19F938F93812C6B
:10720000912C18E4A12E12E4B12E05EFC02E0FE050
:10721000D02E1AE9E12E19E9F12E09E11EE320E052
:1072200030E040E752E460E070E080EA91E40F94DF
:107230009D280F94EC6F0F900F90A2019101609127
:1072400040097091410980914209909143090F943E
:1072500081B187FF07C088EE93E00E9480930E946F
:10726000F88EEBCF60E086EA9FE00F940AB780E0EB
:1072700090E0A0EAB0E48093F10F9093F20FA09316
:10728000F30FB093F40F2091ED0F3091EE0F40917A
:10729000EF0F5091F00F6091E90F7091EA0F80911C
:1072A000EB0F9091EC0FE4E16E2EE5E17E2E7F92E4
:1072B0006F92812C912CF8E4AF2EF2E4BF2EA5EF53
:1072C000CA2EAFE0DA2EE12CF12C00EA10E40F9484
:1072D0009D28EAE1F0E5659175918591949160931F
:1072E000E90F7093EA0F8093EB0F9093EC0FEEE1B0
:1072F000F0E525913591459154912093ED0F309310
:10730000EE0F4093EF0F5093F00FE090F10FF090DD
:10731000F20F0091F30F1091F40F7F926F920F9480
:107320009D280F94EC6F60E070E080E89FEB0F9475
:1073300091168090F10F9090F20FA090F30FB09003
:10734000F40F2C968CAE9DAEAEAEBFAE2C97E6EF92
:10735000F3E184910F900F900F900F908F0188238D
:1073600039F00E9479860F5F1F4FF8018491F7CFA3
:107370008AE00E947986EFEEF3E184918F01882301
:1073800039F00E9479860F5F1F4FF8018491F7CF83
:107390006091F10F7091F20F8091F30F9091F40FC3
:1073A00042E00F94B103EEEEF3E184918F01882364
:1073B00039F00E9479860F5F1F4FF8018491F7CF53
:1073C0008AE00E9479865EEA652E5FE0752E812C48
:1073D000912C5401839473E2C72ED12CE12CF12C13
:1073E00062969FAE8EAE6297A401425051092896D4
:1073F0005FAF4EAF2897B6010D2C000C880B990B90
:107400000F9487B160966CAF7DAF8EAF9FAF6097E2
:10741000E7EEF3E184918F01882339F00E947986A9
:107420000F5F1F4FF8018491F7CFC501B4010F948E
:107430009603EAEDF3E184918F01882339F00E94ED
:1074400079860F5F1F4FF8018491F7CF8AE00E9481
:107450007986E6ECF3E184918F01882339F00E946C
:1074600079860F5F1F4FF8018491F7CFC701B601EE
:107470000F949603E7EBF3E184918F01882339F0B1
:107480000E9479860F5F1F4FF8018491F7CF60E06B
:1074900070E0CB010F949603E6EBF3E184918F014A
:1074A000882339F00E9479860F5F1F4FF80184917D
:1074B000F7CF8AE00E94798628962EAD3FAD2897B7
:1074C0002F3F3F4F11F40C945C73BE016F5F7F4FF1
:1074D000C3010E9448EC60962CAD3DAD4EAD5FAD52
:1074E0006097C201B1010F9481B11816D4F462966D
:1074F0008EAD9FAD6297069771F0F5E0CF0ED11C6F
:10750000E11CF11C2FEF821A920AA20AB20A32E0A1
:10751000630E711C65CFA5E0B0E02896BFAFAEAF9B
:107520002897412C512C32012896EEADFFAD2897BB
:1075300031966496FFAFEEAF6497CF01FF0FAA0BB1
:10754000BB0B9C01AD012E5F3F4F4F4F5F4F6A96C3
:107550002CAF3DAF4EAF5FAF6A9728964EAD5FAD93
:1075600028974D5F5F4F6C965FAF4EAF6C9744E1CD
:10757000242E45E1342E28968EAD9FAD2897875254
:10758000984F6E969FAF8EAF6E9762965FAE4EAE7F
:10759000629764968EAD9FAD6497840D951D059797
:1075A00008F0C3C128968EAD9FAD2897840D951D18
:1075B00025E0289FB001299F700D1124635D7F4F46
:1075C000072E000C880B990B0F9487B160966CAF57
:1075D0007DAF8EAF9FAF6097EFEAF3E184918F01AB
:1075E000882339F00E9479860F5F1F4FF80184913C
:1075F000F7CF6A966CAD7DAD8EAD9FAD6A97640D89
:10760000751D861D971D0F949603ECEAF3E1849196
:107610008F01882339F00E9479860F5F1F4FF80190
:107620008491F7CF8AE00E9479866C968EAD9FADEB
:107630006C9762968EAC9FAC6297880D991D909363
:107640001B0980931A0920E030E040EF51E4609676
:107650006CAD7DAD8EAD9FAD60970F9483B720E08C
:1076600030E040E251E40F94D4AC20E030E040EA56
:1076700050E40F9472B820E030E048E452E40F94F4
:1076800084B70F94E3B8709395086093940820E052
:1076900030E040EA51E42093E90F3093EA0F409341
:1076A000EB0F5093EC0F80E090E0A0E7B2E4809302
:1076B000ED0F9093EE0FA093EF0FB093F00F1AE938
:1076C000812E19E9912E19E1A12E1EE3B12E80928F
:1076D000F10F9092F20FA092F30FB092F40F3F923D
:1076E0002F92812C912C08E4A02E02E4B02E25EFDD
:1076F000C22E2FE0D22E1AE9E12E19E9F12E09E16E
:107700001EE39C01AD0160E070E080EA91E40F941B
:107710009D280F94EC6F0F900F9060962CAD3DADAF
:107720004EAD5FAD609760914009709141098091C5
:107730004209909143090F9481B187FF07C088EEF9
:1077400093E00E9480930E94F88EE7CF80E090E063
:10775000A0EAB0E48093F10F9093F20FA093F30F9F
:10776000B093F40F2091ED0F3091EE0F4091EF0F99
:107770005091F00F6091E90F7091EA0F8091EB0F3B
:107780009091EC0F3F922F92812C912C08E4A02E27
:1077900002E4B02EE5EFCE2EEFE0DE2EE12CF12C50
:1077A00000EA10E40F949D28EAE1F0E565917591F7
:1077B000859194916093E90F7093EA0F8093EB0F9A
:1077C0009093EC0FEEE1F0E52591359145915491C0
:1077D0002093ED0F3093EE0F4093EF0F5093F00F87
:1077E000E090F10FF090F20F0091F30F1091F40F71
:1077F0003F922F920F949D280F94EC6F60E070E001
:1078000080E89FEB0F9491162C962CAD3DAD4EADBC
:107810005FAD2C976091F10F7091F20F8091F30F93
:107820009091F40F0F9483B720911A0B30911B0B9A
:1078300040911C0B50911D0B0F94D4AC0F94E3B8E6
:107840007A836983EBEAF3E184910F900F900F90B4
:107850000F908F01882339F00E9479860F5F1F4FA8
:10786000F8018491F7CF8AE00E947986E7E9F3E195
:1078700084918F01882339F00E9479860F5F1F4F12
:10788000F8018491F7CF609140097091410980918E
:1078900042099091430942E00F94B103E8E8F3E113
:1078A00084918F01882339F00E9479860F5F1F4FE2
:1078B000F8018491F7CF2C962CAD3DAD4EAD5FAD68
:1078C0002C976091F10F7091F20F8091F30F9091CE
:1078D000F40F0F9483B742E00F94B103E7E8F3E1AC
:1078E00084918F01882339F00E9479860F5F1F4FA2
:1078F000F8018491F7CF8AE00E9479866E968EAD6A
:107900009FAD6E9762968EAC9FAC6297880D991D65
:10791000BE016F5F7F4F880F991F0E9448EC2FEFC9
:10792000421A520A620A720A30CE10924C0F10921A
:107930004B0F10924D0F61E086EA9FE00F940AB75B
:10794000E8E4F3E184918F01882339F00E9479867D
:107950000F5F1F4FF8018491F7CF8AE00E9479866C
:10796000179A10927A08169A10927B08149A10921D
:10797000950810929408E091AB0FF0E0EE0FFF1F16
:10798000EC5BFC4E859194910E9419EB81E00F9481
:107990005C4282E00F94EB400C94A067C12CD12C88
:1079A0007601CA94A1E4AA2EA3E1BA2ED092A90F1F
:1079B000C092A80F04E610E084E690E00E94809355
:1079C00001501109C9F7C701B6010F949603F501DB
:1079D000849101E413E1882339F00E9479860F5FD6
:1079E0001F4FF8018491F7CF8091B11A9091B21A8C
:1079F0000F94E706F5E0CF1AD108E108F108B1F6D7
:107A00000C94A06781E080936C1A86E50E943D99F2
:107A1000882359F0E0915508F0915608818189300A
:107A200021F08F7D11F00E94139920917A088091A6
:107A3000670F9091680F222341F020917B08222349
:107A400021F060907C0861100FC0029749F081E03E
:107A500080931F128AE393E10F94F2420C94A06783
:107A600010926C1A0C94A067109254080297C1F3FC
:107A700080904D0F63968FAE6397A0904B0FB090A0
:107A80004C0F6896BFAEAEAE689720911A09309140
:107A90001B096C963FAF2EAF6C9781E080934D0F22
:107AA00081E090E090934C0F80934B0F83E190E046
:107AB00090931B0980931A0981E00F94EB400F9477
:107AC0005D4E0F9417A380E090E0A0EAB0E48093AD
:107AD000F10F9093F20FA093F30FB093F40F209156
:107AE000ED0F3091EE0F4091EF0F5091F00F60913C
:107AF000E90F7091EA0F8091EB0F9091EC0FE4E1A8
:107B00004E2EE5E15E2E5F924F92F5E58F2E982C7A
:107B1000A82CF1E4BF2EA5EFCA2EAFE0DA2EE12C9F
:107B2000F12C00EA10E40F949D28EAE1F0E585913C
:107B30009591A591B4918093E90F9093EA0FA0934A
:107B4000EB0FB093EC0FEEE1F0E585919591A591E7
:107B5000B4918093ED0F9093EE0FA093EF0FB0933D
:107B6000F00F6DEE7FE089EE9FE00E94239AE09097
:107B7000F10FF090F20F0091F30F1091F40F20919C
:107B8000ED0F3091EE0F4091EF0F5091F00F60919B
:107B9000E90F7091EA0F8091EB0F9091EC0F5F92DB
:107BA0004F92812C912CE8ECAE2EE2E4BE2E0F9485
:107BB0009D280F94EC6F0F900F900F900F9005EC95
:107BC0001FE0C8010F9405B7019649F00E5F1F4FE3
:107BD000053D4FE01407A9F729966FAE299780E07D
:107BE0000E942A948AE190E52E969FAF8EAF2E9741
:107BF00028961FAE1EAE289728968EAD9FAD28976B
:107C000063E070E00F943CBC62967FAF6EAF62970A
:107C10003C0160FF05C0A2E0B0E0A81BB90B3D012C
:107C20002996BFAD2997BB2399F12896EEADFFADFC
:107C30002897EF2B69F162968EAD9FAD6297880F02
:107C4000991F62968EAC9FAC6297880D991D860D28
:107C5000971D880F991F8D53904F0F9405B7BC0146
:107C6000990F880B990B0F9487B12AE037ED43E207
:107C70005CE30F94D4AC2091490B30914A0B4091B6
:107C80004B0B50914C0B0F9484B71B012C0103C07C
:107C9000212C312C210120E030E040EA50E42093F7
:107CA000F10F3093F20F4093F30F5093F40F2091A4
:107CB000ED0F3091EE0F4091EF0F5091F00F60916A
:107CC000E90F7091EA0F8091EB0F9091EC0FA4E116
:107CD000B5E1BF93AF93812C912CE0EAAE2EE1E4A5
:107CE000BE2EF5EFCF2EFFE0DF2EE12CF12C00EAC7
:107CF00010E40F949D280F94EC6F2E96EEADFFAD1F
:107D00002E9785919591A591B4918093E90F9093C9
:107D1000EA0FA093EB0FB093EC0F2E96EEADFFADF4
:107D20002E97349685919591A591B4918093ED0FFE
:107D30009093EE0FA093EF0FB093F00F6DEE7FE0F6
:107D400089EE9FE00E94239AE090F10FF090F20FED
:107D50000091F30F1091F40F2091ED0F3091EE0F81
:107D60004091EF0F5091F00F6091E90F7091EA0F81
:107D70008091EB0F9091EC0FA4E1B5E1BF93AF932D
:107D8000812C912CB6E1AB2EB3E4BB2E0F949D2831
:107D90000F94EC6F0F900F900F900F902996FFADFE
:107DA0002997FF2379F028968EAC9FAC28978928D5
:107DB00049F020E030E040E85FE3C201B1010F94F8
:107DC00083B704C060E070E080E291EC0F949116FC
:107DD000811108C0E091AB0FF0E0EE0FFF1FEA5CED
:107DE000FC4E1FC0C090F10FD090F20FE090F30F47
:107DF000F090F40FA701960160E070E080EA90E453
:107E00000F9483B72DEC3CEC4CEC5DE30F9481B107
:107E100087FF0AC0E091AB0FF0E0EE0FFF1FEE5CB2
:107E2000FC4E659074908EC029969FAC299799203E
:107E3000B9F0A7019601C201B1010F9483B79F77F2
:107E400020E030E040E85FE30F94CFB9181644F427
:107E5000E091AB0FF0E0EE0FFF1FE25DFC4EE1CFD3
:107E6000C0904009D0904109E0904209F090430948
:107E7000809182088823B9F086EA9FE00F94F8B6D3
:107E8000882389F0C701B6010E944E8F20911A0BFA
:107E900030911B0B40911C0B50911D0B0F9472B82D
:107EA0009B01AC0103C020E030E0A90167E06296CD
:107EB000AEACBFAC62976A9D80016B9D100D112422
:107EC000060D171D000F111F000F111F085B144F27
:107ED0006091F10F7091F20F8091F30F9091F40F78
:107EE0000F9483B7D80111966D937D938D939C93D6
:107EF000149780911A0990911B09019790931B097F
:107F000080931A092896EEADFFAD289731962896F2
:107F1000FFAFEEAF289781E00F94EB402E962EAD89
:107F20003FAD2E97285F3F4F2E963FAF2EAF2E9737
:107F300028964EAD5FAD28974930510509F05CCECB
:107F4000612C712C80E090E0A0EAB0E48093F10F06
:107F50009093F20FA093F30FB093F40F2091ED0FD5
:107F60003091EE0F4091EF0F5091F00F6091E90FBB
:107F70007091EA0F8091EB0F9091EC0FE4E1F5E145
:107F8000FF93EF93812C912CE0EAAE2EE1E4BE2E1C
:107F9000F5EFCF2EFFE0DF2EE12CF12C00EA10E40C
:107FA0000F949D280F94EC6F0F900F9028968EAD34
:107FB0009FAD2897099721F060E0C3010C94044C11
:107FC0000E9405940F9498506091551A7091561A1A
:107FD000072E000C880B990B0F9487B190582091B5
:107FE0001A0B30911B0B40911C0B50911D0B0F94E1
:107FF00072B80F94D5A280EC9FE00F94F8B6682E6B
:108000008E010F5F1F4F712C502E412E60EC262EDB
:1080100062E1362E88E0E6EAF2E0A52DB42D01906B
:108020000D928A95E1F7D8018D918D010E943D99BD
:10803000882329F00F94EC9F6B017C012EC0B1E0E6
:108040006B1223C2872D90E0FC013197E730F105D8
:1080500030F48827EE58FF4F8F4F0D946BBC86E0AD
:108060009FE014C08DEB9FE011C085E09FE00EC043
:108070008EEB9FE00BC084E09FE008C08CEB9FE09C
:1080800005C083E09FE002C08FEB9FE00F94F8B63D
:10809000C82E880FDD08EE08FF08C114D104E104E2
:1080A000F10409F4F2C1C701B6010F9487B12FE6BC
:1080B00032E143E85AE30F94D4AC4B015C019F7763
:1080C00022EF32ED4DE45EE30F94CFB918160CF0B9
:1080D00033C0E7E7FFE484917F01882341F00E94E9
:1080E0007986EFEFEE1AFE0AF7018491F6CFEAE007
:1080F000F3E184917F01882341F00E947986FFEFAC
:10810000EF1AFF0AF7018491F6CF42E0C501B401EE
:108110000F94B103E1E0F3E184917F01882341F002
:108120000E947986FFEFEF1AFF0AF7018491F6CFDC
:108130008AE00E947986A9C1872D90E0FC013197E1
:10814000A5019401E730F10530F48827E758FF4F87
:108150008F4F0D946BBC6091490B70914A0B8091CD
:108160004B0B90914C0B0F9484B76093490B709319
:108170004A0B80934B0B90934C0BE2EFF2E184910E
:108180005F01882341F00E947986FFEFAF1ABF0A92
:10819000F5018491F6CFC701B6010F949603E8EE7E
:1081A000F2E184917F01882309F4C2CF0E9479868D
:1081B000FFEFEF1AFF0AF7018491F5CF60914D0BA5
:1081C00070914E0B80914F0B9091500B0F9484B790
:1081D00060934D0B70934E0B80934F0B9093500B0D
:1081E000E9EDF2E184915F01882341F00E947986F4
:1081F000FFEFAF1ABF0AF5018491F6CFC701B601B0
:108200000F949603EFECF2E184917F01882309F447
:108210008FCF0E947986FFEFEF1AFF0AF701849152
:10822000F5CF6091510B7091520B8091530B90914F
:10823000540B0F9484B76093510B7093520B80933F
:10824000530B9093540BF101849150ECA52E52E105
:10825000B52E882341F00E947986FFEFAF1ABF0A3E
:10826000F5018491F6CFC701B6010F949603E6EBB2
:10827000F2E184917F01882309F45ACF0E94798624
:10828000FFEFEF1AFF0AF7018491F5CF60916D0BB4
:1082900070916E0B80916F0B9091700B0F9484B75F
:1082A00060936D0B70936E0B80936F0B9093700BBC
:1082B000E7EAF2E184915F01882341F00E94798628
:1082C000FFEFAF1ABF0AF5018491F6CFC701B601DF
:1082D0000F949603EDE9F2E184917F01882309F47C
:1082E00027CF0E947986FFEFEF1AFF0AF7018491EA
:1082F000F5CF6091890B70918A0B80918B0B9091D7
:108300008C0B0F9484B76093890B70938A0B8093C6
:108310008B0B90938C0BEEE8F2E184915F01882344
:1083200041F00E947986FFEFAF1ABF0AF5018491F0
:10833000F6CFC701B6010F949603E4E8F2E1849109
:108340007F01882309F4F4CE0E947986FFEFEF1AAB
:10835000FF0AF7018491F5CF6091850B7091860B30
:108360008091870B9091880B0F9484B76093850B55
:108370007093860B8093870B9093880BE5E7F2E16F
:1083800084915F01882341F00E947986FFEFAF1A44
:10839000BF0AF5018491F6CFC701B6010F94960389
:1083A000EBE6F2E184917F01882309F4C1CE0E94BB
:1083B0007986FFEFEF1AFF0AF7018491F5CF6091FC
:1083C000810B7091820B8091830B9091840B0F94A1
:1083D00084B76093810B7093820B8093830B90938F
:1083E000840BECE5F2E184915F01882341F00E9467
:1083F0007986FFEFAF1ABF0AF5018491F6CFC70166
:10840000B6010F949603E2E5F2E184917F0188239F
:1084100009F48ECE0E947986FFEFEF1AFF0AF7016A
:108420008491F5CF6091650B7091660B8091670B1D
:108430009091680B0F9484B76093650B7093660BF3
:108440008093670B9093680BE5E4F2E184915F0100
:10845000882341F00E947986FFEFAF1ABF0AF50129
:108460008491F6CFC701B6010F949603EBE3F2E1D6
:1084700084917F01882309F45BCE0E947986FFEF07
:10848000EF1AFF0AF7018491F5CF7394F8E07F1299
:10849000C1CD0F94D34A81E08093480B0F941451BF
:1084A000E091141524E0E29FF0011124E75AFB4EFD
:1084B00020E030E04EE353E460817181828193815A
:1084C0000F94CFB9181694F480918208882371F024
:1084D00086EA9FE00F94F8B6882341F080919408D3
:1084E00090919508C29714F00C943E6881E090E05A
:1084F000909373028093720263963FAD63973093BB
:108500004D0F68964EAD5FAD689750934C0F4093FA
:108510004B0F6C968EAD9FAD6C9790931B0980931B
:108520001A0910926C1A1092240A82E00F94EB4000
:108530000C94A0678091480B882309F495C0E1E36F
:10854000F2E184918F01882339F00E9479860F5FD0
:108550001F4FF8018491F7CF67E070E080E090E072
:108560000F949603EFE2F2E184918F01882339F0B2
:108570000E9479860F5F1F4FF8018491F7CF67E063
:1085800070E080E090E00F949603ECE1F2E18491DA
:108590008F01882339F00E9479860F5F1F4FF80101
:1085A0008491F7CF65E070E080E090E00F9496034F
:1085B000EAE0F2E184918F01882339F00E94798604
:1085C0000F5F1F4FF8018491F7CF8AE00E947986F0
:1085D00000E010E037E0C32E32E1D32E45E0A42EB8
:1085E00042E1B42EE12CF12C480128EA820E911CC4
:1085F000F601849127E0622E22E1722E882341F059
:108600000E947986FFEF6F1A7F0AF3018491F6CFFB
:10861000F701E80DF91DE85BF44F618172818381F8
:10862000948145E00F94B103F4E0EF0EF11C2CE1CE
:10863000E216F104E9F6F501849195E0E92E92E164
:10864000F92E882341F00E947986FFEFEF1AFF0A86
:10865000F7018491F6CF0C5111090C33FFEF1F077E
:1086600009F0C0CF0C94A067E7EEF1E184918F018F
:10867000882311F40C94BD330E9479860F5F1F4F3D
:10868000F8018491F5CF86EE0E9452990C94A06770
:108690001092911A0C94A06785E40E943D99811173
:1086A00002C00F94EC6FB2E96B2EB3E07B2E19EE93
:1086B000A12E1FE0B12E02EC802E0AE0902ED12CCC
:1086C000D3018D913D010E943D998823B9F1B3E01A
:1086D000DB120CC00E942099F501608371838283B4
:1086E000938385EF9FE00F94427928C00E942099E0
:1086F000D4012D913D914D915C910F9484B7F5017A
:108700006083718382839383E090F10FF090F20F86
:108710000091F30F1091F40F2091ED0F3091EE0FB7
:108720004091EF0F5091F00F6091E90F7091EA0FB7
:108730008091EB0F9091EC0F0F94D94CD394F4E00F
:10874000AF0EB11C24E0820E911C34E0D312B8CFDE
:108750000C94A06781E08093480F0F94133C6093C2
:10876000210C7093220C8093230C9093240C609125
:10877000480F84EC9FE00F940AB70C94A06781E83F
:1087800094E09F938F930F9424BD80910F14909148
:1087900010148B5D9D4E9F938F930F9424BD8AE0A0
:1087A00090E00F9438BD0F900F900F900F900C94A5
:1087B000A0678DE40E943D99882311F40C944765CD
:1087C000E0915508F0915608319691919032E9F375
:1087D0009930D9F390539A30D0F082E994E09F9386
:1087E0008F930F9424BD80910F14909110148B5D82
:1087F0009D4E9F938F930F9424BD8AE090E00F9439
:1088000038BD0F900F900F900F900C94A0670E94AE
:1088100020990F94E3B89B01693C710511F40C9405
:1088200081530CF0E7C06135710511F40C944C4F85
:108830000CF063C06931710509F449C43CF5643139
:10884000710509F4C5C394F46131710509F4B4C329
:1088500034F46230710508F4F1C20C942E65623173
:10886000710511F40C947B4F0C942E6566317105E3
:1088700009F4FCC30CF4F6C36731710509F4FCC3B9
:108880006831710509F410C40C942E656E317105C0
:1088900009F416C58CF46B31710509F430C40CF47D
:1088A00020C46C31710509F4DFC46D31710511F418
:1088B0000C94A0670C942E656C32710509F451C7B5
:1088C00054F46F31710509F4F5C66032710509F48D
:1088D00058C60C942E656D32710509F451C76F327C
:1088E000710511F00C942E6584E090E09093730272
:1088F000809372020E94ABEF4AC76E36710511F485
:108900000C945F50B4F56C35710511F40C94CF4F95
:10891000A4F46335710511F40C94764F14F40C949F
:10892000724F6435710511F40C947B4F65357105F8
:1089300011F40C94B44F0C942E656A36710511F441
:108940000C94164F54F46836710509F43FC7693624
:10895000710509F46CC70C942E656B36710511F422
:108960000C94464F6D36710511F40C94364D0C94F1
:108970002E656737710511F40C94EB51DCF4613707
:10898000710511F40C9472504CF46037710511F0BC
:108990000C942E6563E080E095E036C76237710580
:1089A00011F40C9407516337710511F40C9498502D
:1089B0000C942E656C38710509F428C77CF468376F
:1089C000710511F40C94E7516937710511F00C949D
:1089D0002E6581E0809362020C94A0676E3B710566
:1089E00011F40C94DE4D683C710511F40C940D5398
:1089F0000C942E65663F41E0740711F40C947F5C83
:108A00000CF08CC0603F710511F40C94A0670CF061
:108A100045C06F3C710511F40C94A3545CF56C3C9B
:108A2000710511F40C94BB5384F46B3C710511F087
:108A30000C942E65F2E0EF2EFBE0FF2E02E913E02E
:108A4000A4E0DA2ED00E0C94AB536D3C710511F4FA
:108A50000C94DD536E3C710511F00C942E6572EC94
:108A6000E72E7AE0F72E02E913E0E3E0DE2ED00EE7
:108A70000C949354613D710511F40C94025514F457
:108A80000C94DA546C3D710511F40C9457556D3DFE
:108A9000710511F40C9468550C942E656033A1E0B7
:108AA0007A0711F40C948056D4F46D32E1E07E071D
:108AB00011F40C94C4553CF46C32714011F40C94D4
:108AC00092550C942E656E32714011F40C94185727
:108AD0002F32314011F40C942D570C942E656039CF
:108AE000A1E07A0711F40C94435B4CF46E5571408D
:108AF0006230710510F40C94A0670C942E65643FED
:108B0000E1E07E0711F40C94475B653F714011F082
:108B10000C942E650F9433040C94A0676E3843E0D8
:108B2000740711F40C9498630CF032C12A3562E09A
:108B3000360711F40C94406304F52D3F91E039079A
:108B400011F40C94E96064F4273F314011F00C9467
:108B50002E6509EF16E4F801849178010C94835C8A
:108B60002835E2E03E0711F40C94D36129353240F8
:108B700011F40C9432630C942E65233543E03407D2
:108B800011F40C9406610CF0F6C02D3B62E0360740
:108B900011F40C9412652E3B324011F00C942E65AA
:108BA00070901B0210921B0281E080934D0F82E0B7
:108BB00090E090934C0F80934B0FE091AB0FF0E05F
:108BC000EE0FFF1FE25DFE4E859194910F94933F4F
:108BD00020E030E044E352E46091F50F7091F60F2D
:108BE0008091F70F9091F80F0F9483B76093F50F72
:108BF0007093F60F8093F70F9093F80FE090F10FBA
:108C0000F090F20F0091F30F1091F40F2091ED0FFF
:108C10003091EE0F4091EF0F5091F00F6091E90FFE
:108C20007091EA0F8091EB0F9091EC0FE4E14E2EE2
:108C3000E5E15E2E5F924F92812C912CFCEAAF2EE3
:108C4000F2E4BF2EA5EFCA2EAFE0DA2E0F949D28D6
:108C50000F94EC6F20E030E040E751E46091F50FB5
:108C60007091F60F8091F70F9091F80F0F9483B7E2
:108C70006093F50F7093F60F8093F70F9093F80FB2
:108C8000E090F10FF090F20F0091F30F1091F40FBC
:108C90002091ED0F3091EE0F4091EF0F5091F00FBA
:108CA0006091E90F7091EA0F8091EB0F9091EC0FBA
:108CB0005F924F92812C912CB0E8AB2EB1E4BB2E89
:108CC0000F949D280F94EC6F20E030E040EA51E4CF
:108CD0006091F50F7091F60F8091F70F9091F80F5A
:108CE0000F9483B76093F50F7093F60F8093F70F8F
:108CF0009093F80FE090F10FF090F20F0091F30FC6
:108D00001091F40F2091ED0F3091EE0F4091EF0F85
:108D10005091F00F6091E90F7091EA0F8091EB0F85
:108D20009091EC0F5F924F920F949D280F94EC6FEF
:108D3000E091AB0FF0E0EE0FFF1FE65DFE4E859178
:108D400094910E945E99149A64E670E080E090E04D
:108D50000F94DB3B9FB7F89480910201846080936D
:108D600002019FBF0F900F900F900F900F900F90E8
:108D700010E00C9428652B3893E0390711F40C941B
:108D80004E632C38334011F40C94A0670C942E657C
:108D90006339B3E07B0711F40C942B64CCF4603995
:108DA000F3E07F0711F40C94CD6314F40C949B63EF
:108DB0006139734011F40C94FF632239334011F090
:108DC0000C942E65109283080E948DD90C94A06794
:108DD000263983E0380711F40C94E0646CF42439EC
:108DE000A3E03A0711F40C9431642539334011F4AF
:108DF0000C94AE640C942E65203AE3E03E0709F42F
:108E00002AC4273E334011F00C942E6510926B0952
:108E10001092830F80919A1A90919B1AA0919C1A9C
:108E2000B0919D1A8093570890935808A0935908C1
:108E3000B0935A080F948DAC0C94A067E09155083C
:108E4000F09156088F010E5F1F4F80E50E943D99FB
:108E5000882371F00E9420990F94E9B86B017C017E
:108E6000AA24A394672B682B692B31F4A12C04C08E
:108E7000A12CC12CD12C760183E50E943D99882339
:108E800091F00E94209920E030E04AE754E40F94EA
:108E9000D4AC0F94E9B86B017C01BB24B394672B6D
:108EA000682B692B09F4B12C6AE270E0C8010F94B9
:108EB000D2BC009711F0DC011C92F801CF01219186
:108EC0002032E1F3A11007C0B11005C0222319F030
:108ED0000F94A83F06C0E5EEF1E1859194910F94BF
:108EE000933F81E080935A1A1092591A0F94EC6FB5
:108EF0000F94133C6093961A7093971A8093981A64
:108F00009093991AC114D104E104F10419F10F945A
:108F1000133CC60ED71EE81EF91E84E090E0909325
:108F20007302809372020F94133C6C157D058E05BD
:108F30009F0510F00C9480680F946F3F81110C9482
:108F400080680F94526981E00F94C88780E00F9485
:108F5000EB40E9CF84E090E090937302809372023B
:108F60000F946F3F811109C00F94526981E00F94F3
:108F7000C88780E00F94EB40F3CF82E090E09093BD
:108F80007302809372028091270CE091AB0FF0E0A6
:108F9000EE0FFF1F882341F0EF51FE4E8591949113
:108FA0000F94933F0C94A067E05EF54E85919491E9
:108FB0000F94933F0C94A067EFEDF1E185919491AC
:108FC0000F94933F17981698159814980C94A067CF
:108FD000EDEDF1E105911491F8018491882329F0D8
:108FE0000E9479860F5F1F4FF7CF8AE00E94798633
:108FF00010923B0F10923A0F40E050E0BA018EE71A
:109000009CE00E944D798BE1EEE7FCE0DE011596D5
:1090100001900D928A95E1F780917C0C90917D0CE6
:109020009C838B8386E593E09A83898340E050E0BC
:10903000BE016F5F7F4F80E095E00F94E107CE01A6
:1090400001960E942787EBEDF1E105911491F8015B
:109050008491882311F40C94BD330E9479860F5FAC
:109060001F4FF5CF0F9469790C94A0671092270CCD
:109070001092280C0C94A067809155089091560886
:109080006AE270E004960F94D2BC009711F0DC0104
:109090001C92809155089091560841E061E0049639
:1090A0000F940B180C94A0678091280C882319F05A
:1090B00081E08093270C0F94133C6093631A7093A4
:1090C000641A8093651A9093661A0C94A067809135
:1090D000270C882311F40C94A0671092270C0C9491
:1090E000A0678091280C882311F40C94A06783E575
:1090F0000E943D9981110C948C680C94A06780911A
:10910000270C882309F49EC002E41CE0F801819139
:109110008F01882319F00E946675F8CFE8E4FCE01F
:1091200084918F01882339F00E9466750F5F1F4F6D
:10913000F8018491F7CFE6E4FCE005911491F80181
:109140008491882329F00E9466750F5F1F4FF7CF27
:109150006091350F7091360F8091370F9091380FD5
:109160004AE00F940F03E4E4FCE084918F0188232C
:1091700039F00E9466750F5F1F4FF8018491F7CF99
:1091800060912D0F70912E0F80912F0F9091300FC5
:109190004AE00F940F038AE00E9466750F94133C17
:1091A000F0E68F2EFAEE9F2EA12CB12CA501940192
:1091B0000F9448B769017A016091631A7091641A3B
:1091C0008091651A9091661AA50194010F9448B791
:1091D000C21AD30AC6016CE370E00F9428BC6983FD
:1091E000CE0101960F943E3F8C01D8018D918D01E7
:1091F000882319F00E946675F8CF8AE30E943A9B93
:10920000C6016CE370E00F9428BC8983CE010196FF
:109210000F943E3F8C01F80181918F01882319F052
:109220000E946675F8CFE2E4FCE084918F01882308
:1092300011F40C94A0670E9466750F5F1F4FF80130
:109240008491F5CFE6E9F3E084918F01882339F02A
:109250000E9466750F5F1F4FF8018491F7CF8AE077
:109260000E9466750C94A0678091550890915608ED
:109270006AE270E004960F94D2BC8C01892BA9F0AD
:1092800080910F14909110146EE470E08B5D9D4EF0
:109290000F94D2BC60E270E00F94D2BC0196909320
:1092A000560880935508D8011C92809155089091DA
:1092B000560841E060E004960F940B180C94A067E8
:1092C0008091280C882311F40C94A0670F94B34666
:1092D00080915508909156086AE270E004960F94C8
:1092E000D2BC8C01892BA9F080910F14909110149D
:1092F0006EE470E08B5D9D4E0F94D2BC60E270E036
:109300000F94D2BC01969093560880935508F801AB
:10931000108200915508109156085801F4E0AF0EE4
:10932000B11C8091280C882311F40C94A06780E86C
:109330009EE00E94CD821092270C1D8218861C820E
:109340001B8286E593E09A8389838AE79CE0909369
:109350009A0C8093990CD80114968C918F3209F055
:1093600082C06FE270E0C5010F94D2BC8C010F5F28
:109370001F4FFE0131964F010115110509F479C007
:109380006FE270E0C8010F94D2BC6C01009709F441
:1093900071C00817190708F06DC03C01601A710A06
:1093A000A301B801CE0180960F94FBBCE0E2F0E08F
:1093B000EC0FFD1FE60DF71D10828E01005E1F4FA2
:1093C0003801D3018D913D01882319F00E94667503
:1093D000F8CF8AE00E9466756091990C70919A0CA2
:1093E0006115710511F06C5F7F4F21E0AE01405EA9
:1093F0005F4FCE0105960E94D68281112CC0E3EA10
:10940000F3E084917F01882341F00E946675BFEFED
:10941000EB1AFB0AF7018491F6CFD8018D918D01EB
:10942000882319F00E946675F8CFE2E7FCE084918A
:109430008F01882339F00E9466750F5F1F4FF80176
:109440008491F7CF8AE00E946675CE0101960E9452
:1094500027870C94A06790929A0C8092990C8601B1
:109460000F5F1F4F89CF8BE99CE090939A0C8093FC
:10947000990C85016091990C70919A0C6115710598
:1094800011F06C5F7F4F18A21BA222E0A801CE0151
:1094900080960E94D6828823F1F0CE0180960F94A8
:1094A0004F078823C1F06CA57DA58EA59FA541E03F
:1094B0000E94D075882379F0E8A920E2E29FF001AC
:1094C0001124E75FFF4E309731F085EE80831BA2B9
:1094D0000E949075F82ECE0180960E945899FF2028
:1094E00021F1E4E6FCE084917F01882341F00E94B1
:1094F00066753FEFE31AF30AF7018491F6CFD801BE
:109500008D918D01882319F00E946675F8CF8AE04D
:109510000E9466751092350F1092360F1092370F19
:109520001092380F0F94491B26C0ECE4FCE08491A4
:109530007F01882341F00E946675BFEFEB1AFB0A9A
:10954000F7018491F6CFD8018D918D01882319F010
:109550000E946675F8CFEAE4FCE084918F018823CD
:1095600039F00E9466750F5F1F4FF8018491F7CFA5
:109570008AE00E946675CE0101960E9427870C94AE
:10958000A0678091270C81110F94EC6F0091550812
:10959000109156080C5F1F4F6AE270E0C8010F94EB
:1095A000D2BC7C0161E270E0C8010F94D2BC00978C
:1095B00019F08C010F5F1F4FE114F10411F0D70176
:1095C0001C9280E50E943D99F82E8091550890915B
:1095D00056080817190708F4F12C8091280C8823E5
:1095E00011F40C94A06741E04F2561E0C8010F948D
:1095F0000B1883E50E943D998823B9F080915508A6
:10960000909156088017910780F40F94EC9FAB015E
:10961000BC014093350F5093360F6093370F709312
:10962000380F80E89EE00E944D798091280C8823B5
:1096300019F081E08093270CF1100C94A0670F942F
:10964000133C6093631A7093641A8093651A909325
:10965000661A0C94A06780915508909156086AE2AA
:1096600070E005960F94D2BC8C01892BA9F08091F3
:109670000F14909110146EE470E08B5D9D4E0F946A
:10968000D2BC60E270E00F94D2BC01969093560871
:1096900080935508F80110828091550890915608E2
:1096A00021E02093260C41E060E005960F940B1812
:1096B0000C94A0670F94133C6093671A7093681A18
:1096C0008093691A90936A1A0091631A1091641A30
:1096D0002091651A3091661A601B710B820B930BF7
:1096E00028EE33E040E050E00F9448B7CA01B901DA
:1096F0002CE330E040E050E00F9448B77F936F9345
:109700003F932F938CEC91E19F938F938E010F5F8A
:109710001F4F1F930F930F9452B1E9EFF6E484911A
:109720000FB6F894DEBF0FBECDBF7F01882341F096
:109730000E9479863FEFE31AF30AF7018491F6CF8E
:109740007801D7018D917D01882319F00E947986D7
:10975000F8CF8AE00E947986C8010F94A83F0C9444
:10976000A0678FEF0E94529960E070E088EF9FE061
:109770000F9424B70F94035B0F94775A0C94A0674F
:109780008AE50E943D990E94DFC60C94A0670F9461
:10979000526981E00F94C8870F94C7020F946F3FFE
:1097A0008823A9F30F946F3F8111FCCF6AE070E02A
:1097B00080E090E00F94DB3B0F946F3F8111FCCF72
:1097C0000E94ABEF0F9429920C94A06788E690E07A
:1097D0000F946EA581110C94A06783E50E943D99BA
:1097E000882311F40C94A06700919E1A0E9420997E
:1097F00010E0000F111F0A56174F0F94E3B8F8013D
:10980000718360830C94A0670F94598783E50E944D
:109810003D99882311F40C94A0670E9420990F941D
:10982000E3B870939508609394080C94A06789E658
:1098300090E00F946EA581110C94A067E6ECF1E125
:1098400084918F01882339F00E9479860F5F1F4F22
:10985000F8018491F7CFE0919E1A24E0E29FF00195
:109860001124E75AFB4E608171818281938141E02E
:109870000F94B103E3ECF1E184918F01882339F077
:109880000E9479860F5F1F4FF8018491F7CFE09116
:109890009E1AF0E0EE0FFF1FEA56F74F60817181CC
:1098A000072E000C880B990B0F9487B141E00F94A1
:1098B000B103EFEBF1E184918F01882339F00E942D
:1098C00079860F5F1F4FF8018491F7CF60917E0872
:1098D00070917F08809180089091810841E00F94F9
:1098E000B103ECEBF1E184918F01882339F00E9400
:1098F00079860F5F1F4FF8018491F7CF609194082C
:1099000070919508072E000C880B990B0F9487B166
:1099100041E00F94B103E9EBF1E184918F018823D9
:1099200039F00E9479860F5F1F4FF8018491F7CFBD
:1099300060E070E0CB010F949603E7EBF1E18491D6
:109940008F01882339F00E9479860F5F1F4FF8013D
:109950008491F7CF6091591470915A1480915B14DF
:1099600090915C1441E00F94B103E4EBF1E1849138
:109970008F01882339F00E9479860F5F1F4FF8010D
:109980008491F7CF6091960870919708072E000C8C
:10999000880B990B0F9487B141E00F94B103E0EB72
:1099A000F1E184918F01882339F00E9479860F5F5D
:1099B0001F4FF8018491F7CFE0919E1AF0E0E7592C
:1099C000F64F608170E080E090E00F949603EBEA40
:1099D000F1E184918F01882339F00E9479860F5F2D
:1099E0001F4FF8018491F7CF6091680970E080E023
:1099F00090E00F949603E7EAF1E184918F018823C8
:109A000039F00E9479860F5F1F4FF8018491F7CFDC
:109A100060914009709141098091420990914309F8
:109A200041E00F94B103E3EAF1E184918F018823CF
:109A300039F00E9479860F5F1F4FF8018491F7CFAC
:109A400060913C0970913D0980913E0990913F09D8
:109A500041E00F94B1038AE00E94798681E090E0B2
:109A600090937302809372020C946C738DE690E075
:109A70000F946EA581110C94A067E091AB0FF0E0FC
:109A8000EE0FFF1FE855FC4B859194910F94933F87
:109A900081E090E09093E5098093E4098091480F7C
:109AA000882321F081E090E00E9416FF83E50E9468
:109AB0003D99882391F000919E1A0E94209910E010
:109AC000000F111F0A56174F0F94E3B8D8016D937A
:109AD0007C9381E08093090215C082E50E943D9944
:109AE000882381F000919E1A0E94209910E0000FB7
:109AF000111F0A56174F0F94E3B8F8017183608362
:109B0000109209020F94133C6B017C01E0919E1AA4
:109B10000E2F10E0F801EE0FFF1FEA56F74F60819D
:109B20007181072E000C880B990B0F9487B1F801F7
:109B3000EE0FFF1FEE0FFF1FE75AFB4E11E02081D3
:109B40003181428153810F94CFB918160CF010E087
:109B50001093530881E090E0909373028093720217
:109B600010926D1A46015701CC24CA94DC2C760160
:109B7000F4E72F2EFCE03F2EA8EE4A2EA3E05A2E4B
:109B8000612C712C80916D1A81110C949D68FFEFEE
:109B9000CF16DF06EF06FF0611F40C94C568F7FE3A
:109BA00002C00C949D680F94133C6C197D09683BAE
:109BB0007B4010F40C94C5680C949D68E091AB0F49
:109BC000F0E0EE0FFF1FE056FC4B859194910F944F
:109BD000933F83E090E09093E5098093E4098091BE
:109BE000480F882321F081E090E00E9416FF83E572
:109BF0000E943D99882361F00E9420990F94E3B858
:109C0000709395086093940881E0809309020FC0D7
:109C100082E50E943D99882351F00E9420990F947B
:109C2000E3B87093950860939408109209020F941A
:109C3000133C4B015C0110926D1A60919408709175
:109C40009508072E000C880B990B0F9487B111E033
:109C500020917E0830917F084091800850918108C2
:109C60000F94CFB918160CF010E01093530881E050
:109C700090E0909373028093720200EA11E1ACE9E4
:109C8000EA2EA1E1FA2EB8E9CB2EB1E1DB2E8091CC
:109C900053086091940870919508882309F48CC04A
:109CA00080916D1A811188C0072E000C880B990BCA
:109CB0000F9487B120917E0830917F0840918008F1
:109CC000509181080F94CFB918160CF08CC00F94E6
:109CD000133CDC01CB0188199909AA09BB09893E0B
:109CE0009340A105B10508F45EC08091480F811131
:109CF00056C0E091141544E0E49FF0011124E75AA6
:109D0000FB4E4080518062807380F8018491F0EABC
:109D1000AF2EF1E1BF2E882341F00E947986FFEF3C
:109D2000AF1ABF0AF5018491F6CF42E0C301B20138
:109D30000F94B103F7018491ECE9AE2EE1E1BE2E60
:109D4000882341F00E947986FFEFAF1ABF0AF50120
:109D50008491F6CF6091141570E080E090E00F944C
:109D60009603F601849178E9A72E71E1B72E882336
:109D700041F00E947986FFEFAF1ABF0AF501849186
:109D8000F6CF60917E0870917F0880918008909155
:109D9000810841E00F94B1038AE00E9479860F9414
:109DA000133C4B015C010F94526980E00F94C8870B
:109DB00080E00F94EB406BCF072E000C880B990BC3
:109DC0000F9487B120917E0830917F0840918008E0
:109DD000509181080F9481B187FF05C080910902DD
:109DE000882309F474CFE091AB0FF0E0EE0FFF1F72
:109DF000E456FC4B859194910F94933F82E090E060
:109E0000909373028093720284E090E09093E5094E
:109E10008093E4090F94133C6093961A7093971AF9
:109E20008093981A9093991A0C94A06783E50E94E6
:109E30003D99882319F10E94209920E030E0A90182
:109E40000F9481B187FD0FC00E94209920E030E07F
:109E50004FE753E40F94CFB9181644F00E942099AD
:109E60000F94E3B805C060E070E002C06FEF70E0EF
:109E70007093A90F6093A80F0C94A0678FEF90E0E8
:109E80009093A90F8093A80F0C94A0671092A90F2C
:109E90001092A80F0C94A0670E94CCDB0F94EC6F7B
:109EA000149A0F94C26F1092A90F1092A80F68EE27
:109EB00073E080E090E00F94DB3B10920802E6E94B
:109EC000F1E14591549122E931E164E971E183EADC
:109ED00094E00F9431A30F94933F80E00F94EB40F4
:109EE0000C94A06710921F090C94A06781E08093E6
:109EF0001F090C94A06783E50E943D99882399F07F
:109F00000E94209920E030E04AE754E40F94D4AC5A
:109F10000F94E9B86093A2027093A3028093A40205
:109F20009093A5021DC088E50E943D9981110C9473
:109F3000E26989E50E943D9981110C94E2698AE504
:109F40000E943D9981110C94E26985E40E943D993B
:109F500081110C94E2690F94EC6F149A0F94C26F04
:109F6000109252080C94A06783E50E943D998823C3
:109F700011F40C94A0670E94209920E030E04AE799
:109F800054E40F94D4AC0F94E9B86093921A709390
:109F9000931A8093941A9093951A0C94A06742E9AF
:109FA000842E43E0942E02E11BE052E0A52E5BE0FC
:109FB000B52E28E934E128963FAF2EAF2897312CF3
:109FC000D4018D914D010E943D99882309F462C00E
:109FD000B3E03B1258C00E9420992B013C0120E0C5
:109FE00030E040EA51E40F9481B187FF45C0A301FE
:109FF0009201F80160817181828193810F9472B81E
:10A000006B017C019B01AC016091DA0A7091DB0A63
:10A010008091DC0A9091DD0A0F94D4AC6093DA0A47
:10A020007093DB0A8093DC0A9093DD0AA701960106
:10A03000D5016D917D918D919C910F94D4ACF501DA
:10A0400060837183828393832896AEADBFAD2897DA
:10A050006D917D918D919C910F9485B1A701960191
:10A060000F94D4AC0F94E9B82896EEADFFAD2897C5
:10A070006083718382839383D8014D925D926D9248
:10A080007C92139707C00E942099F8016083718326
:10A090008283938333940C5F1F4FF4E0AF0EB11CA7
:10A0A00028962EAD3FAD28972C5F3F4F28963FAFA7
:10A0B0002EAF289734E0331283CF0C94A0678EE440
:10A0C0000E943D99882311F40C94A0670F94EC9F93
:10A0D00060935708709358088093590890935A08D2
:10A0E0000C94A06783E50E943D99882331F00E947B
:10A0F0001399809320020C94A067E9EFF6E4849111
:10A100008F01882339F00E9479860F5F1F4FF80175
:10A110008491F7CF4091200250E060E070E08BE83E
:10A1200091E10F94D09F8AE00E9479860C94A067F9
:10A1300086E50E943D99882379F0E2E5FEE5849169
:10A140008F01882311F40C94BD330E9479860F5F30
:10A150001F4FF8018491F5CF85E50E943D99382E77
:10A16000882309F445C000915508109156080F5FE7
:10A170001F4F1093560800935508780128013201AB
:10A18000D2018D912D0190ED980F9A30C0F38E324F
:10A1900011F00C94A0676D014601F60181916F01E9
:10A1A00090ED980F9A30C0F38E3211F00C94A067A6
:10A1B0009F015901D9019C912F5F3F4F80ED890F7D
:10A1C0008A30B8F3892FCB57DF4F9883C558D040DA
:10A1D0000F94693CCB57DF4F9881C558D04081110F
:10A1E0000C94016A9D3211F00C94A0670C94016AE2
:10A1F000E9E8F1E105911491F8018491882311F4C3
:10A200000C94A0670E9479860F5F1F4FF5CFE6E898
:10A21000F1E184918F01882339F00E9479860F5FE4
:10A220001F4FF8018491F7CF6091E90F7091EA0F09
:10A230008091EB0F9091EC0F42E00F94B103E2E8B4
:10A24000F1E184918F01882339F00E9479860F5FB4
:10A250001F4FF8018491F7CF6091ED0F7091EE0FD1
:10A260008091EF0F9091F00F42E00F94B103EEE771
:10A27000F1E184918F01882339F00E9479860F5F84
:10A280001F4FF8018491F7CF6091F10F7091F20F99
:10A290008091F30F9091F40F42E00F94B103EAE73D
:10A2A000F1E184918F01882339F00E9479860F5F54
:10A2B0001F4FF8018491F7CF6091F50F7091F60F61
:10A2C0008091F70F9091F80F42E00F94B103E8E707
:10A2D000F1E105911491F8018491882329F00E94FD
:10A2E00079860F5F1F4FF7CF0F94CB6F0F9487B115
:10A2F0002091120B3091130B4091140B5091150BC0
:10A300000F9472B842E00F94B103E4E7F1E1849155
:10A310008F01882339F00E9479860F5F1F4FF80163
:10A320008491F7CF81E00F94CB6F0F9487B1209188
:10A33000160B3091170B4091180B5091190B0F947D
:10A3400072B842E00F94B103E0E7F1E184918F012C
:10A35000882339F00E9479860F5F1F4FF80184919E
:10A36000F7CF82E00F94CB6F0F9487B120911A0B37
:10A3700030911B0B40911C0B50911D0B0F9472B828
:10A3800042E00F94B103ECE6F1E184918F01882360
:10A3900039F00E9479860F5F1F4FF8018491F7CF43
:10A3A00083E00F94CB6F0F9487B120911E0B3091F7
:10A3B0001F0B4091200B5091210B0F9472B842E07B
:10A3C0000F94B1038AE00E9479860C94A0671092E2
:10A3D00062020C94A067EAE6F1E105911491F8019C
:10A3E0008491882329F00E9479860F5F1F4FF7CF51
:10A3F0008AE00E947986E8E6F1E105911491F8017E
:10A400008491882329F00E9479860F5F1F4FF7CF30
:10A410001E9B15C0E6E6F1E105911491F8018491C7
:10A42000882329F00E9479860F5F1F4FF7CF8AE0BB
:10A430000E947986E2E6F1E1059114910DC0E4E60F
:10A44000F1E105911491F8018491882381F30E9430
:10A4500079860F5F1F4FF7CFF8018491882329F089
:10A460000E9479860F5F1F4FF7CF8091060182FF10
:10A4700015C0E6E6F1E105911491F8018491882375
:10A4800029F00E9479860F5F1F4FF7CF8AE00E9464
:10A490007986E0E6F1E1059114910DC0E4E6F1E181
:10A4A00005911491F8018491882381F30E947986A3
:10A4B0000F5F1F4FF7CFF8018491882329F00E9486
:10A4C00079860F5F1F4FF7CF1D9B15C0E6E6F1E1C0
:10A4D00005911491F8018491882329F00E947986CE
:10A4E0000F5F1F4FF7CF8AE00E947986EEE5F1E11A
:10A4F000059114910DC0E4E6F1E105911491F80184
:10A500008491882381F30E9479860F5F1F4FF7CFD4
:10A51000F8018491882329F00E9479860F5F1F4FEC
:10A52000F7CF8091060187FF15C0E6E6F1E10591BE
:10A530001491F8018491882329F00E9479860F5F95
:10A540001F4FF7CF8AE00E947986ECE5F1E1059193
:10A5500014910DC0E4E6F1E105911491F8018491A4
:10A56000882381F30E9479860F5F1F4FF7CFF80190
:10A570008491882329F00E9479860F5F1F4FF7CFBF
:10A580001C9B15C0E6E6F1E105911491F801849158
:10A59000882329F00E9479860F5F1F4FF7CF8AE04A
:10A5A0000E947986EAE5F1E1059114910DC0E4E697
:10A5B000F1E105911491F8018491882381F30E94BF
:10A5C00079860F5F1F4FF7CFF8018491882329F018
:10A5D0000E9479860F5F1F4FF7CF01990FC0E6E603
:10A5E000F1E105911491F8018491882311F40C9400
:10A5F000BD330E9479860F5F1F4FF5CFE4E6F1E18E
:10A6000005911491F8018491882311F40C94BD33C1
:10A610000E9479860F5F1F4FF5CF809114158093AC
:10A620009E1A84E50E943D99882319F10E94209981
:10A630000F94E9B860939E1A6623D9F0E9EFF6E427
:10A6400084918F01882339F00E9479860F5F1F4F14
:10A65000F8018491F7CFE8E5F1E105911491D80173
:10A660008D918D01882311F40C94A0670E94798646
:10A67000F6CF84E40E943D99882311F40C94A067DE
:10A680000E94209920E030E0A9010F9481B181114E
:10A6900003C01092B40A31C000919E1A10E00E94CB
:10A6A0002099000F111F000F111FF801E65CFD4FEC
:10A6B0006083718382839383C0903A02D0903B027F
:10A6C000E0903C02F0903D0220E030E0A901C7019B
:10A6D000B6010F9481B1811105C0C12CD12C90E439
:10A6E000E92EFE2CC0923A02D0923B02E0923C024C
:10A6F000F0923D0281E08093B40A0F9448860C9456
:10A70000A067B2EFEB2EBAE0FB2E02E913E084E083
:10A71000D82ED00EF80181918F010E943D99882397
:10A7200051F00E9420990F94E9B8D7016D937D9361
:10A730008D939C931397B4E0EB0EF11CD012EACFEB
:10A740000F94FA780C94A067B4E0EB0EF11CD016CD
:10A7500011F40C94A067F80181918F010E943D993A
:10A76000882391F30E942099D7016D937D938D9357
:10A770009C931397E9CF83E50E943D99882351F07C
:10A780000E9420996093EE0A7093EF0A8093F00A7A
:10A790009093F10A84E50E943D99882311F40C946A
:10A7A000A0670E9420996093EA0A7093EB0A809355
:10A7B000EC0A9093ED0A0C94A06783E50E943D9902
:10A7C000882351F00E9420996093E60A7093E70A6B
:10A7D0008093E80A9093E90A84E50E943D998823D2
:10A7E00051F00E9420996093E20A7093E30A8093EB
:10A7F000E40A9093E50A82E40E943D99882361F07F
:10A800000E9420990F94E9B86093DE0A7093DF0AE2
:10A810008093E00A9093E10A88E50E943D9988239D
:10A8200091F00E9420996093D20A7093D30A80938A
:10A83000D40A9093D50A6093CE0A7093CF0A80937E
:10A84000D00A9093D10A89E50E943D99882351F05E
:10A850000E9420996093D20A7093D30A8093D40AFD
:10A860009093D50A8AE50E943D99882351F00E9471
:10A8700020996093D60A7093D70A8093D80A909350
:10A88000D90A85E40E943D99882351F00E942099BD
:10A890006093DA0A7093DB0A8093DC0A9093DD0AF6
:10A8A00020E030E040E251E46091CE0A7091CF0A9E
:10A8B0008091D00A9091D10A0F94CFB9181664F400
:10A8C00080E090E0A0E2B1E48093CE0A9093CF0ABA
:10A8D000A093D00AB093D10A20E030E040E251E4E6
:10A8E0006091D20A7091D30A8091D40A9091D50ACE
:10A8F0000F94CFB9181614F00C94A06780E090E084
:10A90000A0E2B1E48093D20A9093D30AA093D40A30
:10A91000B093D50A0C94A067B4E0EB0EF11CD016EE
:10A9200011F40C94A067F80181918F010E943D9968
:10A93000882391F30E942099D7016D937D938D9385
:10A940009C931397E9CF83E50E943D99882351F0AA
:10A950000E942099609346027093470280934802B8
:10A960009093490286E40E943D99882381F00E94D9
:10A97000209920E030E040E752E40F9472B86093F1
:10A9800042027093430280934402909345028AE509
:10A990000E943D99882311F40C94A0670E9420998D
:10A9A0006093B90A7093BA0A8093BB0A9093BC0A69
:10A9B0000C94A06783E50E943D99882351F00E9482
:10A9C00020996093B50A7093B60A8093B70A909362
:10A9D000B80A86E40E943D99882311F40C94A0677C
:10A9E0000E94209920E030E040E752E40F9472B8D2
:10A9F00060933E0270933F02809340029093410225
:10AA00000C94A06783E50E943D99882311F40C946F
:10AA1000A0670E9420990F94E3B86115710551F069
:10AA20006130710569F481E08093BD0A10920215CE
:10AA30000C94A0671092BD0A109202150C94A067A6
:10AA4000E9EFF6E484918F01882339F00E9479863A
:10AA50000F5F1F4FF8018491F7CFE6E5F1E1059113
:10AA60001491F8018491882329F00E9479860F5F60
:10AA70001F4FF7CF00910F14109110140B5D1D4E56
:10AA8000D8018D918D01882319F00E947986F8CF25
:10AA9000E1E5F1E184918F01882311F40C94BD3339
:10AAA0000E9479860F5F1F4FF8018491F5CF83E5EF
:10AAB0000E943D99882311F40C94A0670E9420996C
:10AAC0000F94E3B870936802609367020C94A067D8
:10AAD00083E50E943D99882311F40C94A0670E949D
:10AAE00020990F94E3B86B017C0184E50E943D99A5
:10AAF000882391F08DED90E00F946EA581110C9458
:10AB0000A067E0919E1AF0E0EE0FFF1FEA5FFD4F95
:10AB1000D182C0820C94A067D0926602C092650276
:10AB20000C94A06783E50E943D99882331F00E9430
:10AB300020990F94E3B88B0102C00EE610E080E587
:10AB40000E943D99882329F00E9420990F94E3B830
:10AB500002C068EE73E06B01770FEE08FF08101675
:10AB6000110664F4C8010F94CF43C701B6010F94D6
:10AB7000DB3B84E50F942B3A0C94A067C701B60128
:10AB80000F94DB3B0C94A06780E50E943D998823DD
:10AB900051F00E94209960935E0270935F0280934F
:10ABA00060029093610289E40E943D99882381F0BC
:10ABB0000E9420992CEA35EC47E25EE30F94D4AC76
:10ABC00060935A0270935B0280935C0290935D02E3
:10ABD00084E40E943D99882381F00E9420992CEA08
:10ABE00035EC47E25EE30F9472B8609356027093BF
:10ABF0005702809358029093590283E40E943D9932
:10AC0000882351F00E9420996093020270930302FE
:10AC100080930402909305020F94AE6DE3EDFAE188
:10AC200005911491F8018491882329F00E94798676
:10AC30000F5F1F4FF7CF00EB14E0D8018D918D010E
:10AC4000882319F00E947986F8CF60915E02709196
:10AC50005F02809160029091610242E00F94B10323
:10AC600004EB14E0F80181918F01882319F00E9410
:10AC70007986F8CF2CEA35EC47E25EE360915A0220
:10AC800070915B0280915C0290915D020F9472B8AA
:10AC900042E00F94B10308EB14E0D8018D918D01CF
:10ACA000882319F00E947986F8CF2CEA35EC47E228
:10ACB0005EE3609156027091570280915802909124
:10ACC00059020F94D4AC42E00F94B1030CEB14E0A2
:10ACD000F80181918F01882319F00E947986F8CFBD
:10ACE000609102027091030280910402909105022A
:10ACF00042E00F94B1038AE00E9479860C94A06729
:10AD000080E50E943D99882351F00E94209960932C
:10AD1000520270935302809354029093550289E437
:10AD20000E943D99882381F00E9420992CEA35ECFD
:10AD300047E25EE30F94D4AC60934E0270934F02EF
:10AD4000809350029093510284E40E943D9988239D
:10AD500081F00E9420992CEA35EC47E25EE30F94E3
:10AD600072B860934A0270934B0280934C029093A6
:10AD70004D020F94AE6DE3EDFAE105911491F801E7
:10AD80008491882329F00E9479860F5F1F4FF7CFA7
:10AD900000EB14E0D8018D918D01882319F00E94F9
:10ADA0007986F8CF609152027091530280915402DB
:10ADB0009091550242E00F94B10304EB14E0F801C6
:10ADC00081918F01882319F00E947986F8CF2CEAAF
:10ADD00035EC47E25EE360914E0270914F02809144
:10ADE0005002909151020F9472B842E00F94B10357
:10ADF00008EB14E0D8018D918D01882319F00E9491
:10AE00007986F8CF2CEA35EC47E25EE360914A029E
:10AE100070914B0280914C0290914D020F94D4ACF2
:10AE200042E00F94B1038AE00E9479860C94A067F7
:10AE300083E50E943D99882319F00E94209903C060
:10AE400060E070E0CB016093690270936A028093C6
:10AE50006B0290936C020C94A06785E40E943D996C
:10AE6000882359F00E9420990F94E3B82E967FAF63
:10AE70006EAF2E9777FF05C013C02E961FAE1EAE85
:10AE80002E9767961FAE67976B961FAE6B9726E15E
:10AE90006D962FAF6D9733E4A3963FAFA3970EC087
:10AEA00067961FAE67976B961FAE6B974CE86D96D3
:10AEB0004FAF6D9752E4A3965FAFA39783E50E94CF
:10AEC0003D99882371F00E94209967966FAF67972C
:10AED0006B967FAF6B976D968FAF6D97A3969FAF75
:10AEE000A39783E40E943D99882349F00E9420990A
:10AEF0000F94E3B8E4967FAF6EAFE49706C085E0A9
:10AF000090E0E4969FAF8EAFE497E4968EAC9FAC52
:10AF1000E4979092E1098092E00910921909109249
:10AF2000E3091092E2090F94133C66966CAF7DAF73
:10AF30008EAF9FAF66972E96AEACBFAC2E97B7FC88
:10AF400005C02AE0E9962FAFE99704C03DE2E996F3
:10AF50003FAFE9970F94133CC358DF4F6883798361
:10AF60008A839B83CD57D0402E968EAC9FAC2E9774
:10AF7000181419041CF000EC14E016C003ED14E0E2
:10AF8000D8018D918D01882319F00E94B8DBF8CF8C
:10AF90008AE00E94B8DB81E0809319091092E309EE
:10AFA0001092E2090C94A067F80181918F01882327
:10AFB00019F00E94B8DBF8CF8AE00E94B8DB0E944B
:10AFC000CCDB2E968EAC9FAC2E978FE7892809F4A8
:10AFD0004FC08093680966968CAC9DACAEACBFAC9C
:10AFE0006697AB968CAE9DAEAEAEBFAEAB97ED9610
:10AFF0008CAE9DAEAEAEBFAEED9761961FAE6197C3
:10B000006F961FAE6F9720E4AC962FAFAC973CE1E4
:10B01000AD963FAFAD9746E4AE964FAFAE97AF96C5
:10B020001FAEAF97E0961FAEE097E1961FAEE19797
:10B03000E2961FAEE2974FE7442E512C612C712C03
:10B040005FE7C52ED12CE12CF12CE8961CAE1DAE8D
:10B050001EAE1FAEE89751E0A4965FAFA497279667
:10B060001FAE279729961FAE2997212C312C06C099
:10B0700080936909B0CF80E00F94EB40A895809150
:10B080006A09882309F48FC10F9458682E968EACF4
:10B090009FAC2E97892879F090907E0827969FAED6
:10B0A0002797A0907F082996AFAE29972090800817
:10B0B000309081080EC0B09059142796BFAE2797E4
:10B0C00080905A1429968FAE299720905B14309067
:10B0D0005C1427962FAD279729963FAD2997A1019C
:10B0E000AF966FADAF97E0967FADE097E1968FADED
:10B0F000E197E2969FADE2970F94CFB9181694F0BE
:10B1000027969FAC2797AF969FAEAF972996AFAC87
:10B110002997E096AFAEE097E1962FAEE197E296E1
:10B120003FAEE29727962FAD279729963FAD2997F7
:10B13000A1016F966FAD6F97AC967FADAC97AD9652
:10B140008FADAD97AE969FADAE970F9481B187FD51
:10B1500012C02796BFAC27976F96BFAE6F97299600
:10B160008FAC2997AC968FAEAC97AD962FAEAD97BE
:10B17000AE963FAEAE970F94133CDC01CB01C358A3
:10B18000DF4F88809980AA80BB80CD57D040881936
:10B190009909AA09BB09853C9940A105B10560F050
:10B1A0000F9430690F94133CC358DF4F6883798341
:10B1B0008A839B83CD57D040A4968FACA4978820D8
:10B1C00009F473C067962FAD67976B963FAD6B9789
:10B1D0006D964FAD6D97A3965FADA39727966FAD14
:10B1E000279729967FAD2997C1010F94CFB91816DB
:10B1F0000CF0D9C00F94133CDC01CB0166968CACEB
:10B200009DACAEACBFAC669788199909AA09BB0979
:10B2100089389341A105B10508F4C5C0D701C6011D
:10B2200084199509A609B7092E968EAC9FAC2E9766
:10B23000B595A79597958795892819F08093680902
:10B2400002C0809369090F94133CAB966CAF7DAF3D
:10B250008EAF9FAFAB974B015C0166962CAD3DADB9
:10B260004EAD5FAD6697821A930AA40AB50AE896B6
:10B270008CAE9DAEAEAEBFAEE89767968FAC6797CB
:10B28000AF968FAEAF976B969FAC6B97E0969FAEE5
:10B29000E0976D96AFAC6D97E196AFAEE197A39650
:10B2A000BFACA397E296BFAEE29767962FAD6797C4
:10B2B0006B963FAD6B976D964FAD6D97A3965FAD57
:10B2C000A39727966FAD279729967FAD2997C10140
:10B2D0000F9481B187FD02C00C941B6D0F94133C39
:10B2E000DC01CB01AB968CAC9DACAEACBFACAB97EC
:10B2F00088199909AA09BB0989389341A105B105A3
:10B3000010F40C941B6D0F94133C66966CAF7DAFDC
:10B310008EAF9FAF6697DC01CB0188199909AA0906
:10B32000BB092091E2093091E3091216130614F4C7
:10B330000C943C6BD701C601840D951DA61DB71D4D
:10B340002E968EAC9FAC2E97B595A7959795879521
:10B35000892811F40C94176D809368098091E20993
:10B360009091E30901969093E3098093E20967962F
:10B370009FAC67976F969FAE6F976B96AFAC6B97CE
:10B38000AC96AFAEAC976D96BFAC6D97AD96BFAEB9
:10B39000AD97A3968FACA397AE968FAEAE9721E0F4
:10B3A000A4962FAFA49720E030E040EA51E46796DE
:10B3B0006FAD67976B967FAD6B976D968FAD6D9701
:10B3C000A3969FADA3970F9484B79B01AC012796DA
:10B3D0006FAD279729967FAD2997C1010F94CFB9FB
:10B3E000181674F4E1E1FDE084918F01882309F4DB
:10B3F000CFCD0E94B8DB0F5F1F4FF8018491F6CFCD
:10B400000F94133CDC01CB01ED968CAC9DACAEAC43
:10B41000BFACED9788199909AA09BB09813D9740EE
:10B42000A105B10508F4D3C02E968EAC9FAC2E9723
:10B43000892889F00091680910E0EBE0FDE0849133
:10B440005F018823C9F00E94B8DB2FEFA21AB20A6D
:10B45000F5018491F6CF0091690910E0E5E0FDE087
:10B4600084915F01882341F00E94B8DBFFEFAF1A9F
:10B47000BF0AF5018491F6CF42E027966FAD27977A
:10B4800029967FAD2997C1010F94B103E1E0FDE05A
:10B4900084915F01882341F00E94B8DBFFEFAF1A6F
:10B4A000BF0AF5018491F6CFB801110F880B990BF3
:10B4B0000F9496038AE00E94B8DB61968FAC619787
:10B4C000882009F45EC0E9969FACE997891418F4C6
:10B4D000282D2F5F71C061968FAC6197E9969FAC64
:10B4E000E99789106CC0282D2F5F61962FAF619767
:10B4F000CF57DF4F2881C158D040CE57DF4F38811A
:10B50000C258D040CD57DF4F4881C358D040CC57A8
:10B51000DF4F5881C458D04027966FAD27972996A2
:10B520007FAD2997C1010F9483B74B015C0120E0E7
:10B5300030E0A9010F94CFB918165CF420E030E098
:10B5400040EA50E4C501B4010F9481B187FF37C0D0
:10B550000AC020E030E040EA50ECC501B4010F948D
:10B56000CFB9181664F52E966FAD2E97661F662715
:10B57000661F80E00E9445DE81E0809319090C94EB
:10B58000A06727968FAC2797CF57DF4F8882C15887
:10B59000D04029969FAC2997CE57DF4F9882C2584A
:10B5A000D040CD57DF4F2882C358D040CC57DF4F13
:10B5B0003882C458D04021E061962FAF61970F9434
:10B5C000133CED966CAF7DAF8EAF9FAFED970F94B0
:10B5D000133CC757DF4F688379838A839B83C9589D
:10B5E000D0400F94133CAB960CAD1DAD2EAD3FADCE
:10B5F000AB9766968CAC9DACAEACBFAC6697080DB5
:10B60000191D2A1D3B1DC757DF4F88809980AA80CE
:10B61000BB80C958D040801A910AA20AB30A860E8C
:10B62000971EA81EB91E21E882162FE4920622E179
:10B63000A206B10470F0E4EEFCE084918F0188234F
:10B6400009F4A6CC0E94B8DB0F5F1F4FF80184916C
:10B65000F6CF8091E2099091E309E4968EAC9FAC1D
:10B66000E497881699060CF006CDE8E8FCE0849192
:10B670008F01882309F48CCC0E94B8DB0F5F1F4F29
:10B68000F8018491F6CF0F94EC6F0C94A06780E3DF
:10B6900090E3A0E3B0E088A399A3AAA3BBA304E12D
:10B6A00010E026961FAF0EAF269744E0BE01605E05
:10B6B0007F4FCE018C5B9F4F0F94F79F40E162E17B
:10B6C0007BE0CE018C5B9F4F0F94F79F40E162E0DF
:10B6D0007BE0CE018C5B9F4F0F94F79F40E162EFC0
:10B6E0007AE0CE018C5B9F4F0F94F79F44E06EEEA3
:10B6F0007AE0CE018C5B9F4F0F94F79F44E06AEE97
:10B700007AE0CE018C5B9F4F0F94F79F44E066EE8A
:10B710007AE0CE018C5B9F4F0F94F79F44E062EE7E
:10B720007AE0CE018C5B9F4F0F94F79F44E06EED63
:10B730007AE0CE018C5B9F4F0F94F79F44E06EEC54
:10B740007AE0CE018C5B9F4F0F94F79F44E062ED4F
:10B750007AE0CE018C5B9F4F0F94F79F44E066ED3B
:10B760007AE0CE018C5B9F4F0F94F79F44E06AED27
:10B770007AE0CE018C5B9F4F0F94F79F4CE062EC18
:10B780007AE0CE018C5B9F4F0F94F79F44E06EEB05
:10B790007AE0CE018C5B9F4F0F94F79F44E06EE5FB
:10B7A00072E0CE018C5B9F4F0F94F79F44E06AE5F7
:10B7B00072E0CE018C5B9F4F0F94F79F44E066E5EB
:10B7C00072E0CE018C5B9F4F0F94F79F44E062E5DF
:10B7D00072E0CE018C5B9F4F0F94F79F44E06EE4C4
:10B7E00072E0CE018C5B9F4F0F94F79F44E06AE4B8
:10B7F00072E0CE018C5B9F4F0F94F79F80E290E048
:10B800009CAF8BAF42E0BE01655C7F4FCE018C5B8D
:10B810009F4F0F94F79F41E06DEB7AE0CE018C5B78
:10B820009F4F0F94F79F44E066E472E0CE018C5B7B
:10B830009F4F0F94F79F44E062E472E0CE018C5B6F
:10B840009F4F0F94F79F44E069EB7AE0CE018C5B49
:10B850009F4F0F94F79F44E065EB7AE0CE018C5B3D
:10B860009F4F0F94F79F44E06EE372E0CE018C5B34
:10B870009F4F0F94F79F41E064EB7AE0CE018C5B21
:10B880009F4F0F94F79F44E06AE372E0CE018C5B18
:10B890009F4F0F94F79F86E591E3A0E0B0E0898386
:10B8A0009A83AB83BC8326961FAF0EAF269744E0E6
:10B8B000BE016F5F7F4FCE018C5B9F4F0F94F79F50
:10B8C000E9EFF6E484918F01882339F00E9493A078
:10B8D0000F5F1F4FF8018491F7CFE2E8FDE08491FC
:10B8E0008F01882339F00E9493A00F5F1F4FF8014A
:10B8F0008491F7CF8AE00E9493A00C94A0670E94E5
:10B90000A7A00C94A067882341F00E9493A0FFEFAA
:10B91000EF1AFF0AF7018491F6CFEDE8F0E1849188
:10B920007F01882341F00E9493A0FFEFEF1AFF0AE6
:10B93000F7018491F6CF8AE00E9493A0F8018491E8
:10B94000A9EFEA2EA6E4FA2E882341F00E9493A0E4
:10B95000FFEFEF1AFF0AF7018491F6CF4091120B27
:10B960005091130B6091140B7091150B85E890E1C9
:10B970000E94F7984091160B5091170B6091180B8D
:10B980007091190B82E890E10E94F79840911A0B90
:10B9900050911B0B60911C0B70911D0B8FE790E178
:10B9A0000E94F79840911E0B50911F0B6091200B45
:10B9B0007091210B8CE790E10E94F7988AE00E9439
:10B9C00093A0F8018491F9EFEF2EF6E4FF2E88237F
:10B9D00041F00E9493A0FFEFEF1AFF0AF701849154
:10B9E000F6CFE2E6F0E184917F01882341F00E94E6
:10B9F00093A0FFEFEF1AFF0AF7018491F6CF8AE0D8
:10BA00000E9493A0F8018491E9EFEE2EE6E4FE2E69
:10BA1000882341F00E9493A0FFEFEF1AFF0AF7017D
:10BA20008491F6CF4091020B5091030B6091040B6F
:10BA30007091050B89E590E10E94F7984091060B03
:10BA40005091070B6091080B7091090B86E590E10E
:10BA50000E94F79840910A0B50910B0B60910C0BD0
:10BA600070910D0B83E590E10E94F79840910E0BC9
:10BA700050910F0B6091100B7091110B80E590E1CC
:10BA80000E94F7988AE00E9493A0F801849179EFD0
:10BA9000E72E76E4F72E882341F00E9493A0FFEF73
:10BAA000EF1AFF0AF7018491F6CFE2E3F0E1849107
:10BAB0007F01882341F00E9493A0FFEFEF1AFF0A55
:10BAC000F7018491F6CF8AE00E9493A0F801849157
:10BAD00069EFE62E66E4F62E882341F00E9493A0DB
:10BAE000FFEFEF1AFF0AF7018491F6CF4091F20AB7
:10BAF0005091F30A6091F40A7091F50A89E290E19D
:10BB00000F94D09F4091F60A5091F70A6091F80A7D
:10BB10007091F90A86E290E10F94D09F4091FA0A61
:10BB20005091FB0A6091FC0A7091FD0A83E290E15A
:10BB30000F94D09F4091FE0A5091FF0A6091000B34
:10BB40007091010B80E290E10F94D09F8AE00E94F7
:10BB500093A0F801849159EFE52E56E4F52E882341
:10BB600041F00E9493A0FFEFEF1AFF0AF7018491C2
:10BB7000F6CFEBEEFFE084917F01882341F00E9435
:10BB800093A0FFEFEF1AFF0AF7018491F6CF8AE046
:10BB90000E9493A0F801849149EFE42E46E4F42E2C
:10BBA000882341F00E9493A0FFEFEF1AFF0AF701EC
:10BBB0008491F6CF4091EE0A5091EF0A6091F00A1D
:10BBC0007091F10A82EE9FE00E94F7984091EA0A94
:10BBD0005091EB0A6091EC0A7091ED0A8FED9FE0B5
:10BBE0000E94F7988AE00E9493A0F801849139EFAF
:10BBF000E32E36E4F32E882341F00E9493A0FFEF5A
:10BC0000EF1AFF0AF7018491F6CFECE2FFE084918E
:10BC10007F01882341F00E9493A0FFEFEF1AFF0AF3
:10BC2000F7018491F6CF8AE00E9493A0F8018491F5
:10BC300029EFE22E26E4F22E882341F00E9493A001
:10BC4000FFEFEF1AFF0AF7018491F6CF4091E60A61
:10BC50005091E70A6091E80A7091E90A83E29FE057
:10BC60000E94F7984091E20A5091E30A6091E40A39
:10BC70007091E50A80E29FE00E94F7984091DE0A09
:10BC80005091DF0A6091E00A7091E10A8DE19FE036
:10BC90000F94D09F4091CE0A5091CF0A6091D00A64
:10BCA0007091D10A8AE19FE00E94F7984091D20AF0
:10BCB0005091D30A6091D40A7091D50A87E19FE030
:10BCC0000E94F7984091D60A5091D70A6091D80AFD
:10BCD0007091D90A84E19FE00E94F7984091DA0AB6
:10BCE0005091DB0A6091DC0A7091DD0A81E19FE0EE
:10BCF0000E94F7988AE00E9493A0F801849199EF3E
:10BD0000E92E96E4F92E882341F00E9493A0FFEFDC
:10BD1000EF1AFF0AF7018491F6CFEFEFFEE084916E
:10BD20007F01882341F00E9493A0FFEFEF1AFF0AE2
:10BD3000F7018491F6CF8AE00E9493A0F8018491E4
:10BD4000B9EFEB2EB6E4FB2E882341F00E9493A0BE
:10BD5000FFEFEF1AFF0AF7018491F6CF4091C20A74
:10BD60005091C30A6091C40A7091C50A86EF9EE0A3
:10BD70000E94F7984091C60A5091C70A6091C80A7C
:10BD80007091C90A83EF9EE00E94F7984091CA0A19
:10BD90005091CB0A6091CC0A7091CD0A80EF9EE061
:10BDA0000E94F7988AE00E9493A0F8018491A9EF7D
:10BDB000EA2EA6E4FA2E882341F00E9493A0FFEF1A
:10BDC000EF1AFF0AF7018491F6CFE2EEFEE08491CC
:10BDD0007F01882341F00E9493A0FFEFEF1AFF0A32
:10BDE000F7018491F6CF8AE00E9493A0F801849134
:10BDF000F9EFEF2EF6E4FF2E882341F00E9493A086
:10BE0000FFEFEF1AFF0AF7018491F6CF40915E022F
:10BE100050915F02609160027091610288ED9EE036
:10BE20000E94F7982CEA35EC47E25EE360915A02F3
:10BE300070915B0280915C0290915D020F9472B8E8
:10BE4000AB01BC0185ED9EE00E94F7982CEA35EC31
:10BE500047E25EE36091560270915702809158026A
:10BE6000909159020F94D4ACAB01BC0182ED9EE0DD
:10BE70000E94F7988AE00E9493A0F8018491E9EF6C
:10BE8000EE2EE6E4FE2E882341F00E9493A0FFEF01
:10BE9000EF1AFF0AF7018491F6CFECEBFEE08491F4
:10BEA0007F01882341F00E9493A0FFEFEF1AFF0A61
:10BEB000F7018491F6CF8AE00E9493A0F801849163
:10BEC00079EFE72E76E4F72E882341F00E9493A0C5
:10BED000FFEFEF1AFF0AF7018491F6CF409152026B
:10BEE00050915302609154027091550282EB9EE092
:10BEF0000E94F7982CEA35EC47E25EE360914E022F
:10BF000070914F0280915002909151020F9472B83B
:10BF1000AB01BC018FEA9EE00E94F7982CEA35EC59
:10BF200047E25EE360914A0270914B0280914C02BD
:10BF300090914D020F94D4ACAB01BC018CEA9EE011
:10BF40000E94F7988AE00E9493A0F801849169EF1B
:10BF5000E62E66E4F62E882341F00E9493A0FFEFC0
:10BF6000EF1AFF0AF7018491F6CFE8E7FEE084912B
:10BF70007F01882341F00E9493A0FFEFEF1AFF0A90
:10BF8000F7018491F6CF8AE00E9493A0F801849192
:10BF900059EFE52E56E4F52E882341F00E9493A038
:10BFA000FFEFEF1AFF0AF7018491F6CF40914602A6
:10BFB0005091470260914802709149028EE69EE0DE
:10BFC0000E94F79820E030E040E752E4609142029E
:10BFD0007091430280914402909145020F94D4AC39
:10BFE000AB01BC018BE69EE00E94F7984091B90A34
:10BFF0005091BA0A6091BB0A7091BC0A88E69EE033
:10C000000E94F7988AE00E9493A0F801849149EF7A
:10C01000E42E46E4F42E882341F00E9493A0FFEF23
:10C02000EF1AFF0AF7018491F6CFECE3FEE084916A
:10C030007F01882341F00E9493A0FFEFEF1AFF0ACF
:10C04000F7018491F6CF8AE00E9493A0F8018491D1
:10C0500039EFE32E36E4F32E882341F00E9493A0BB
:10C06000FFEFEF1AFF0AF7018491F6CF4091B50A6E
:10C070005091B60A6091B70A7091B80A82E39EE0C7
:10C080000E94F79820E030E040E752E460913E02E1
:10C0900070913F0280914002909141020F94D4AC84
:10C0A000AB01BC018FE29EE00E94F7988AE00E94FB
:10C0B00093A0F801849129EFE22E26E4F22E882342
:10C0C00041F00E9493A0FFEFEF1AFF0AF70184915D
:10C0D000F6CFE5EDFDE084917F01882341F00E94D9
:10C0E00093A0FFEFEF1AFF0AF7018491F6CF8AE0E1
:10C0F0000E9493A0F801849199EFE92E96E4F92E1D
:10C10000882341F00E9493A0FFEFEF1AFF0AF70186
:10C110008491F6CF4091BD0A50E060E070E08BEC76
:10C120009DE00F94D09F8AE00E9493A0F801849133
:10C13000B9EFEB2EB6E4FB2E882341F00E9493A0CA
:10C14000FFEFEF1AFF0AF7018491F6CF8091B40A4E
:10C15000882371F1E8EBFDE084917F01882341F0B1
:10C160000E9493A0FFEFEF1AFF0AF7018491F6CF28
:10C170008AE00E9493A0F801849109EF16E48823D5
:10C1800039F00E9493A00F5F1F4FF8018491F7CF01
:10C1900040913A0250913B0260913C0270913D0205
:10C1A0008EEA9DE00E94F7988AE00E9493A0C8C69C
:10C1B000E2E9FDE084918F01882339F00E9493A089
:10C1C0000F5F1F4FF8018491F7CF8AE00E9493A080
:10C1D000B7C60E945CFCE9EFF6E484918F018823E6
:10C1E00039F00E9479860F5F1F4FF8018491F7CFD5
:10C1F000E1E4F1E184918F01882309F4A1C60E9452
:10C2000079860F5F1F4FF8018491F6CF8AE50E946F
:10C210003D99882309F493C00E9420996B017C0109
:10C2200020E030E040E751EC0F94CFB987FD43C0E8
:10C2300020E030E040EA50ECC701B6010F9481B134
:10C2400018160CF438C0F7FAF094F7F8F094C0928E
:10C25000BE0AD092BF0AE092C00AF092C10AE9EF8A
:10C26000F6E484918F01882339F00E9479860F5F6C
:10C270001F4FF8018491F7CFE3EDFAE14591549116
:10C28000EFE3F1E1859194912EE331E16EE178E005
:10C290000F9431A38C01F8018491882329F00E9426
:10C2A00079860F5F1F4FF7CF8AE00E9479868AE078
:10C2B0000E94798645C6E9EFF6E484918F018823D0
:10C2C00039F00E9479860F5F1F4FF8018491F7CFF4
:10C2D000EFE3F1E105911491F8018491882329F0AD
:10C2E0000E9479860F5F1F4FF7CFECE5F1E10591D2
:10C2F0001491F8018491882329F00E9479860F5FB8
:10C300001F4FF7CF61EF7FEF8FEF9FEF0F949603F3
:10C31000EAE5F1E105911491F8018491882329F06F
:10C320000E9479860F5F1F4FF7CF6BEF7FEF8FEF84
:10C330009FEF0F9496038AE00E94798601C6E9EF89
:10C34000F6E484918F01882339F00E9479860F5F8B
:10C350001F4FF8018491F7CFEFE3F1E185919491BC
:10C360006AE371E10F94985C8C01F8018491882351
:10C3700029F00E9479860F5F1F4FF7CF8AE00E9455
:10C3800079868091BE0A9091BF0AA091C00AB091AF
:10C39000C10ABC01CD01905842E00F94B1038AE07C
:10C3A0000E947986CDC550901B0210921B020F94FB
:10C3B000EC6F8091480F882321F086E190E00E9485
:10C3C00016FF80916702909168029093010280931A
:10C3D0000002E0911415F0E0EE0FFF1FEA56F74F50
:10C3E000608071802090A80F3090A90FC090E90F55
:10C3F000D090EA0FE090EB0FF090EC0FC8A2D9A21A
:10C40000EAA2FBA20091ED0F1091EE0F2091EF0F29
:10C410003091F00F0CA31DA32EA33FA34091F10F69
:10C420005091F20F6091F30F7091F40F48A759A744
:10C430006AA77BA78091F50F9091F60FA091F70F57
:10C44000B091F80F8CA79DA7AEA7BFA7C982DA82CB
:10C45000EB82FC820D831E832F83388749875A879E
:10C460006B877C878D879E87AF87B88B85E40E941A
:10C470003D99882359F00E9420999B01AC016CA53D
:10C480007DA58EA59FA50F9484B70AC020E030E05B
:10C4900040E050E46CA57DA58EA59FA50F9483B7C1
:10C4A0006CA77DA78EA79FA7E8A4F9A40AA51BA542
:10C4B0002CA13DA14EA15FA168A179A18AA19BA158
:10C4C000E4E1F5E1FF93EF93812C912CE8EEAE2EA1
:10C4D000E2E4BE2EDE019C966D010F949D288AE554
:10C4E0000E943D990F900F90882349F00E94209957
:10C4F0009B01AC0168A579A58AA59BA51EC020E07B
:10C5000030E040E050E468A579A58AA59BA50F948A
:10C5100084B76B017C0168A779A78AA79BA720E055
:10C5200030E040E251E40F9481B187FF0CC020E07D
:10C5300030E040E251E4C701B6010F9484B768A728
:10C5400079A78AA79BA7E8A4F9A40AA51BA52CA1F3
:10C550003DA14EA15FA168A179A18AA19BA1E4E1BF
:10C56000F5E1FF93EF93812C912CB0E7AB2EB1E472
:10C57000BB2EFE01BC966F010F949D2888E50E949A
:10C580003D990F900F90882379F00E9420999B018C
:10C59000AC0168A179A18AA19BA10F9484B768A37B
:10C5A00079A38AA39BA308C080E090E0A3E5B3E44D
:10C5B00088A399A3AAA3BBA389E50E943D998823D8
:10C5C00039F00E9420996CA37DA38EA39FA304C081
:10C5D0001CA21DA21EA21FA2E8A4F9A40AA51BA5C5
:10C5E0002CA13DA14EA15FA168A179A18AA19BA127
:10C5F000E4E1F5E1FF93EF93812C912CE8E4AE2E7A
:10C60000E2E4BE2EDE019C966D010F949D280F94EE
:10C61000EC6F84E090E0909373028093720210922A
:10C62000A90F1092A80F0F94133C6B017C01E091AD
:10C63000AB0FF0E0EE0FFF1FEA5CFE4E8591949188
:10C640000E945E990F900F90412C00E010E0411085
:10C650000C946E6D0F946F3F882311F40C946E6DE3
:10C660000C94626E8091670F9091680F892B09F08E
:10C6700067C485E090E09093680F8093670F60C473
:10C680008091670F9091680F892B09F059C486E05B
:10C6900090E09093680F8093670F52C488E50E94E2
:10C6A0003D99882399F00E9420990F94E3B8DB010B
:10C6B0002FEF30E00F9473BC20ED37E040E050E006
:10C6C0000F944FBCB9018EE20F94093B8AE50E949A
:10C6D0003D99882399F00E9420990F94E3B8DB01DB
:10C6E0002FEF30E00F9473BC20ED37E040E050E0D6
:10C6F0000F944FBCB9018DE20F94093B85E40E9471
:10C700003D99882309F41CC40E9420990F94E3B832
:10C71000DB012FEF30E00F9473BC20ED37E040E0F9
:10C7200050E00F944FBCB9018CE20F94093B08C450
:10C730000E948DD905C488E50E943D99882339F06F
:10C740000E9420990F94E9B880E00F940BA189E52D
:10C750000E943D99882339F00E9420990F94E9B8EE
:10C7600081E00F940BA18AE50E943D99882339F05E
:10C770000E9420990F94E9B882E00F940BA185E400
:10C780000E943D99882309F4DBC30E9420990F94ED
:10C79000E9B883E00F940BA1D3C388E50E943D99CB
:10C7A000882339F00E9420990F94E9B880E00F9413
:10C7B000D9A089E50E943D99882339F00E942099EB
:10C7C0000F94E9B881E00F94D9A08AE50E943D99C1
:10C7D000882339F00E9420990F94E9B882E00F94E1
:10C7E000D9A085E40E943D99882309F4A9C30E9439
:10C7F00020990F94E9B883E00F94D9A0A1C3809148
:10C800002E021F928F9380912A021F928F93809104
:10C810002D021F928F93809129021F928F938091F6
:10C820002C021F928F93809128021F928F938091E8
:10C830002B021F928F93809127021F928F9389EB77
:10C8400090E19F938F930F94FAB00FB6F894DEBFE8
:10C850000FBECDBF75C381E0809383080E948DD940
:10C860006FC388E50E943D99882331F00E9420998A
:10C870000F94E9B86093230289E50E943D998823CB
:10C8800031F00E9420990F94E9B8609324028AE560
:10C890000E943D99882331F00E9420990F94E9B8B5
:10C8A0006093250285E40E943D99882331F00E941F
:10C8B00020990F94E9B86093260203E015E0D801AF
:10C8C0008D918D01882319F00E947986F8CF6091AF
:10C8D000230270E080E090E04AE00F940F030F9491
:10C8E000D50606E115E0F80181918F01882319F042
:10C8F0000E947986F8CF6091240270E080E090E099
:10C900004AE00F940F030F94D50609E215E0D80111
:10C910008D918D01882319F00E947986F8CF60915E
:10C92000250270E080E090E04AE00F940F030F943E
:10C93000D5060CE315E0F80181918F01882319F0E9
:10C940000E947986F8CF6091260270E080E090E046
:10C950004AE00F940F030F94D506F2C288E50E94B7
:10C960003D99882339F00E9420990F94E9B880E01E
:10C970000F948CA089E50E943D99882339F00E948C
:10C9800020990F94E9B881E00F948CA08AE50E9469
:10C990003D99882339F00E9420990F94E9B882E0EC
:10C9A0000F948CA085E40E943D99882309F4C8C2A5
:10C9B0000E9420990F94E9B883E00F948CA0C0C224
:10C9C00088E50E943D99882339F00E9420990F94B0
:10C9D000E9B880E00F943FA089E50E943D99882343
:10C9E00039F00E9420990F94E9B881E00F943FA09C
:10C9F0008AE50E943D99882339F00E9420990F947E
:10CA0000E9B882E00F943FA085E40E943D99882315
:10CA100009F496C20E9420990F94E9B883E00F941C
:10CA20003FA08EC20F948B938BC2123311F40C94DF
:10CA30002E73163040F09FB7F894809102018B7FDF
:10CA4000809302019FBF84E690E00E9480931F5F65
:10CA50000F946F3F81110C942E73E7CF8FE495E014
:10CA60009F938F930F9424BD80910F149091101475
:10CA70008B5D9D4E9F938F930F9424BD8AE090E031
:10CA80000F9438BD0F900F900F900F9059C284E50E
:10CA90000E943D99882309F4C5C10F94EC6FE09181
:10CAA0005508F0915608319681918032E9F389302A
:10CAB000D9F390ED980F9A3008F425C18F3379F0AF
:10CAC000E9E0F1E184918F01882311F40C94BD33E6
:10CAD0000E9479860F5F1F4FF8018491F5CFA090D7
:10CAE000AA0F0A2C000CBB080E94ABEFE091AB0F21
:10CAF000F0E0EE0FFF1FE650FF4E859194910E94EB
:10CB000074EF41E060E083E29BE00E946C9C61E096
:10CB100075E083E29BE00F94D33911E028EFE22E19
:10CB200020E1F22E88EFC82E80E1D82EF701459142
:10CB30005491612F81E00E9450EF1F5F143091F7F4
:10CB400084E090E0909373028093720211E0E12CF4
:10CB5000F12C88248394912CF601859194910F9463
:10CB600059B062E0680F482D83E29BE00E946C9C04
:10CB7000C4018E0D9F1D0F94A74AFFEF8F1A9F0AC5
:10CB800024E08216910441F70F94526981E00F94DA
:10CB9000C8878091AA0F082E000C990B9501281BBD
:10CBA000390B37FF03C03195219531092530310507
:10CBB0000CF488C08A159B050CF41150A816B90610
:10CBC0000CF41F5F143014F1E114F10411F00C9413
:10CBD00059730E94ABEFE091AB0FF0E0EE0FFF1F37
:10CBE000E650FF4E859194910E9474EF11E0F6019A
:10CBF00045915491612F81E00E9450EF1F5F1430E6
:10CC0000B1F7EE24E394F12C0C9459731116FCF057
:10CC1000E114F104D9F031E0E31AF1080E94ABEF1E
:10CC2000E091AB0FF0E0EE0FFF1FE650FF4E859155
:10CC300094910E9474EF11E0F60145915491612F97
:10CC400081E00E9450EF1F5F1430B1F711E041E026
:10CC500060E083E29BE00E946C9C6EE178E083E2FE
:10CC60009BE00F94D33942E060E083E29BE00E94B6
:10CC70006C9C6EE178E083E29BE00F94D33943E053
:10CC800060E083E29BE00E946C9C6EE178E083E2CE
:10CC90009BE00F94D339412F60E083E29BE00E9438
:10CCA0006C9C61E075E083E29BE00F94D339A09027
:10CCB000AA0F0A2C000CBB0864E670E080E090E04C
:10CCC0000F94DB3B0F946F3F882309F442CF82E03F
:10CCD0000F94EB400F946F3F8111FCCF6AE070E03E
:10CCE00080E090E00F94DB3B0F946F3F8111FCCF0D
:10CCF00082E090E090937302809372021E0D1150B7
:10CD000010939E1A06C00E9420990F94E9B8609370
:10CD10009E1A20919E1A81E090E0022E01C0880F99
:10CD20000A94EAF790915208892B809352082223A3
:10CD300009F433C0E9EFF6E484918F01882339F0D8
:10CD40000E9479860F5F1F4FF8018491F7CFE7E0CB
:10CD5000F1E184918F01882339F00E9479860F5F79
:10CD60001F4FF8018491F7CF60919E1A70E080E028
:10CD700090E00F9496038AE00E947986E5E0F1E165
:10CD800005911491F8018491882311F40C94BD331A
:10CD90000E9479860F5F1F4FF5CF86E40E943D9970
:10CDA0008823D9F00E9420996B017C0160938D1A31
:10CDB00070938E1A80938F1A9093901A20E030E02F
:10CDC000A9010F94CFB9181644F4C0928602D092EC
:10CDD0008702E0928802F0928902E9EFF6E48491FA
:10CDE0008F01882339F00E9479860F5F1F4FF80169
:10CDF0008491F7CFE3E0F1E105911491F80184917A
:10CE0000882329F00E9479860F5F1F4FF7CF60912A
:10CE1000141570E080E090E00F9496038AE00E9481
:10CE200079868EC0E9EFF6E484918F01882339F08A
:10CE30000E9479860F5F1F4FF8018491F7CFE6E5D6
:10CE4000F1E105911491F8018491882329F00E9461
:10CE500079860F5F1F4FF7CF00910F1410911014B8
:10CE60000B5D1D4ED8018D918D01882319F00E9414
:10CE70007986F8CFEEEFF0E184918F01882311F4E9
:10CE80000C94BD330E9479860F5F1F4FF801849187
:10CE9000F5CF61104BC0552009F448C081E0809364
:10CEA000480B0F94D96F9B01AC0180E0CB57DF4F4B
:10CEB0002883C558D040CA57DF4F3883C658D04062
:10CEC000C957DF4F4883C758D040C857DF4F5883F2
:10CED000C858D0400F94D96FCB57DF4F2881C55821
:10CEE000D040CA57DF4F3881C658D040C957DF4FAE
:10CEF0004881C758D040C857DF4F5881C858D040E4
:10CF00000F94C0469B01AC016091F10F7091F20F3C
:10CF10008091F30F9091F40F0F9483B76093F10F0A
:10CF20007093F20F8093F30F9093F40F8091480F5A
:10CF3000882321F084E190E00E9416FF10926B1A82
:10CF400081E090E090937302809372020F94133CFF
:10CF50006093961A7093971A8093981A9093991ADF
:10CF6000E0910F14F0911014EE5DFD4E8081813040
:10CF700011F00C946C73E3EDFAE105911491F80152
:10CF80008491882329F00E9479860F5F1F4FF7CF85
:10CF90008AE00E9479860C946C73C0900F15D09033
:10CFA0001015E0901115F09012152091F50F3091A9
:10CFB000F60F4091F70F5091F80FC701B6010F948B
:10CFC00083B72DEC3CEC4CEC5DE30F94CFB9181615
:10CFD00014F00C943735C092F50FD092F60FE09212
:10CFE000F70FF092F80F85EF9FE00F94427980E001
:10CFF0000F9481A30C946C730E9420992091C20A13
:10D000003091C30A4091C40A5091C50A0F9484B765
:10D010006093E90F7093EA0F8093EB0F9093EC0FFE
:10D020000C942B360E9420992091C60A3091C70A91
:10D030004091C80A5091C90A0F9484B76093ED0FCC
:10D040007093EE0F8093EF0F9093F00F0C9438369F
:10D050000E9420992091CA0A3091CB0A4091CC0AB3
:10D060005091CD0A0F9484B76093F10F7093F20F33
:10D070008093F30F9093F40F0C94253720E030E069
:10D0800040E85FE36091F50F7091F60F8091F70F24
:10D090009091F80F0F9484B76093F50F7093F60F8B
:10D0A0008093F70F9093F80FE090F10FF090F20F4C
:10D0B0000091F30F1091F40F2091ED0F3091EE0FCE
:10D0C0004091EF0F5091F00F6091E90F7091EA0FCE
:10D0D0008091EB0F9091EC0FE4E1F5E1FF93EF937A
:10D0E000812C912CE8ECAE2EE3E4BE2EF5EFCF2E92
:10D0F000FFE0DF2E0F949D280F900F900C94764246
:10D1000082E090E0909373028093720210925A1A18
:10D110001092591A0C94C3470F94EC9FAB01BC01B9
:10D120004093350F5093360F6093370F7093380F3D
:10D1300080E89EE00E944D7903CFE091AB0FF0E0D4
:10D14000EE0FFF1FEC55FC4B859194910F94933F8C
:10D1500082E090E090937302809372029093E509CD
:10D160008093E4098091480F882321F082E090E0C9
:10D170000E9416FF0F94133C6093961A7093971AAF
:10D180008093981A9093991ADBCE0F94133CDC018C
:10D19000CB0188199909AA09BB09893E9340A105C9
:10D1A000B10508F46EC08091480F811166C0ECE7AC
:10D1B000FCE084918F01882339F00E9479860F5F0B
:10D1C0001F4FF8018491F7CFE0919E1A24E0E29F6F
:10D1D000F0011124E75AFB4E6081718182819381B5
:10D1E00041E00F94B103E8E7FCE084918F018823CC
:10D1F00039F00E9479860F5F1F4FF8018491F7CFB5
:10D2000060919E1A70E080E090E00F949603F10127
:10D21000849104E71CE0882339F00E9479860F5F2F
:10D220001F4FF8018491F7CFF7FE03C006E416E024
:10D2300019C00F94133C970186010854144F2F4FC7
:10D240003F4F48015901861A970AA80AB90AC50131
:10D25000B401A30192010F9448B7CA01B9010F9418
:10D26000960308C0D8018D918D01882319F00E9482
:10D270007986F8CF8AE00E9479860F94133C4B019F
:10D280005C010F94526980E00F94C88780E00F948E
:10D29000EB40BFEFCB16DB06EB06FB0609F056C0F2
:10D2A0009091530880919E1A992341F190E08C014E
:10D2B000000F111F000F111F075A1B4E880F991FD7
:10D2C000FC01EA56F74F60817181072E000C880B34
:10D2D000990B0F9487B120E030E040E85FE30F94B2
:10D2E00083B79B01AC01F8016081718182819381D8
:10D2F0000F94CFB987FF60C00C94C24D90E08C01B1
:10D30000000F111F000F111F075A1B4E880F991F86
:10D31000FC01EA56F74F60817181072E000C880BE3
:10D32000990B0F9487B120E030E040E85FE30F9461
:10D3300084B79B01AC01D8016D917D918D919C9139
:10D340000F9481B11816C4F50C94C24DF7FE02C0BB
:10D350000C94C24D80919E1A90E08C01000F111F19
:10D36000000F111F075A1B4E880F991FFC01EA5628
:10D37000F74F60817181072E000C880B990B0F9479
:10D3800087B19B01AC01F801608171818281938139
:10D390000F9483B70F94E3B897FF07C090958095DB
:10D3A000709561957F4F8F4F9F4F66307105810556
:10D3B000910514F40C94C24D0F94133C6B017C0145
:10D3C0000C94C24D0F94EC6F88E50E943D99882320
:10D3D00019F0179A10927A0889E50E943D998823DE
:10D3E00019F0169A10927B088AE50E943D9985E40F
:10D3F0000E943D99882311F40C94B04F149A0C9418
:10D40000B04F1A8219824AE050E0BE016F5F7F4F31
:10D41000C8010F940EAF79A368A389819A818615FC
:10D42000970509F08DCD4AE050E0BE016F5F7F4F58
:10D43000C2010F940EAF7BA36AA389819A818815DC
:10D44000990509F07DCD4AE050E0BE016F5F7F4F46
:10D45000C6010F940EAF7DA36CA309811A810A1532
:10D460001B0509F06DCD8FE790E09FA38EA34501CA
:10D47000BFEF8B1A9B0AF50180818D3201F55401B3
:10D480006501FFEFAF1ABF0AD6018C910F94693C7A
:10D49000382E8823A9F3C818D908BC2C9601332745
:10D4A0002330310569F543E050E06AE67EE5C401CA
:10D4B0000F947AB0892B09F043C01FA21EA233201B
:10D4C00009F43ECDCE0101960F94297D882309F4FD
:10D4D00037CDFE01B096DE011196AE01485D5F4F7B
:10D4E000219131918D919D918217930708F449C044
:10D4F0002817390708F424CDE417F50789F720CD5C
:10D500002530310571F445E050E064E67EE5C40164
:10D510000F947AB0892BA1F481E090E09FA38EA3B1
:10D52000CECF2430310561F444E050E06FE57EE574
:10D53000C4010F947AB0892B19F482E090E0EECF09
:10D540008EEF8C0D823008F0FBCCF80181818237A0
:10D5500009F0F6CC8281833609F0F2CCF2E0BF12FA
:10D5600003C083E090E0DACFD80113968C9190ED60
:10D57000980F9A3008F0E4CC082E000C990B8E9787
:10D58000CDCFE091AB0FF0E0EE0FFF1FEC57F34F64
:10D59000859194910E945E9943E85CE062E080E0AE
:10D5A0000E9450EFF70161917F01862FCB57DF4F2B
:10D5B0006883C558D0400F94693CCB57DF4F6881D2
:10D5C000C558D040811105C083E29BE00E94929F24
:10D5D000E9CFE091AB0FF0E0EE0FFF1FE158F34F02
:10D5E0004591549163E080E00E9450EF88EE93E013
:10D5F0000F94CF4382E390E00E94809384E50F94E0
:10D600002B3A84EF91E00E94809388EE93E00F9490
:10D61000CF4382E390E00E94809384E50F942B3AFD
:10D6200084E090E090937302809372020F945269A9
:10D6300081E00F94C8870F946F3F8823B9F30F944C
:10D640006F3F8111FCCF6AE070E080E090E00F94C2
:10D65000DB3B0F946F3F8111FCCF82E090E0909311
:10D6600073028093720281E00F945C420E94ABEFE0
:10D6700080E00F94EB4064CCE8968CAC9DACAEACF3
:10D68000BFACE897880E991EAA1EBB1EA7968CAE4B
:10D690009DAEAEAEBFAEA797E8968CAC9DACAEACDF
:10D6A000BFACE897881A990AAA0ABB0AC501B40157
:10D6B000A30192010F9439B7A7962CAD3DAD4EADA5
:10D6C0005FADA7970F944FBCD701C601820F931F80
:10D6D000A41FB51F84319105A105B105E4F06C01CB
:10D6E0007D018C3E9105A105B1052CF02BEEC22EDB
:10D6F000D12CE12CF12C30E8C316D104E104F10463
:10D70000ACF09EEF492E512C612C712C4C185D0809
:10D710006E087F080DC004E1C02ED12CE12CF12C45
:10D7200084E1482E512C612C712C02C02601370156
:10D73000EAE7FDE084918F01882339F00E94B8DB8D
:10D740000F5F1F4FF8018491F7CFC701B6010F9407
:10D750009603E5E7FDE084918F01882339F00E946C
:10D76000B8DB0F5F1F4FF8018491F7CFC301B201FF
:10D770000F949603EEE6FDE084918F01882339F043
:10D780000E94B8DB0F5F1F4FF8018491F7CF42E092
:10D790006F966FAD6F97AC967FADAC97AD968FAD32
:10D7A000AD97AE969FADAE970F94B103E7E6FDE05F
:10D7B00084918F01882339F00E94B8DB0F5F1F4FDF
:10D7C000F8018491F7CF42E0AF966FADAF97E09646
:10D7D0007FADE097E1968FADE197E2969FADE2973E
:10D7E0000F94B1038AE00E94B8DB8091E209909126
:10D7F000E309039714F40C949A59C301B2010F94EE
:10D8000087B120E030E040E850E40F94D4AC4B0105
:10D810005C016F962FAD6F97AC963FADAC97AD9610
:10D820004FADAD97AE965FADAE97AF966FADAF977C
:10D83000E0967FADE097E1968FADE197E2969FADE0
:10D84000E2970F9483B720ED3FE049E450E40F9452
:10D85000D4AC20E030E040E05FE30F94D4AC9B0117
:10D86000AC01C501B4010F9472B84B015C01A796DD
:10D870006CAD7DAD8EAD9FADA7970F9487B120E0C5
:10D8800030E04AE754E40F9472B8A2966CAF7DAFD3
:10D890008EAF9FAFA297E1E6FDE084918F018823D0
:10D8A00039F00E94B8DB0F5F1F4FF8018491F7CF6A
:10D8B00042E0C501B4010F94B103EBE5FDE08491B2
:10D8C0008F01882339F00E94B8DB0F5F1F4FF801EA
:10D8D0008491F7CF42E0A2966CAD7DAD8EAD9FAD49
:10D8E000A2970F94B1038AE00E94B8DB2AE939E9D4
:10D8F00049E15FE3C501B4010F94D4AC4B015C0175
:10D90000609315097093160980931709909318096D
:10D910009B01AC010F9484B7A2962CAD3DAD4EADEA
:10D920005FADA2970F9472B86093110970931209BA
:10D930008093130990931409A2962CAD3DAD4EAD82
:10D940005FADA297C501B4010F94D4AC20E030E0E4
:10D9500040E05EE30F94D4AC60930D0970930E0920
:10D9600080930F0990931009EDE4FDE084918F01FD
:10D97000882339F00E94B8DB0F5F1F4FF8018491B4
:10D98000F7CF8AE00E94B8DBE7E4FDE084918F01E5
:10D99000882339F00E94B8DB0F5F1F4FF801849194
:10D9A000F7CF609115097091160980911709909130
:10D9B000180942E00F94B1038AE00E94B8DBE1E469
:10D9C000FDE084918F01882339F00E94B8DB0F5F5E
:10D9D0001F4FF8018491F7CF6091110970911209DE
:10D9E000809113099091140942E00F94B1038AE0E9
:10D9F0000E94B8DBEBE3FDE084918F01882339F0CE
:10DA00000E94B8DB0F5F1F4FF8018491F7CF609140
:10DA10000D0970910E0980910F099091100942E053
:10DA20000F94B1038AE00E94B8DB0C949A5980935A
:10DA300069090C94AE59A4961FAEA4970C94D359BF
:10DA400000E010E0809101018460809301010115E4
:10DA5000110509F04EC09FB7F894809102018460CF
:10DA6000809302019FBF0F5F1F4FB1E04B1609F477
:10DA700050C04B1608F047C084E090E00E948093AD
:10DA80000F94133C46015701F0EC8F0EF7E29F1EF6
:10DA9000F9E0AF1EB11C86169706A806B90610F06D
:10DAA0000C942763E091AB0FF0E0EE0FFF1FEE5CEC
:10DAB000FE4E859194910E945E9910929708109263
:10DAC0009608109299081092980810929B0810924C
:10DAD0009A080F94EC6F149A442443940F9452695B
:10DAE00081E00F94C887043F21E0120709F0AACF14
:10DAF000A7CF0431110509F0B6CF9FB7F8948091F4
:10DB000002018B7FADCFE2E04E1609F46BC00C949E
:10DB1000276384E090E00E9480930F946F3F8823F6
:10DB2000E9F2E0911415F0E0EE0FFF1FEA56F74F0F
:10DB300071826082E091AB0FF0E0EE0FFF1FEA52BE
:10DB4000F34D859194910E945E9944E060E083E2F8
:10DB50009BE00E946C9C82E00F94F909E0911415FF
:10DB600024E0E29FF0011124E75AFB4E808191816D
:10DB7000A281B3818BAF9CAFADAFBEAFCE01CB96D0
:10DB80000F94583FBC0183E29BE00F94D3396DEFB3
:10DB900074E083E29BE00F94D339E0911415F0E038
:10DBA000EE0FFF1FEA56F74F60817181072E000CC0
:10DBB000880B990B0F9487B16BAF7CAF8DAF9EAF85
:10DBC000CE01CB960F94583FBC0183E29BE00F94AB
:10DBD000D3396FEF74E083E29BE00F94D33962E0B6
:10DBE000462E7CCFE0911415AE2EB12CF501EE0F30
:10DBF000FF1FEA56F74F60817181072E000C880BDA
:10DC0000990B0F9487B1F501EE0FFF1FEE0FFF1F69
:10DC1000E75AFB4E20813181428153810F9483B7B3
:10DC20004B015C0120E030E0A9010F94CFB9181638
:10DC30005CF420E030E040E85FE3C501B4010F94FC
:10DC400081B187FF1DC00AC020E030E040E85FEBF3
:10DC5000C501B4010F94CFB9181694F4E091AB0F3D
:10DC6000F0E0EE0FFF1FEA5CFE4E859194910E945A
:10DC70005E990F94133C6B017C01412C0C942A6338
:10DC800044E061E083E29BE00E946C9CE09114150B
:10DC900034E0E39FF0011124E75AFB4E808191812B
:10DCA000A281B3818BAF9CAFADAFBEAFCE01CB969F
:10DCB0000F94583FBC0183E29BE00F94D33904E1F9
:10DCC00010E00CCF9FB7F894809102018B7F809376
:10DCD00002019FBF1092510810925008E091AB0FC3
:10DCE000F0E0EE0FFF1FE25DFE4E859194910E94E1
:10DCF0005E9982E090E0909373028093720281E0DB
:10DD000080934D0FE091AB0FF0E0EE0FFF1FE25D4F
:10DD1000FE4E859194910F94933F8CE40E943D991F
:10DD2000882359F00E9420999B01AC016CA57DA528
:10DD30008EA59FA50F9484B70AC020E030E040EA8A
:10DD400052E46CA57DA58EA59FA50F9483B76CA703
:10DD50007DA78EA79FA720E030E040EA52E46CA5A3
:10DD60007DA58EA59FA50F9484B720E030E044E305
:10DD700052E40F9483B76CA77DA78EA79FA7E8A452
:10DD8000F9A40AA51BA52CA13DA14EA15FA168A1E4
:10DD900079A18AA19BA1E4E16E2EE5E17E2E7F921E
:10DDA0006F92812C912CFCEAAF2EF2E4BF2EDE01A3
:10DDB0009C966D010F949D280F94EC6F20E030E04D
:10DDC00040E751E46CA57DA58EA59FA50F9483B770
:10DDD0006CA77DA78EA79FA7E8A4F9A40AA51BA5F9
:10DDE0002CA13DA14EA15FA168A179A18AA19BA10F
:10DDF0007F926F92812C912CA0E8AA2EA1E4BA2EDA
:10DE00000F949D280F94EC6F20E030E040EA51E43D
:10DE10006CA57DA58EA59FA50F9483B76CA77DA744
:10DE20008EA79FA7E8A4F9A40AA51BA52CA13DA134
:10DE30004EA15FA168A179A18AA19BA17F926F9257
:10DE40000F949D280F94EC6F0F94EC6FE091AB0F43
:10DE5000F0E0EE0FFF1FE65DFE4E859194910E946B
:10DE60005E99149A64E670E080E090E00F94DB3BEA
:10DE70009FB7F894809102018460809302019FBF54
:10DE80000F900F900F900F900F900F9000E010E008
:10DE90000F946F3F811115C00233110591F00630C8
:10DEA000110544F09FB7F894809102018B7F809315
:10DEB00002019FBF84E690E00E9480930F5F1F4F96
:10DEC000E7CF9FB7F894809102018B7F8093020186
:10DED0009FBF84E090E09093730280937202E09180
:10DEE000AB0FF0E0EE0FFF1FEA5DFE4E85919491BF
:10DEF00041E060E00E944EEA082E000C990B9093DE
:10DF0000510880935008892B59F4E091AB0FF0E051
:10DF1000EE0FFF1FEE5DFE4E859194910E9419EB6E
:10DF200081E00F945C420E94ABEF41E060E083E24D
:10DF30009BE00E946C9CE091AB0FF0E0EE0FFF1FA6
:10DF4000EF55FF4E859194910E9474EF42E060E09E
:10DF500083E29BE00E946C9CE091AB0FF0E0EE0F3F
:10DF6000FF1FE356FF4E859194910E9474EF84E069
:10DF700090E09093730280937202809163028823F1
:10DF800091F0511004C08091A608882361F00F948D
:10DF9000415D09C00F94526981E00F94C887809158
:10DFA0006302811105C00F946F3F882399F315C058
:10DFB000511004C08091A6088823A9F30F94E55C52
:10DFC000882389F388EE93E00F94CF4382E390E0B7
:10DFD0000E94809384E50F942B3A809163028823FA
:10DFE00061F0511004C08091A608882331F010928E
:10DFF0003514109234141092A70882E090E09093A8
:10E0000073028093720220E030E04CE852E46CA589
:10E010007DA58EA59FA50F9484B76CA77DA78EA71D
:10E020009FA7E8A4F9A40AA51BA52CA13DA14EA178
:10E030005FA168A179A18AA19BA1E4E16E2EE5E12F
:10E040007E2E7F926F92812C912CF0EAAF2EF1E41C
:10E05000BF2EFE01BC966F010F949D2820E030E09A
:10E0600048E452E46CA57DA58EA59FA50F9484B7C6
:10E070006CA77DA78EA79FA7E8A4F9A40AA51BA556
:10E080002CA13DA14EA15FA168A179A18AA19BA16C
:10E090007F926F92812C912CA12CA0E4BA2E0F9428
:10E0A0009D2810925108109250080F943DA184EFC2
:10E0B00091E00F94CF4382E390E00E94809384E547
:10E0C0000F942B3A0F900F900F900F908091500863
:10E0D00090915108019709F4CFC110925108109204
:10E0E0005008E4E0F0E0F0937302E09372020E94C3
:10E0F000ABEF40E060E083E29BE00E946C9CE0912B
:10E10000AB0FF0E0EE0FFF1FE355FF4E85919491AA
:10E110000E9474EF41E061E083E29BE00E946C9C0E
:10E12000E091AB0FF0E0EE0FFF1FEC53F74B859142
:10E1300094910E9474EF42E061E083E29BE00E94D0
:10E140006C9CE091AB0FF0E0EE0FFF1FE755FF4E28
:10E15000859194910E9474EF43E061E083E29BE03B
:10E160000E946C9CE091AB0FF0E0EE0FFF1FEB55AF
:10E17000FF4E859194910E9474EF41E060E083E24C
:10E180009BE00E946C9C61E075E083E29BE00F9451
:10E19000D339E090AA0F0E2C000CFF0801E010E02C
:10E1A000C0905008D0905108C114D10409F07AC031
:10E1B0000F94526981E00F94C8878091AA0F082EAE
:10E1C000000C990B9701281B390B37FF03C03195C1
:10E1D00021953109253031050CF454C08E159F0569
:10E1E00014F401501109E816F90634F40F5F1F4FBB
:10E1F0000430110564F009C00430110534F4011530
:10E20000110529F401E010E002C003E010E041E054
:10E2100060E083E29BE00E946C9C6EE178E083E228
:10E220009BE00F94D33942E060E083E29BE00E94E0
:10E230006C9C6EE178E083E29BE00F94D33943E07D
:10E2400060E083E29BE00E946C9C6EE178E083E2F8
:10E250009BE00F94D339402F60E083E29BE00E9463
:10E260006C9C61E075E083E29BE00F94D339E09011
:10E27000AA0F0E2C000CFF0864E670E080E090E02E
:10E280000F94DB3B0F946F3F882309F489CF1093E1
:10E2900051080093500864EF71E080E090E00F9423
:10E2A000DB3B7ECF0E94ABEF0F942992A2E08A2E37
:10E2B000912C909273028092720222E0C216D104D5
:10E2C00009F453C033E0C316D10409F0BEC020E006
:10E2D00030E048E452E46CA57DA58EA59FA50F947F
:10E2E00084B76CA77DA78EA79FA7E8A4F9A40AA569
:10E2F0001BA52CA13DA14EA15FA168A179A18AA176
:10E300009BA17F926F92812C912CA12CE0E4BE2ED8
:10E31000DE019C966D010F949D280E94ABEF40E0BA
:10E3200060E083E29BE00E946C9CE091AB0FF0E028
:10E33000EE0FFF1FEF54FF4E859194910E9474EFF2
:10E3400042E060E083E29BE00E946C9CE091AB0FB6
:10E35000F0E0EE0FFF1FE05EFD4B859194910E946F
:10E3600074EF0F900F9010E060C020E030E04CE8B8
:10E3700052E46CA57DA58EA59FA50F9484B76CA7CC
:10E380007DA78EA79FA7E8A4F9A40AA51BA52CA189
:10E390003DA14EA15FA168A179A18AA19BA17F9215
:10E3A0006F92812C912CE0EAAE2EE1E4BE2EDE01CC
:10E3B0009C966D010F949D2820E030E048E452E4E3
:10E3C0006CA57DA58EA59FA50F9484B76CA77DA78E
:10E3D0008EA79FA7E8A4F9A40AA51BA52CA13DA17F
:10E3E0004EA15FA168A179A18AA19BA17F926F92A2
:10E3F000812C912CA12CF0E4BF2E0F949D280F941A
:10E400003DA160CE0F94526981E00F94C88765E505
:10E4100070E080E090E00F94DB3BB1E0EB1AF10894
:10E4200089F71F5F143109F451CE43E0612F83E275
:10E430009BE00E946C9C68EE75E083E29BE00F9489
:10E44000D3390AE0E02EF12CDDCF0E94ABEF42E0A1
:10E4500060E083E29BE00E946C9CE091AB0FF0E0F7
:10E46000EE0FFF1FEB54FF4E859194910E9474EFC5
:10E4700081E00F945C422ACE3092A90F2092A80F1F
:10E4800020E030E040EA50E46CA57DA58EA59FA574
:10E490000F9484B76CA77DA78EA79FA7E8A4F9A4C3
:10E4A0000AA51BA52CA13DA14EA15FA168A179A140
:10E4B0008AA19BA1E4E16E2EE5E17E2E7F926F9210
:10E4C000812C912CA12CF0E4BF2EFE01BC966F0193
:10E4D0000F949D28A50194016CA57DA58EA59FA5EF
:10E4E0000F9483B76CA77DA78EA79FA7E8A4F9A474
:10E4F0000AA51BA52CA13DA14EA15FA168A179A1F0
:10E500008AA19BA17F926F92812C912CA8EEAA2EBA
:10E51000A2E4BA2E0F949D28E8A4F9A40AA51BA58D
:10E520002D813E814F81588569817A818B819C81C3
:10E530007F926F92812C912CB8E4AB2EB2E4BB2E6B
:10E540000F949D28E984FA840B851C852D813E81DA
:10E550004F81588569817A818B819C817F926F92EE
:10E56000812C912CE0E7AE2EE1E4BE2E0F949D2885
:10E5700020E030E040E050E46CA57DA58EA59FA58D
:10E580000F9484B76CA77DA78EA79FA7E984FA8410
:10E590000B851C852D813E814F81588569817A814B
:10E5A0008B819C817F926F92812C912CF8EEAF2E03
:10E5B000F2E4BF2E0F949D28CE010D960F94427960
:10E5C000809100029091010280936702909368020B
:10E5D0009F938F9389E191E19F938F938E01055CC7
:10E5E0001F4F1F930F930F9452B160E0C8014FD19A
:10E5F000E091AB0FF0E0EE0FFF1FE05EF54E85916E
:10E6000094910F94933F10924D0F10924C0F1092D3
:10E610004B0F50921B020FB6F894DEBF0FBECDBF5A
:10E620008091A608882311F40C94A067FDD10F9463
:10E63000EC6F8091201290912112892B21F00E9481
:10E640000F32F2D1F6CFB0D080911315882311F498
:10E650000C94A0670F94BA7B0C94A0679FB7F894B2
:10E66000809102018B7F809302019FBF0F94EC6F1A
:10E670000F946F3F882329F084E690E00E948093F6
:10E68000F7CF81E00F945C42E091AB0FF0E0EE0F2A
:10E69000FF1FE05EF54E859194910F94933F109289
:10E6A0004D0F10924C0F10924B0F70921B020C9456
:10E6B000A06713E00C94276660962CAD3DAD4EAD7F
:10E6C0005FAD6097C201B1010F9481B1181614F4C7
:10E6D0000C947D3A0C94913AC457DF4F0FB6F894DE
:10E6E000DEBF0FBECDBFDF91CF911F910F91FF9085
:10E6F000EF90DF90CF90BF90AF909F908F907F90E2
:10E700006F905F904F903F902F900895CF93FC01B2
:10E7100040910F145091101480911D1290911E126F
:10E720004817590739F420912012309121121216FE
:10E730001306BCF1C62F9C012E0F3F1F84179507AF
:10E740003CF424593F4F81E0241735075CF129C080
:10E75000B90163597F4F6E3E714008F12C5F3F4F06
:10E760002E3E314018F449365105CCF4E459FF4FA0
:10E77000E417F507B4F44DEE51E0481B590B60E087
:10E7800070E08E5D9D4E0F94ADBCCC2309F0F894E3
:10E7900010921E1210921D12CC2309F0789481E081
:10E7A00001C080E0CF9108950F945738009719F079
:10E7B0001092B51A03C021E02093B51A61E0892BAD
:10E7C00009F460E060931B021092A6081092A7085B
:10E7D00087E69FE00F940AB780911B028093640242
:10E7E00008959091B30A911107C09091C00095FFD0
:10E7F000FCCF8093C6000895913031F49091C80009
:10E8000095FFFCCF8093CE00089560912012709107
:10E81000211261157105B1F120910F14309110147E
:10E8200040E050E0F901EE5DFD4E8081823021F440
:10E83000A181B2814A0F5B1F6150710931F1C90199
:10E840000396FC01EE5DFD4E208101962111F9CF6A
:10E850008D3E21E0920738F09C018D3E914011F7EA
:10E86000E2E2F2E108C0FC01EE5DFD4E20812111E3
:10E87000F3CF0196EDCF9F0122523241819188233F
:10E88000D1F3D0CF80E090E00895CA010895FF92BF
:10E890000F931F93CF93DF93EC01F62E662321F0A5
:10E8A0000F9459B08C0108C0FC0101900020E9F7D9
:10E8B00031978F01081B190B003611050CF06CC045
:10E8C00060E0C80123DF882309F466C080911D122F
:10E8D00090911E12FC01EE5DFD4E23E02083039615
:10E8E000BE018E5D9D4EFF2019F00F9452B002C004
:10E8F0000F94E6BCE9EFF6E48491EF01882329F058
:10E9000070DF2196FE018491F9CFE0EAF5E1C5912F
:10E91000D491FE018491882319F063DF2196F9CF09
:10E92000C0911D12D0911E12CB5DDD4E89918823BE
:10E9300011F057DFFBCFEEE9F5E18491EF01882379
:10E9400029F04FDF2196FE018491F9CF8AE049DF5B
:10E950000C5F1F4F80911D1290911E12080F191FFE
:10E960000D3EF1E01F0729F010931E1200931D12B7
:10E9700004C010921E1210921D12809120129091CC
:10E98000211201969093211280932012DF91CF9152
:10E990001F910F91FF900895E7E7FFE484918F01A5
:10E9A000882331F01EDF0F5F1F4FF8018491F8CFED
:10E9B000E0EAF5E105911491F8018491882321F0B2
:10E9C00010DF0F5F1F4FF8CFFF2061F0FE01849131
:10E9D000882319F006DF2196F9CFE7E8F5E1849165
:10E9E000EF0105C089918823C1F3FBDEFBCF8823AB
:10E9F00029F0F7DE2196FE018491F9CF8AE0DF91BC
:10EA0000CF911F910F91FF90ECCE109210141092A5
:10EA10000F1410921E1210921D12109221121092B9
:10EA2000201210921F1208958091201290912112AD
:10EA3000181619060CF048C0019790932112809384
:10EA40002012892B79F480911B1290911C12892B32
:10EA500021F410921E1210921D1280911D1290919D
:10EA60001E122CC0E0910F14F0911014EB5DFD4EBE
:10EA7000CF018252924121912111FACF01968D3E10
:10EA800021E0920740F09093101480930F148D3E74
:10EA90009140C1F40BC0AC014F5F5F4FFC01EE5DD4
:10EAA000FD4E20812111EFCFCA01E9CFE2E2F2E170
:10EAB000CF018252924121912223D1F390931014DD
:10EAC00080930F1481E0089580E008959091B30A37
:10EAD000911107C09091C00095FFFCCF8093C600B4
:10EAE0000895913031F49091C80095FFFCCF809348
:10EAF000CE000895FC0120E03EE2DB014C91403263
:10EB000041F0283011F430833196DB014C91408381
:10EB100031962F5F6F5F7F4F2B3079F7108208950A
:10EB2000CF93809111128823B9F14091091250912D
:10EB30000A1260910B1270910C1229E030E1809161
:10EB40001212909113120E946585C82F811102C084
:10EB5000C0E023C040910D1250910E1260910F122F
:10EB600070911012411551056105710591F029E070
:10EB700030E180911212909113120E9465858823D2
:10EB800039F310920D1210920E1210920F12109271
:10EB900010121092111201C0C1E08C2FCF91089574
:10EBA000CF92DF92EF92FF92CF936B017C01C42F43
:10EBB0008091091290910A12A0910B12B0910C123F
:10EBC0008C159D05AE05BF05C9F0AADF811102C0F5
:10EBD00080E018C029E030E1B701A601809112124F
:10EBE000909113120E94C785882391F3C092091255
:10EBF000D0920A12E0920B12F0920C1281E0C11135
:10EC000080931112CF91FF90EF90DF90CF900895F5
:10EC10004F925F926F927F928F929F92AF92BF922C
:10EC2000CF92DF92EF92FF920F931F93CF93DF93D8
:10EC3000EC016A017B01280139014230510561056F
:10EC4000710510F480E064C089859A85AB85BC8528
:10EC50000196A11DB11D84179507A607B70790F36C
:10EC60008F89803149F48D2C9E2CAF2CBB248B894D
:10EC70009C89AD89BE890FC0803221F78B889C8822
:10EC8000AD88BE88DB01CA0157E0B695A795979578
:10EC900087955A95D1F7880E991EAA1EBB1E41E092
:10ECA000C501B4017DDF882369F29F89903161F449
:10ECB000DD24EE24FF249601220F331FF901E75FC4
:10ECC000FF4E5182408211C0E894C7F8DD24EE2443
:10ECD000FF249601220F331F220F331FF901E75F34
:10ECE000FF4E40825182628273829A89923080F014
:10ECF0004D815E816F817885840E951EA61EB71E9C
:10ED000080920D1290920E12A0920F12B0921012D9
:10ED1000DF91CF911F910F91FF90EF90DF90CF90F7
:10ED2000BF90AF909F908F907F906F905F904F902B
:10ED30000895CF92DF92EF92FF920F931F93CF939C
:10ED4000DF93FC0181859285A385B4850196A11D81
:10ED5000B11D84179507A607B70710F480E061C0BE
:10ED60008789803149F4BB27A72F962F852FC38829
:10ED7000D488E588F6880FC0803281F7838994892A
:10ED8000A589B6896A017B01C7E0F694E794D79418
:10ED9000C794CA95D1F78C0D9D1DAE1DBF1DE9010D
:10EDA0006A017B018F014091091250910A12609112
:10EDB0000B1270910C1284179507A607B70799F4E8
:10EDC000F80187898031B1F4B701A601552766277C
:10EDD0007727440F551FFA01E75FFF4E808191812D
:10EDE000A0E0B0E019C040E0BC01CD01D9DE811146
:10EDF000E7CFB4CFB701A6014F775527662777270E
:10EE0000440F551F440F551FFA01E75FFF4E8081E5
:10EE10009181A281B381BF7088839983AA83BB83C8
:10EE200081E0DF91CF911F910F91FF90EF90DF90E4
:10EE3000CF9008954F925F926F927F92AF92BF9260
:10EE4000CF92DF92EF92FF920F931F93CF93DF93B6
:10EE500000D01F92CDB7DEB78C0149835A836B83F4
:10EE60007C835901C12CD12C7601412C82E0582E93
:10EE7000612C712C49815A816B817C819E012F5FAD
:10EE80003F4FC80156DF882341F1D301C201F80189
:10EE9000058404C0880F991FAA1FBB1F0A94D2F7CC
:10EEA000C80ED91EEA1EFB1E49815A816B817C81E6
:10EEB0008789803139F481E0483F5F4F61057105F2
:10EEC00038F4D8CF81E0483F5F4F6F4F7F4090F2DA
:10EED000F501C082D182E282F3820F900F900F90F1
:10EEE0000F90DF91CF911F910F91FF90EF90DF90E6
:10EEF000CF90BF90AF907F906F905F904F900895AC
:10EF00002F923F924F925F926F927F928F929F9239
:10EF1000AF92BF92CF92DF92EF92FF920F931F9327
:10EF2000CF93DF9300D01F92CDB7DEB79C838B8346
:10EF30004B015A01DC0113968C91811103C08FEFB4
:10EF40009FEFE9C0EB81FC81818180FFF8CFAB812D
:10EF5000BC8151960D911D912D913C91549718961D
:10EF60004D915D916D917C911B97C501A0E0B0E042
:10EF700068017901C41AD50AE60AF70A8C159D05BD
:10EF8000AE05BF0518F05801A41AB50A75018B81AA
:10EF90009C8104969A838983612C92E0792EE114F6
:10EFA000F10409F48AC0AB81BC8118964D915D9142
:10EFB0006D917C911B976A01B1E0DB22EB81FC81B2
:10EFC00023811A012B0189E05694479437942794A2
:10EFD0008A95D1F7818D928D223061F4FC01828D6A
:10EFE000938DA48DB58DBC01CD01620D731D841D63
:10EFF000951D49C0DC0114961C9111501221C114B9
:10F00000D104F9F411111DC0452B462B472B59F49F
:10F01000EB81FC8185899689A789B08D848395834E
:10F02000A683B7830EC0AB81BC8114964D915D91D0
:10F030006D917C91179729813A817BDE882309F4B1
:10F040007ECFEB81FC81218D328D84819581A681DB
:10F05000B7810297A109B109F901058404C0880F9D
:10F06000991FAA1FBB1F0A94D2F74685578560894E
:10F070007189840F951FA61FB71FBC01CD01610FB9
:10F08000711D811D911D93012C193D0987012E15BC
:10F090003F0508F489010115F2E01F0779F5209179
:10F0A000091230910A1240910B1250910C12621702
:10F0B00073078407950719F421C0C5012CC094017A
:10F0C000AB01BC0180911212909113120E94C7856E
:10F0D000882309F434CF800E911EEB81FC8180855A
:10F0E0009185A285B385800F911FA11DB11D8087D9
:10F0F0009187A287B387E01AF10A51CF40E050DD33
:10F10000882309F41CCFB601675F7F4EA801C401B4
:10F110000F94A4BCE0CF0F900F900F900F90DF9151
:10F12000CF911F910F91FF90EF90DF90CF90BF9004
:10F13000AF909F908F907F906F905F904F903F9097
:10F140002F900895DF92EF92FF920F931F93CF932A
:10F15000DF938C01EB017A018DE0D82E40E250E084
:10F16000BE01C801CDDE8032910539F021E0892B46
:10F1700009F420E0822F819547C028812223C1F025
:10F18000253E61F32E3251F33B853F733F3061F4EE
:10F19000E114F10449F04A8D5B8D452B29F42F7160
:10F1A0003FEF320F343030F02B8523FDD7CF2CC00A
:10F1B00080E02AC030E021503109D29EC001D39EA8
:10F1C000900D1124F701E80FF91F298120832B816D
:10F1D00021832D8122832F812383298524832E85DA
:10F1E0002583288926832A8927832C8920872E89AD
:10F1F0002187288D22872C8D23872E8D2487288197
:10F2000026FFD2CF1586D0CFDF91CF911F910F91DE
:10F21000FF90EF90DF900895CF93DF93EC018B8107
:10F220008823A9F1898187FF2FC06C857D858E8514
:10F230009F8541E0B5DC882351F1E88980E2E89FB1
:10F24000F0011124DF01A75FBF4E109701F18C91EF
:10F25000853EE9F08B81823050F449895A896B8967
:10F260007C895C964D935D936D937C935F978D89BC
:10F270009E89AF89B88DE75FFF4E938F828FB58BE4
:10F28000A48B89818F778983DF91CF9149CC81E0ED
:10F29000888380E0DF91CF9108958F929F92AF9203
:10F2A000BF92CF92DF92EF92FF920F931F93CF9373
:10F2B000DF93EC018B81811102C080E076C0098967
:10F2C0001A892B893C890417150726073707A8F3E5
:10F2D0006A017B01823029F4C886D986EA86FB86DA
:10F2E0000DC0C114D104E104F10451F41C821D824B
:10F2F0001E821F82188619861A861B8681E055C0D9
:10F3000088849984AA84BB84E98DFA8D258530E0B0
:10F31000275F3F4FB501A4014150510961097109AF
:10F32000022E04C076956795579547950A94D2F7B3
:10F33000D701C6010197A109B10904C0B695A795E7
:10F34000979587952A95D2F784179507A607B7074B
:10F3500020F089288A288B2849F44D895E896F8995
:10F36000788D4C835D836E837F8304C0841B950BF3
:10F37000A60BB70B4C015D018E010C5F1F4F811472
:10F380009104A104B10409F4A7CF4C815D816E8181
:10F390007F819801898D9A8DCCDC91E0891A910842
:10F3A000A108B1088111EBCF88CFDF91CF911F91D8
:10F3B0000F91FF90EF90DF90CF90BF90AF909F9014
:10F3C0008F9008952F923F924F925F926F927F920B
:10F3D0008F929F92AF92BF92CF92DF92EF92FF9265
:10F3E0000F931F93CF93DF9300D01F92CDB7DEB75B
:10F3F0008C014B011A01DC0113968C91139781301B
:10F40000C1F411968C9181FF14C082FF18C0F801DD
:10F41000418952896389748980859185A285B385E4
:10F4200084179507A607B70751F0C80136DF811189
:10F4300006C081E0F80180838FEF9FEF2CC161014E
:10F4400085C0D80159968D919C915A97FC012481D1
:10F4500021502A013B0139E07694679457944794F0
:10F460003A95D1F7722E74207A01F1E0FF227720CD
:10F4700009F478C080E092E08E199F0956018C153E
:10F480009D0508F45C01D80159962D913C915A973D
:10F4900014968D919D910D90BC91A02D0297A1097C
:10F4A000B109F901058404C0880F991FAA1FBB1F69
:10F4B0000A94D2F74685578560897189840F951F14
:10F4C000A61FB71F9C01AD01270D311D411D511D08
:10F4D00029013A01A11432E0B30609F089C08091F4
:10F4E000091290910A12A0910B12B0910C1284157E
:10F4F0009505A605B70569F4109211128FEF9FEFDD
:10F50000DC018093091290930A12A0930B12B0931E
:10F510000C129401B301A201809112129091131266
:10F520000E946585882309F484CFF8018085918540
:10F53000A285B3858A0D9B1DA11DB11D8087918772
:10F54000A287B3878A0C9B1CCA18DB08D8011896BF
:10F550004D915D916D917C911B97C114D10409F07F
:10F5600070CF7AC0E114F10409F084CF14964D9164
:10F570005D916D917C91179741155105610571055C
:10F5800059F455968D919D910D90BC91A02D0097A9
:10F59000A105B10539F520C09E012F5F3F4FC9DBA2
:10F5A000882309F446CF89819A81AB81BC81F80117
:10F5B000218D328DF9012789203139F4883FFFEF01
:10F5C0009F07A105B10540F40DC0883F2FEF9207BA
:10F5D000A2072FE0B20730F0C8010E94C683811154
:10F5E00049CF27CFF80184839583A683B78342CF81
:10F5F000E114F10411F5D80118964D915D916D91CA
:10F600007C911B9751968D919D910D90BC91A02D51
:10F61000481759076A077B0780F082DA882309F4C4
:10F6200008CF81E0809311124092091250920A1281
:10F6300060920B1270920C1207C041E0C301B2013C
:10F64000AFDA882309F4F5CEA501B401C701875FBD
:10F650009F4E0F94A4BC69CF51968D919D910D90B2
:10F66000BC91A02D84179507A607B70740F4F801B1
:10F67000418B528B638B748B818180688183D8012D
:10F6800011968C9183FD02C0C10105C0C801C4DD83
:10F690008111FACFCECE0F900F900F900F90DF9187
:10F6A000CF911F910F91FF90EF90DF90CF90BF907F
:10F6B000AF909F908F907F906F905F904F903F9012
:10F6C0002F900895CF93DF931F92CDB7DEB7698354
:10F6D00041E050E0BE016F5F7F4F049673DE0F90F4
:10F6E000DF91CF910895CF93DF931F92CDB7DEB70F
:10F6F00041E050E0BE016F5F7F4F02DC019719F4DB
:10F70000898190E002C08FEF9FEF0F90DF91CF9142
:10F7100008952F923F924F925F926F927F928F92B5
:10F720009F92AF92BF92CF92DF92EF92FF920F9390
:10F730001F93CF93DF93CDB7DEB76F970FB6F894D3
:10F74000DEBF0FBECDBF61E08FE590E00E94867303
:10F75000882309F48EC42091B10A3091B20A8091B5
:10F76000AF0A9091B00A821B930B8F7799278F373E
:10F77000910591F43093B00A2093AF0AE2EDF5E1E0
:10F7800084918F01882331F02CD80F5F1F4FF8012F
:10F790008491F8CF8AE025D803EC15E131ECE32E13
:10F7A00035E1F32E44E2B42E8091AF0A9091B00A75
:10F7B0002091B10A3091B20A821B930B8F7799275F
:10F7C000892B09F4B2C10F94B9068F8F0F94133CA3
:10F7D0006093110C7093120C8093130C9093140C83
:10F7E0000F94133C60930D0C70930E0C80930F0CD0
:10F7F0009093100C4F8D47FDD7CF20911B12309165
:10F800001C124A3031F04D3021F02F3531050CF407
:10F8100072C12115310519F4109260082AC4C090F4
:10F820001D12D0901E122E5D3D4EF901EC0DFD1DF6
:10F83000138280916008811142C166EE73E0C601B7
:10F840008B5D9D4E0F940ABD892B09F07EC0F60199
:10F85000EE5DFD4E83818E3409F077C04AE050E0C2
:10F8600060E070E0C6018A5D9D4E0F940EAF60931C
:10F870005C0870935D0880935E0890935F084090E9
:10F880005708509058086090590870905A08A30182
:10F8900092012F5F3F4F4F4F5F4FC0901D12D0908E
:10F8A0001E12621773078407950709F4EAC16DEC0D
:10F8B00075E1C6018B5D9D4E0F9497B0892B09F0C1
:10F8C000E0C1E7E7FFE484918F01882339F00E94CB
:10F8D000F1730F5F1F4FF8018491F7CFEBECF5E167
:10F8E00005911491F8018491882329F00E94F17305
:10F8F0000F5F1F4FF7CFC301B2010F9496038AE049
:10F900000E94F1730F948DAC10921C1210921B1276
:10F91000B0C3E0915508F09156081082E0911D1295
:10F92000F0911E12EE5DFD4EB38280915C089091C5
:10F930005D08A0915E08B0915F088093570890938E
:10F940005808A0935908B0935A0880911D129091BD
:10F950001E12FC01EE5DFD4E2381AC014D5F5F4F39
:10F960006A012E3409F433C0243289F16AE270E06E
:10F97000CA018E5D9D4E0F94D2BC892B41F1E7E701
:10F98000FFE484918F01882339F00E94F1730F5FA7
:10F990001F4FF8018491F7CFE5ECF5E10591149143
:10F9A000F8018491882329F00E94F1730F5F1F4FA3
:10F9B000F7CF60915708709158088091590890913D
:10F9C0005A080F9496038AE00E94F1739DCF67E472
:10F9D00070E0C6018E5D9D4E0F94D2BC9093560888
:10F9E00080935508009781F12091270C211109C0BF
:10F9F0002AE030E03093AD082093AC0821E020935A
:10FA0000AB0820916B092223F9F04AE050E060E056
:10FA100070E001960F940EAF64307105A8F4F80100
:10FA2000C590D490F6018491882331F00E94F1733F
:10FA3000FFEFCF1ADF0AF6CF8AE00E94F173F701D9
:10FA4000859194910F94933FC0901D12D0901E12F7
:10FA500096012B5D3D4E490160E675E0C9010F94AA
:10FA6000DDBC892B29F462E080E095E00F94598792
:10FA7000F601EE5DFD4E81E08083F40101900020EF
:10FA8000E9F73197E819F90934E0C30ED11CEC0D00
:10FA9000FD1DED3E41E0F40729F0F0931E12E093C6
:10FAA0001D1204C010921E1210921D12809120127D
:10FAB000909121120196909321128093201210921E
:10FAC0001C1210921B128091AF0A9091B00A2091E3
:10FAD000B10A3091B20A821B930B8F779927892B39
:10FAE00009F4C7C261E08FE590E00E948673882325
:10FAF00009F4BFC259CE4B3319F481E080936008FA
:10FB000080916008811150CEE0911D12F0911E127B
:10FB1000C901019690931C1280931B122E0F3F1F58
:10FB2000F901EB5DFD4E40833FCE8091480F882365
:10FB300009F467C00F94133C60930D0C70930E0C86
:10FB400080930F0C9093100C0091110C1091120CDB
:10FB50002091130C3091140CDC01CB01801B910B14
:10FB6000A20BB30B81329340A105B10508F449C043
:10FB700080911B1290911C12181619060CF041C0AE
:10FB800020911D1230911E128E5D9D4EDC01A20F40
:10FB9000B31F13961C92D901AB5DBD4EFD010190C0
:10FBA0000020E9F73197EA1BFB0B2C5F3F4FE20F78
:10FBB000F31FED3E81E0F80729F0F0931E12E09369
:10FBC0001D1204C010921E1210921D12809120125C
:10FBD00090912112019690932112809320121092FD
:10FBE0001C1210921B12E8EBF5E184918F0188231F
:10FBF00009F43FC20E94F1730F5F1F4FF801849117
:10FC0000F6CF8091270C882309F433C280911B1210
:10FC100090911C12892B09F02CC280912012909196
:10FC20002112892B11F410925B0802E08CE3482E1C
:10FC3000512C612C712C92EA292E95E1392E9E01CE
:10FC40002F5F3F4F790124E0C22ED12C4091350F18
:10FC50005091360F6091370F7091380F80912D0FB2
:10FC600090912E0FA0912F0FB091300F4817590788
:10FC70006A077B0708F0FDC180915B088111F9C11B
:10FC800063C096012B5D3D4E69016AE270E0C901D7
:10FC90000F94D2BC90935608809355080097D9F4DE
:10FCA000E7E7FFE484918F01882339F00E94F17324
:10FCB0000F5F1F4FF8018491F7CFE7ECF5E1059155
:10FCC0001491F8018491882309F415CE0E94F173F0
:10FCD0000F5F1F4FF6CFF601D12CE817F90719F087
:10FCE0002191D226FACF4AE050E060E070E0CF01E7
:10FCF00001960F940EAF2D2D30E02617370709F42B
:10FD000008CEE7E7FFE484918F01882339F00E9451
:10FD1000F1730F5F1F4FF8018491F7CFE9ECF5E124
:10FD200005911491F8018491882329F00E94F173C0
:10FD30000F5F1F4FF7CF609157087091580880915F
:10FD4000590890915A08D9CD8091880E9091890ECA
:10FD5000A0918A0EB0918B0E8093350F9093360F41
:10FD6000A093370FB093380F80E89EE0BCDC182FCB
:10FD70008A30B1F01D30A1F0133211F01A3321F4A2
:10FD800020916008222361F0E0911B12F0911C1277
:10FD9000EF35F1052CF48F3F3FEF930709F04EC18B
:10FDA0004091350F5091360F6091370F7091380F99
:10FDB00080912D0F90912E0FA0912F0FB091300FA9
:10FDC000481759076A077B0708F4AEC0E6EBF5E170
:10FDD000A590B490F5018491882331F00E94F173CD
:10FDE000FFEFAF1ABF0AF6CF8AE00E94F1730F94BB
:10FDF000133C6093671A7093681A8093691A909302
:10FE00006A1A8090631A9090641AA090651AB09054
:10FE1000661ADC01CB0188199909AA09BB098090EF
:10FE20005F1A9090601AA090611AB090621ABC019B
:10FE3000CD01681979098A099B0928EE33E040E071
:10FE400050E00F9448B749015A0110925F1A10927E
:10FE5000601A1092611A1092621A60915B1A709186
:10FE60005C1A80915D1A90915E1A0F948D86C5017F
:10FE7000B401A30192010F9448B7CA01B901A301CB
:10FE800092010F9448B77F936F93C501B40120E1AD
:10FE90003EE040E050E00F9448B73F932F933F92ED
:10FEA0002F92FF92EF920F9452B1E9EFF6E4849112
:10FEB0000FB6F894DEBF0FBECDBF5F01882341F0BF
:10FEC0000E94F1733FEFA31AB30AF5018491F6CFB4
:10FED0005701F50181915F01882319F00E94F173A8
:10FEE000F8CF8AE00E94F173C7010F94A83F0F94E6
:10FEF000061B1092390F8091280C882319F00F945B
:10FF0000040A06C00F9469798091280C8111F7CFFB
:10FF10008091480F882341F086E090E00E9416FF10
:10FF2000D092680FC092670F133219F481E080936A
:10FF30005B0820911B1230911C122115310519F418
:10FF40001092600883CE8091830E882349F08090C0
:10FF5000350F9090360FA090370FB090380F03C038
:10FF6000812C912C54014091371A5091381A81E01C
:10FF700090E0841B950B880E991E80911D12909124
:10FF80001E12FC01EE5DFD4E0083818292822E5D89
:10FF90003D4EF901E80FF91F1382DC01AB5DBD4E48
:10FFA000FD0101900020E9F73197EA1BFB0BF89463
:10FFB00080912012909121120196909321128093AA
:10FFC0002012EC5F80911D1290911E128E0F911DD8
:10FFD00090931E1280931D122091830E222349F0CC
:10FFE0004091350F5091360F6091370F7091380F57
:10FFF00003C040E050E0BA014F5F5F4F6F4F7F4F4B
:020000021000EC
:100000004093371A5093381A6093391A70933A1AFA
:100010008D3E914021F410921E1210921D12789480
:100020001092600810921C1210921B1261E08FE572
:1000300090E00E948673811109CE1BC01B3321F40E
:1000400081E08093600802CE209160082111FECDEE
:1000500020911D1230911E12AF014F5F5F4F5093E0
:100060001C1240931B12E20FF31FEB5DFD4E8083C9
:10007000EDCD6F960FB6F894DEBF0FBECDBFDF910A
:10008000CF911F910F91FF90EF90DF90CF90BF9095
:10009000AF909F908F907F906F905F904F903F9028
:1000A0002F9008950F931F93CF93DF93FC0123812B
:1000B000222311F080E044C08B01EC01FB01878911
:1000C000803139F18032B1F783E08B83F801428DC2
:1000D000538D648D758D4D8B5E8B6F8B788F9E01EC
:1000E0002F5E3F4FC8010E941A77882319F31A8F99
:1000F000098F81E089831C821D821E821F821886DF
:1001000019861A861B861C861D861E861F86188ADF
:1001100017C082E08B831D8A1E8A1F8A188EFB01FE
:10012000808D918DA0E0B0E025E0880F991FAA1F77
:10013000BB1F2A95D1F7898B9A8BAB8BBC8BD7CF02
:10014000DF91CF911F910F9108958F929F92AF925F
:10015000BF92CF92DF92EF92FF920F931F93CF93B4
:10016000DF93EC018B017A01D22EDB0159968D9140
:100170009C915A979A8F898F40E050E0BA01C8014C
:100180008CD8C12CF80180859185A285B3854189E1
:1001900052896389748984179507A607B70708F001
:1001A00054C025E0B695A795979587952A95D1F7E0
:1001B000E82FEF70BE2ED80113968C91823008F490
:1001C00055C0C80190DA97FD51C0F801808591852E
:1001D000A285B3854F96A11DB11D80879187A28707
:1001E000B387F0E2BF9EC0011124BC01675F7F4E60
:1001F00061157105D9F1DB012C91222319F0253EFF
:10020000C9F46BC1C1100DC04091091250910A127E
:1002100060910B1270910C124C875D876E877F87FF
:10022000B88AFC01E75FFF4E8081882361F0CC240F
:10023000C394A8CF4BE050E0C7010F9497BC892B23
:1002400009F0A0CF15C0CC24C3948D2D82748234C4
:1002500069F4CC2009F481C0B8886C857D858E85D1
:100260009F8541E00E94D07581116BC080E038C14C
:10027000D7FCFCCF20E2B29EF00111249F01275F42
:100280003F4ED9011B968C91817121F08D2D827189
:1002900009F055C08091091290910A12A0910B1299
:1002A000B0910C128C879D87AE87BF87B88AE75FB5
:1002B000FF4E4489558960E070E0BA015527442714
:1002C0004D8B5E8B6F8B788F828D938DA0E0B0E02D
:1002D000482B592B6A2B7B2B4D8B5E8B6F8B788F2A
:1002E000D9011B968C91887151F4848D958DA68DC2
:1002F000B78D898B9A8BAB8BBC8B81E00CC0803126
:10030000F1F49E012F5E3F4F898D9A8D0E941A77DE
:100310008823A9F084E08B838D2D8F7089831C82C4
:100320001D821E821F82188619861A861B86D4FE9D
:10033000BDC0CE010F944F078111B8C097CF1B826B
:1003400095CF6889F0E26F9FB0011124675F7F4EFF
:100350006115710509F08AC089CFD80113968C9177
:100360001397823009F482CF51968D919D910D9013
:10037000BC91A02D803E9F4FAF41B10508F076CFD4
:10038000C80104D2882309F471CF0E949075882394
:1003900009F46CCFD80159962D913C915A97149637
:1003A0008D919D910D90BC91A02D0297A109B1094D
:1003B000F901058404C0880F991FAA1FBB1F0A9466
:1003C000D2F786849784A088B188880E991EAA1EC9
:1003D000BB1E81E0809311128092091290920A1242
:1003E000A0920B12B0920C1280E092E0E9E0F0E1F2
:1003F000DF019C011D9221503040E1F7CC24C394D1
:10040000D8015996ED91FC915A978481C81690F4C1
:1004100029E030E1B501A4014C0D511D611D711D94
:10042000809112129091131250D3882309F41ECF99
:10043000C394E6CF80E092E0A0E0B0E0058404C081
:10044000880F991FAA1FBB1F0A94D2F7F801418990
:10045000528963897489840F951FA61FB71F818BEA
:10046000928BA38BB48B69E070E1B12C80E2DB014D
:100470001D928A95E9F78BE0F701DB0101900D925F
:100480008A95E1F781E298E2FB01918B808B20E075
:1004900038E037872687938B828B918F808F378BBD
:1004A000268B0E9490758111E5CEE0CED5FE13C05B
:1004B00049895A896B897C89CE01DF91CF911F913F
:1004C0000F91FF90EF90DF90CF90BF90AF909F90F3
:1004D0008F900C944D7981E003C0C110A8CE94CECA
:1004E000DF91CF911F910F91FF90EF90DF90CF9010
:1004F000BF90AF909F908F9008950F931F93CF93CD
:10050000DF93EB01FC012381211102C080E040C098
:100510002250223028F48FE28883198281E038C08B
:100520008C01FC01648575858685978540E00E9475
:10053000D075882359F3F8014089F0E24F9FA0015C
:1005400011249A01275F3F4E232B01F320E030E076
:1005500090E06EE2F901E40FF51FE75FFF4E708156
:10056000703271F02830310529F4DE01A90FB11D78
:100570006C939F5FDE01A90FB11D70817C939F5F1B
:100580002F5F3F4F2B30310529F7C90FD11D18823E
:10059000DF91CF911F910F910895CF93DF93EC01DD
:1005A0000E940C791B82DF91CF9108952F923F9288
:1005B0004F925F926F927F928F929F92AF92BF9273
:1005C000CF92DF92EF92FF920F931F93CF93DF931F
:1005D000CDB7DEB7C554D1090FB6F894DEBF0FBE54
:1005E000CDBF3C015B018A01322E1C8E1F8E198209
:1005F0001C82672B11F410E0A6C0FC0183818111DD
:10060000FACFFA0180818F3261F4CA018C01019620
:10061000F80120812F32D1F3F5018381825082309D
:1006200010F475010AC0618D728DCE0101963ADD1C
:10063000882309F3CE0101967C016E019CE1C90E6D
:10064000D11C26014E01E7E38E0E911CFBE0F80D54
:100650002596FFAF2597CE01019624969FAF8EAFCA
:1006600024972696CFAE26972D2C35C080E2819315
:1006700025969FAD25979E13F9CFD80190E027E0EE
:100680004A2F3B2F8D91811128C08FA9803209F408
:10069000B2CF842F932F8C01FC01208101962F3241
:1006A000D1F3222309F449C021E0A401B701C60116
:1006B0004CDD882309F49FCFEA14FB0411F0C70135
:1006C0006CDFC414D50491F126969FAD2697822D38
:1006D0007601C92ED82EF401C9CF8F32B1F28E32F5
:1006E00019F0E8EBFFE10AC02A3009F484CF98E062
:1006F0002AE0C6CF3196381709F47DCF34913111F5
:10070000F9CF291708F477CF3FED380F3E3508F0C1
:1007100072CF31E0390FF401E90FF11D9FE9980F15
:100720009A3108F480528083932FAACF23969FADED
:10073000239724968FAD2497CBCF232DA401B70107
:10074000C30103DD182FCE0101960E945899CE01F6
:100750004C960E945899812FCB5BDF4F0FB6F894CF
:10076000DEBF0FBECDBFDF91CF911F910F91FF90E4
:10077000EF90DF90CF90BF90AF909F908F907F9041
:100780006F905F904F903F902F9008953F924F92BF
:100790005F926F927F928F929F92AF92BF92CF9211
:1007A000DF92EF92FF920F931F93CF93DF93CDB71A
:1007B000DEB72C970FB6F894DEBF0FBECDBF5C013D
:1007C000DC0159968D909C905A97F4018185928511
:1007D000A385B4859C01AD012F5F3F4F4F4F5F4F05
:1007E00029873A874B875C87D5011496CD90DD9099
:1007F000ED90FC901797C114D104E104F10439F095
:10080000BFEFCB1ADB0AEB0AFB0A312C07C0F4015D
:10081000C080D180E280F3803324339426013701F5
:100820001D821E821F821886F40181859285A38510
:10083000B4852D813E814F815885281739074A0795
:100840005B0708F064C089859A85AB85BC858C15EB
:100850009D05AE05BF0550F482E0C82ED12CE12CD9
:10086000F12C92E0492E512C612C712C9E012F5FAE
:100870003F4FB701A601C4010E949976882309F46D
:1008800046C089819A81AB81BC81892B8A2B8B2BB5
:1008900041F0260137019FEF491A590A690A790A7E
:1008A00005C0C414D504E604F70491F02D813E81FF
:1008B0004F8158852F5F3F4F4F4F5F4F2D833E83B2
:1008C0004F8358873FEFC31AD30AE30AF30AACCF2A
:1008D0000FEF1FEF2FEF3FE0B301A201C4010E9411
:1008E0000876F82E882399F0D50114964D915D91E4
:1008F0006D917C911797411551056105710549F07E
:1009000093018201C4010E940876811102C0F12C7A
:1009100029C0D50114964D925D926D927C921797E5
:10092000332051F0D301C2010196A11DB11DF40184
:1009300080839183A283B383F50185899689A789F2
:10094000B08D892B8A2B8B2B69F4D50155964D924E
:100950005D926D927C92589711968C911197806858
:1009600011968C938F2D2C960FB6F894DEBF0FBE88
:10097000CDBFDF91CF911F910F91FF90EF90DF904E
:10098000CF90BF90AF909F908F907F906F905F902F
:100990004F903F90089561E0FC0180810D94FC39F7
:1009A0008EBD0DB407FEFDCF08958FEF8EBD0DB443
:1009B00007FEFDCF8EB508950F931F93CF93DF935E
:1009C0008B010F94133CEB01F0DF8F3F49F00F9444
:1009D000133C6C1B7D0B60177107B0F380E001C006
:1009E00081E0DF91CF911F910F910895CF92DF9217
:1009F000EF92FF921F93CF93DF9300D01F92CDB75A
:100A0000DEB76C01162FFC019281892F806A8695D2
:100A10008CBD90FD03C081E0963009F480E08DBD6F
:100A200060E0F601808129833A834B835C830F94D5
:100A3000FC396CE271E0C601BFDF812F8064B0DF5A
:100A400088E1E82EF12C5C814B813A812981DA0121
:100A5000C9010E2C04C0B695A795979587950A9461
:100A6000D2F729833A834B835C839ADFF8E0EF1A4D
:100A7000F10829813A814B815C8188EFE8168FEF7C
:100A8000F80629F7112321F0183021F08FEF03C069
:100A900085E901C087E884DF1C3009F486DF10E0B7
:100AA00084DFF601838387FF04C01F3F11F01F5FBF
:100AB000F7CF0F900F900F900F90DF91CF911F9174
:100AC000FF90EF90DF90CF9008950F931F93CF93F7
:100AD000DF93EC0189018C81833039F089E0440F88
:100AE000551F661F771F8A95D1F79A01AB0168E100
:100AF000CE017CDF882311F086E02FC08EEF8EBD03
:100B000080E090E00DB407FEFDCFF801E80FF91F7B
:100B100020812EBD0DB407FEFDCF21812EBD029692
:100B2000811522E0920771F70DB407FEFDCF8FEF1C
:100B300037DF8FEF35DF39DF8B838F71853029F019
:100B400083E18983CE0127DF09C068E572E0CE0129
:100B500033DF182F811106C087E18983CE011BDFA7
:100B600010E00FC020E030E0A9016DE0CE013EDFD3
:100B7000811103C01ADF882311F086E1EECFCE0188
:100B80000ADF812FDF91CF911F910F9108952F924E
:100B90003F924F925F926F927F928F929F92AF920D
:100BA000BF92CF92DF92EF92FF920F931F93CF935A
:100BB000DF93EC014A015B0179018C81833039F0CC
:100BC00059E0880C991CAA1CBB1C5A95D1F743E02C
:100BD000542E44244A94670181E0C81A8EEFD80A43
:100BE0001701EEEF3E1A5A94A501940161E1CE017E
:100BF000FDDE882319F0F4E0F98357C00F94133C0D
:100C00008B01D3DE8B838F3F51F40F94133C601B19
:100C1000710B6D327140A8F381E189833FC08E3F33
:100C200019F0EFE0E9833AC04EBCD701F7010DB4EB
:100C300007FEFDCF8EB581934EBCEC15FD05B9F7CF
:100C40000DB407FEFDCF8EB5F6018083612C712CAB
:100C50008D91E72DFF27E827EE0FFF1FE854F24E96
:100C600085919491762C662468267926A215B30581
:100C700079F79BDE082F10E0102F002796DE082B57
:100C80006016710619F0F0E2F98308C0CE0183DE28
:100C90008D818823D1F08FEF83DE17C0CE017BDEFC
:100CA0008D81882311F08FEF7BDE552051F0CE012E
:100CB00072DE20E030E0A9016CE0CE0197DE1982FF
:100CC00092CFCE0168DE80E001C081E0DF91CF915C
:100CD0001F910F91FF90EF90DF90CF90BF90AF905A
:100CE0009F908F907F906F905F904F903F902F904C
:100CF00008959091B30A911107C09091C00095FF9B
:100D0000FCCF8093C6000895913031F49091C800D3
:100D100095FFFCCF8093CE0008958F929F92AF9263
:100D2000BF92CF92DF92EF92FF92CF93DF930F9417
:100D3000133C6B017C0120912002222309F474C032
:100D400040917202509173024130510509F46CC018
:100D500080911C0290911D02A0911E02B0911F0271
:100D600046015701881A990AAA0ABB0A30E0A8EE80
:100D7000B3E00F9474B786169706A806B9060CF46C
:100D80005BC04430510541F14CF4423051050CF444
:100D90004BC0E9EFF6E48491EF0109C045305105FD
:100DA00009F042C0E9EFF6E48491EF012BC08823FB
:100DB00029F09FDF2196FE018491F9CFE7EAFDE15A
:100DC0008491EF01882329F094DF2196FE0184911C
:100DD000F9CF8AE08EDF28C0E9EFF6E48491EF01D5
:100DE000882329F086DF2196FE018491F9CFE1E97D
:100DF000FDE18491EF01882361F37BDF2196FE0101
:100E00008491F9CF882329F074DF2196FE01849123
:100E1000F9CFEAE7FDE18491EF018823D1F269DFA0
:100E20002196FE018491F9CFC0921C02D0921D023E
:100E3000E0921E02F0921F02DF91CF91FF90EF909F
:100E4000DF90CF90BF90AF909F908F90089526E550
:100E500033E0FC013183208304960C9458996F92FF
:100E60007F928F929F92AF92BF92CF92DF92EF923A
:100E7000FF920F931F93CF93DF93CDB7DEB7C85583
:100E8000D1090FB6F894DEBF0FBECDBFB82E81E0FA
:100E90000F945C4282E00F94EB40E091AB0FF0E0E6
:100EA000EE0FFF1FEA58F24E859194910F94933FF5
:100EB0008DE99FE00F9400B76093E90F7093EA0FFC
:100EC0008093EB0F9093EC0F81EA9FE00F9400B7B3
:100ED0006093ED0F7093EE0F8093EF0F9093F00FF0
:100EE0008DE89FE00F9400B76B017C0183E79FE0E2
:100EF0000F9405B78C012AE037ED43E25FE3C701A9
:100F0000B6010F9484B76B017C0187E094E0801BED
:100F1000910B74E0969587957A95E1F7BC0180E096
:100F200090E00F9485B120911A0B30911B0B4091EA
:100F30001C0B50911D0B0F9472B89B01AC01C701A3
:100F4000B6010F9484B76093F10F7093F20F809302
:100F5000F30F9093F40F82E79FE00F94F8B6882385
:100F600099F18EE69FE00F9400B76093F50F7093B0
:100F7000F60F8093F70F9093F80F8AE29CE19F930E
:100F80008F939E012F5F3F4F79013F932F930F94D3
:100F900052B1F70101900020E9F78F0101501109CA
:100FA0006091F50F7091F60F8091F70F9091F80F07
:100FB00023E046E00F9488AD60E0C7010E944774CB
:100FC0000F900F900F900F9080E1E9EEFFE0A3E00B
:100FD000B5E101900D928A95E1F7E8EFFBE184918C
:100FE0008F01882331F085DE0F5F1F4FF801849158
:100FF000F8CFE1E9FBE184918F01882331F079DEBC
:101000000F5F1F4FF8018491F8CF6091E90F709145
:10101000EA0F8091EB0F9091EC0F43E00F94B10336
:10102000EEE8FBE184918F01882331F062DE0F5FEF
:101030001F4FF8018491F8CF6091ED0F7091EE0F82
:101040008091EF0F9091F00F43E00F94B103EBE824
:10105000FBE184918F01882331F04BDE0F5F1F4F3E
:10106000F8018491F8CF6091F10F7091F20F8091A7
:10107000F30F9091F40F43E00F94B103E9E8FBE123
:1010800084918F01882331F034DE0F5F1F4FF80108
:101090008491F8CF8AE02DDE0F94495B1092480BC3
:1010A00045E7E42E4FE0F42EA12C53E0952E6E017F
:1010B000FFE1CF0ED11C882483948A2D692D0F94D3
:1010C0001BBC082F792E42E050E0B701C6010F94F7
:1010D000E8B66F8D78A16115710511F08092480B0B
:1010E00027E0020380011124070D111D77FC1A95DA
:1010F000000F111F000F111F085B144F072E000C6B
:10110000880B990B0F9487B12FE632E143E85AE33D
:101110000F94D4ACF8016183728383839483A39486
:10112000F2E0EF0EF11C29E0A212C7CF8091480B2C
:1011300081110F94D34A0F949850E090F10FF090E2
:10114000F20F0091F30F1091F40F2091ED0F3091F9
:10115000EE0F4091EF0F5091F00F6091E90F7091F9
:10116000EA0F8091EB0F9091EC0F0F94D94C81E036
:1011700080937A08179880937B08169880937C0850
:101180001598E6ECFBE184918F01882331F0B1DD05
:101190000F5F1F4FF8018491F8CFEEEAFBE18491D5
:1011A0008F01882331F0A5DD0F5F1F4FF801849177
:1011B000F8CF0F94D96F43E00F94B103EBEAFBE152
:1011C00084918F01882331F094DD0F5F1F4FF80168
:1011D0008491F8CF81E00F94D96F43E00F94B1036D
:1011E000E8EAFBE184918F01882331F082DD0F5F13
:1011F0001F4FF8018491F8CF82E00F94D96F43E03C
:101200000F94B103E6EAFBE184918F01882331F06A
:1012100070DD0F5F1F4FF8018491F8CF8AE069DD20
:101220008CE89FE00F94F8B6182F90E0E091141529
:10123000F0E0EE0FFF1FEA56F74F918380838BE8B3
:101240009FE00F94F8B6282F30E030939508209354
:1012500094081F921F938DE69DE19F938F93DF92D9
:10126000CF920F9452B160E0C6010E944774809102
:1012700095088F93809194088F9384E69DE19F93C6
:101280008F93DF92CF920F9452B160E0C6010E941B
:1012900047740FB6F894DEBF0FBECDBF20E030E03C
:1012A00048EC51E46091F10F7091F20F8091F30FCF
:1012B0009091F40F0F9481B187FF05C061E088E53C
:1012C0009DE10E94477461E080E59DE10E944774C2
:1012D000E0911415F0E0EE0FFF1FEA56F74F818101
:1012E0008F9380818F9387E49DE19F938F93DF920B
:1012F000CF920F9452B160E0C6010E944774809172
:1013000095088F93809194088F938EE39DE19F932E
:101310008F93DF92CF920F9452B160E0C6010E948A
:10132000477461E08AE39DE10E9447740FB6F89428
:10133000DEBF0FBECDBFB11005C061E08FE29DE101
:101340000E94477461E083E29DE10E94477460E07F
:1013500085EA9FE00F940AB7EBE0FDE184918F01ED
:10136000882331F0C6DC0F5F1F4FF8018491F8CF5E
:10137000E2EFFCE184918F01882331F0BADC0F5F4A
:101380001F4FF8018491F8CF6091E90F7091EA0F37
:101390008091EB0F9091EC0F0F94F306E9EDFCE1D7
:1013A00084918F01882331F0A4DC0F5F1F4FF80177
:1013B0008491F8CF6091ED0F7091EE0F8091EF0F57
:1013C0009091F00F0F94F30688E89FE00F94F8B621
:1013D000D82EBE01695A7F4F89E89FE00E9432EC07
:1013E000EBE9FCE184918F01882331F082DC0F5F0F
:1013F0001F4FF8018491F8CF69968EAD9FAD699724
:101400000F94E7068AE59FE00F94F8B6E82EF12CDA
:10141000C7010F94E7060AE01FE0A12CB12CAE141F
:10142000BF0424F59E01265B3F4F4901380138E097
:10143000630E711CC8010F94F8B6F40181934F013B
:101440000F5F1F4F06151705A9F763961FAE639729
:10145000CE01865B9F4F0F94DB06CE01865B9F4FCC
:101460000F947A7CFFEFAF1ABF0AD9CF8E01035CCD
:101470001F4F4801E12CF12CC02EB12EC7018B5615
:10148000904F0F94F8B6F40181934F01FFEFEF1ADC
:10149000FF0A28E0E216F10489F726961FAE269788
:1014A000F80181918F01882311F023DCF9CF66E9DF
:1014B0007CE18C2D9B2D0F9447B0BF92CF928FE88B
:1014C0009CE19F938F938E010F5F1F4F1F930F938C
:1014D0000F9452B10F900F900F900F900F900F90AC
:1014E0007E01F5E0EF0EF11CF7018081882349F0C1
:1014F000082E000C990B0F948FBCF70181937F018C
:10150000F3CF60E0C8010E94477481E99FE00F9427
:1015100000B7C62EB72EA82E992EE4E7FCE18491E1
:101520007F01882339F0E5DBFFEFEF1AFF0AF701AF
:101530008491F7CF4AE06C2D7B2D8A2D992D0F9445
:101540000F030F94D50661E080E79CE10E94477489
:101550006BE67CE1C8010F9452B08DE99FE00F94D7
:1015600000B767966CAF7DAF8EAF9FAF6797CE0128
:101570008D5A9F4F0F946E3EBC01C8010F94C7BC9B
:1015800068E67CE1C8010F9447B081EA9FE00F94C0
:1015900000B767966CAF7DAF8EAF9FAF6797CE01F8
:1015A0008D5A9F4F0F946E3EBC01C8010F94C7BC6B
:1015B00061E67CE1C8010F9447B060E0C8010E9479
:1015C00047746CE57CE1C8010F9452B08DE89FE050
:1015D0000F9400B767966CAF7DAF8EAF9FAF6797E4
:1015E000CE018D5A9F4F0F946E3EBC01C8010F94DF
:1015F000C7BC60E0C8010E94477461E08FE49CE1D1
:101600000E94477469968FAD69978F9368968FADE6
:1016100068978F9388E49CE19F938F931F930F9318
:101620000F9452B160E0C8010E94477482E79FE0C6
:101630000F94F8B60F900F900F900F900F900F909F
:10164000882329F061E084E49CE10E9447746DE303
:101650007CE1C8010F9452B02D2D30E065963FAF6C
:101660002EAF6597CE018D5A9F4F0F94243DBC013C
:10167000C8010F94C7BC60E0C8010E9447749F92E4
:10168000AF92BF92CF9284E39CE19F938F931F937D
:101690000F930F9452B160E0C8010E94477461E05B
:1016A00080E39CE10E944774EFEBFCE184910FB66C
:1016B000F894DEBF0FBECDBF8F01882331F019DB58
:1016C0000F5F1F4FF8018491F8CF6091F10F709177
:1016D000F20F8091F30F9091F40F42E00F94B10359
:1016E000E5EAFCE184918F01882331F002DB0F5F92
:1016F0001F4FF8018491F8CF6091F50F7091F60FAC
:101700008091F70F9091F80F42E00F94B103C85AFF
:10171000DF4F0FB6F894DEBF0FBECDBFDF91CF9184
:101720001F910F91FF90EF90DF90CF90BF90AF90FF
:101730009F908F907F906F9008951F920F920FB699
:101740000F9211240BB60F922F923F924F925F92FD
:101750006F927F928F929F92AF92BF92CF92DF92C1
:10176000EF92FF920F931F932F933F934F935F93AB
:101770006F937F938F939F93AF93BF93EF93FF9359
:10178000CF93DF93CDB7DEB76197DEBFCDBFEC98C7
:10179000E4E8FBE184918F01882331F0AADA0F5F3E
:1017A0001F4FF8018491F8CF8AE0A3DA8091270CCB
:1017B000882309F483C20F94133C6D877E878F873B
:1017C000988BF091270CF98B179A10927A08169A39
:1017D00010927B08149A64E182E00F940BA164E1FB
:1017E00082E00F94D9A064E183E00F940BA164E13F
:1017F00083E00F94D9A00F945F7C98878F834090EB
:10180000371A5090381A6090391A70903A1A0F941B
:10181000E378481A590A610871080E940574481A49
:10182000590A6108710877FE03C0412C512C32011E
:101830009091361A8091351A981799F0E091351ADF
:1018400022E5E29FF0011124EB5EFA4E20E030E049
:1018500040E752E462A173A184A195A10F94D4AC96
:1018600008C06091860270918702809188029091F1
:1018700089020F94E3B87E836D830F942E3683E044
:101880000F94D96FAB01BC018EE69FE00F941CB79B
:1018900060911F0981E0682782E79FE00F940AB7F3
:1018A0000E9405751092270C789420E030E040E803
:1018B0005FE36091F50F7091F60F8091F70F9091B3
:1018C000F80F0F9483B769837A838B839C83E090AE
:1018D000F10FF090F20F0091F30F1091F40F20919F
:1018E000ED0F3091EE0F4091EF0F5091F00F60919E
:1018F000E90F7091EA0F8091EB0F9091EC0FE4E10A
:101900002E2EE5E13E2E3F922F92812C912CFEEB64
:10191000AF2EF2E4BF2EFE0131966F010F949D2889
:101920000F94EC6F149A20E030E040E85FE36091A0
:10193000F50F7091F60F8091F70F9091F80F0F94BB
:1019400083B769837A838B839C8367E074E02F81FC
:101950003885621B730BA4E076956795AA95E1F72D
:1019600080E090E00F9485B169877A878B879C87A8
:101970002AE037ED43E25FE36091F10F7091F20FDF
:101980008091F30F9091F40F0F9484B76B017C0159
:1019900020911A0B30911B0B40911C0B50911D0B89
:1019A00069857A858B859C850F9472B89B01AC0103
:1019B000C701B6010F9484B77B018C012091ED0F14
:1019C0003091EE0F4091EF0F5091F00F6091E90FC1
:1019D0007091EA0F8091EB0F9091EC0F3F922F9254
:1019E000812C912CB0E2AB2EB2E4BB2EFE013196DD
:1019F0006F010F949D280F94EC6F149A20E030E053
:101A000040E85FE36091F50F7091F60F8091F70F5A
:101A10009091F80F0F9483B769837A838B839C83AB
:101A20002AE037ED43E25FE36091F10F7091F20F2E
:101A30008091F30F9091F40F0F9484B76B017C01A8
:101A400020911A0B30911B0B40911C0B50911D0BD8
:101A500069857A858B859C850F9472B89B01AC0152
:101A6000C701B6010F9484B77B018C012091ED0F63
:101A70003091EE0F4091EF0F5091F00F6091E90F10
:101A80007091EA0F8091EB0F9091EC0F3F922F92A3
:101A9000FE0131966F010F949D280F94EC6F149AFC
:101AA000B301A20181E99FE00F941CB70F900F9042
:101AB0000F900F900F900F9005E71FE0712C83E0BF
:101AC000682E872D662D0F941BBC2091480B222376
:101AD00021F125E18202F001112433E09302E00DAF
:101AE000F11D1124EE0FFF1FEE0FFF1FE85BF44FF7
:101AF00020E030E04AE754E461817281838194817F
:101B00000F94D4AC20E030E040E05FE30F9484B762
:101B10000F9418B90F94E3B802C060E070E0C801F8
:101B20000F9424B773940E5F1F4F49E07412C9CF0E
:101B30006F81788583E79FE00F9424B74091E90F88
:101B40005091EA0F6091EB0F7091EC0F8DE99FE0DF
:101B50000F941CB74091ED0F5091EE0F6091EF0F75
:101B60007091F00F81EA9FE00F941CB74091F10F44
:101B70005091F20F6091F30F7091F40F8DE89FE098
:101B80000F941CB7BE016B5F7F4F89E89FE00E94F6
:101B900048ECE0911415F0E0EE0FFF1FEA56F74F06
:101BA00060818CE89FE00F940AB7609194088BE8FD
:101BB0009FE00F940AB76091A80F88E89FE00F9408
:101BC0000AB75989552329F061E085EA9FE00F940F
:101BD0000AB70F94EC6FEFE7FBE184918F01882344
:101BE00031F087D80F5F1F4FF8018491F8CF0F9421
:101BF0005F7C0F94ED0684E69FE00F94F8B661E0F9
:101C0000680F84E69FE00F940AB7E4E7FBE1849154
